:020000040801F1
:1000000020C900206D3B0108C9620508593B010861
:10001000593B0108593B0108593B0108593B01086C
:10002000000000000000000000000000C53B0108C7
:10003000593B010800000000113E01081DA5010800
:10004000CD3E0108CD3E0108CD3E0108CD3E010860
:10005000CD3E0108CD3E0108CD3E0108CD3E010850
:10006000CD3E0108CD3E0108CD3E0108CD3E010840
:10007000CD3E0108CD3E0108CD3E0108CD3E010830
:10008000CD3E0108CD3E0108CD3E0108CD3E010820
:10009000CD3E0108CD3E0108CD3E0108CD3E010810
:1000A000CD3E0108CD3E0108CD3E0108CD3E010800
:1000B000CD3E0108CD3E0108CD3E0108CD3E0108F0
:1000C000CD3E0108CD3E0108CD3E0108CD3E0108E0
:1000D000CD3E0108CD3E0108CD3E0108CD3E0108D0
:1000E000CD3E0108CD3E0108CD3E0108CD3E0108C0
:1000F000CD3E0108CD3E0108CD3E0108CD3E0108B0
:10010000CD3E0108CD3E0108CD3E0108CD3E01089F
:10011000CD3E0108CD3E0108CD3E0108CD3E01088F
:10012000CD3E0108CD3E0108CD3E0108CD3E01087F
:10013000CD3E0108CD3E0108CD3E0108CD3E01086F
:10014000CD3E0108CD3E0108CD3E0108CD3E01085F
:10015000CD3E0108CD3E0108CD3E0108CD3E01084F
:10016000CD3E0108CD3E0108CD3E0108CD3E01083F
:10017000CD3E0108CD3E0108CD3E0108CD3E01082F
:10018000CD3E0108CD3E0108CD3E0108CD3E01081F
:10019000CD3E0108CD3E0108CD3E0108CD3E01080F
:1001A000CD3E0108CD3E0108CD3E0108CD3E0108FF
:1001B000CD3E0108CD3E0108CD3E0108CD3E0108EF
:1001C000CD3E0108CD3E0108CD3E0108CD3E0108DF
:1001D000CD3E0108CD3E0108CD3E0108CD3E0108CF
:1001E000CD3E0108CD3E0108CD3E0108CD3E0108BF
:1001F000CD3E0108CD3E0108CD3E0108CD3E0108AF
:08020000CD3E0108CD3E0108CE
:1002080081F0004102E000BF83F0004330B54FEABF
:1002180041044FEA430594EA050F08BF90EA020F2C
:100228001FBF54EA000C55EA020C7FEA645C7FEABF
:10023800655C00F0E2804FEA5454D4EB5555B8BFE2
:100248006D420CDD2C4480EA020281EA030382EA53
:10025800000083EA010180EA020281EA0303362DE5
:1002680088BF30BD11F0004F4FEA01314FF4801CB8
:100278004CEA113102D0404261EB410113F0004FCA
:100288004FEA03334CEA133302D0524263EB430381
:1002980094EA050F00F0A780A4F10104D5F1200E1F
:1002A8000DDB02FA0EFC22FA05F2801841F100017A
:1002B80003FA0EF2801843FA05F359410EE0A5F14E
:1002C80020050EF1200E012A03FA0EFC28BF4CF07F
:1002D800020C43FA05F3C01851EBE37101F0004535
:1002E80007D54FF0000EDCF1000C7EEB00006EEB42
:1002F8000101B1F5801F1BD3B1F5001F0CD34908CC
:100308005FEA30004FEA3C0C04F101044FEA445222
:1003180012F5800F80F09A80BCF1004F08BF5FEAA9
:10032800500C50F1000041EB045141EA050130BD89
:100338005FEA4C0C404141EB0101013C28BFB1F59B
:10034800801FE9D291F0000F04BF01460020B1FAE6
:1003580081F308BF2033A3F10B03B3F120020CDAB9
:100368000C3208DD02F1140CC2F10C0201FA0CF097
:1003780021FA02F10CE002F11402D8BFC2F1200CFC
:1003880001FA02F120FA0CFCDCBF41EA0C019040B2
:10039800E41AA2BF01EB0451294330BD6FEA0404FB
:1003A8001F3C1CDA0C340EDC04F11404C4F12002E6
:1003B80020FA04F001FA02F340EA030021FA04F3F8
:1003C80045EA030130BDC4F10C04C4F1200220FA4F
:1003D80002F001FA04F340EA0300294630BD21FA8D
:1003E80004F0294630BD94F0000F83F4801306BF53
:1003F80081F480110134013D4EE77FEA645C18BF47
:100408007FEA655C29D094EA050F08BF90EA020FDD
:1004180005D054EA000C04BF1946104630BD91EAD5
:10042800030F1EBF0021002030BD5FEA545C05D1D8
:100438004000494128BF41F0004130BD14F5800417
:100448003CBF01F5801130BD01F0004545F0FE418B
:1004580041F470014FF0000030BD7FEA645C1ABFC0
:10046800194610467FEA655C1CBF0B46024650EAF7
:10047800013406BF52EA033591EA030F41F4002123
:1004880030BD00BF90F0000F04BF0021704730B5A9
:100498004FF4806404F132044FF000054FF000017E
:1004A80050E700BF90F0000F04BF0021704730B53F
:1004B8004FF4806404F1320410F0004548BF404214
:1004C8004FF000013EE700BF42004FEAE2014FEA69
:1004D80031014FEA02701FBF12F07F4393F07F4F44
:1004E80081F06051704732F07F4208BF704793F047
:1004F8007F4F04BF41F40021704730B54FF460745A
:1005080001F0004521F000411CE700BF50EA01025C
:1005180008BF704730B54FF000050AE050EA010205
:1005280008BF704730B511F0004502D5404261EB75
:1005380041014FF4806404F132045FEA915C3FF4B6
:10054800D8AE4FF003025FEADC0C18BF03325FEA53
:10055800DC0C18BF033202EBDC02C2F1200300FA04
:1005680003FC20FA02F001FA03FE40EA0E0021FA29
:1005780002F11444BDE600BF70B54FF0FF0C4CF417
:10058800E06C1CEA11541DBF1CEA135594EA0C0FC9
:1005980095EA0C0F00F0DEF82C4481EA030621EA04
:1005A8004C5123EA4C5350EA013518BF52EA03353F
:1005B80041F4801143F4801338D0A0FB02CE4FF0F1
:1005C8000005E1FB02E506F00042E0FB03E54FF021
:1005D8000006E1FB03569CF0000F18BF4EF0010E19
:1005E800A4F1FF04B6F5007F64F5407404D25FEA15
:1005F8004E0E6D4146EB060642EAC62141EA5551C8
:100608004FEAC52040EA5E504FEACE2EB4F1FD0C09
:1006180088BFBCF5E06F1ED8BEF1004F08BF5FEA87
:10062800500E50F1000041EB045170BD06F0004639
:1006380046EA010140EA020081EA0301B4EB5C04E6
:10064800C2BFD4EB0C0541EA045170BD41F48011DE
:100658004FF0000E013C00F3AB8014F1360FDEBF03
:10066800002001F0004170BDC4F10004203C35DADF
:100678000C341BDC04F11404C4F1200500FA05F362
:1006880020FA04F001FA05F240EA020001F0004203
:1006980021F0004110EBD37021FA04F642EB060179
:1006A8005EEA430E08BF20EAD37070BDC4F10C04A3
:1006B800C4F1200500FA04F320FA05F001FA04F267
:1006C80040EA020001F0004110EBD37041F1000153
:1006D8005EEA430E08BF20EAD37070BDC4F120055E
:1006E80000FA05F24EEA020E20FA04F301FA05F2C6
:1006F80043EA020321FA04F001F0004121FA04F26E
:1007080020EA020000EBD3705EEA430E08BF20EA3D
:10071800D37070BD94F0000F0FD101F00046400077
:1007280041EB010111F4801F08BF013CF7D041EAF9
:10073800060195F0000F18BF704703F000465200FD
:1007480043EB030313F4801F08BF013DF7D043EACE
:100758000603704794EA0C0F0CEA135518BF95EA84
:100768000C0F0CD050EA410618BF52EA4306D1D10B
:1007780081EA030101F000414FF0000070BD50EA2A
:10078800410606BF1046194652EA430619D094EAB4
:100798000C0F02D150EA013613D195EA0C0F05D19E
:1007A80052EA03361CBF104619460AD181EA0301F2
:1007B80001F0004141F0FE4141F470014FF00000AA
:1007C80070BD41F0FE4141F4780170BD70B54FF045
:1007D800FF0C4CF4E06C1CEA11541DBF1CEA1355C5
:1007E80094EA0C0F95EA0C0F00F0A7F8A4EB0504A7
:1007F80081EA030E52EA03354FEA013100F088809E
:100808004FEA03334FF0805545EA131343EA126366
:100818004FEA022245EA111545EA10654FEA00261B
:100828000EF000419D4208BF964244F1FD0404F5D4
:10083800407402D25B084FEA3202B61A65EB030530
:100848005B084FEA32024FF480104FF4002CB6EBED
:10085800020E75EB030E22BFB61A754640EA0C006D
:100868005B084FEA3202B6EB020E75EB030E22BFAD
:10087800B61A754640EA5C005B084FEA3202B6EBEE
:10088800020E75EB030E22BFB61A754640EA9C00AD
:100898005B084FEA3202B6EB020E75EB030E22BF7D
:1008A800B61A754640EADC0055EA060E18D04FEA3B
:1008B800051545EA16754FEA06164FEAC30343EADB
:1008C80052734FEAC2025FEA1C1CC0D111F4801FA8
:1008D8000BD141EA00014FF000004FF0004CB6E7A1
:1008E80011F4801F04BF01430020B4F1FD0C88BF40
:1008F800BCF5E06F3FF6AFAEB5EB030C04BFB6EB4B
:10090800020C5FEA500C50F1000041EB045170BD3D
:100918000EF0004E4EEA113114EB5C04C2BFD4EB6A
:100928000C0541EA045170BD41F480114FF0000EEE
:10093800013C90E645EA060E8DE60CEA135594EA6A
:100948000C0F08BF95EA0C0F3FF43BAF94EA0C0F6D
:100958000AD150EA01347FF434AF95EA0C0F7FF4E2
:1009680025AF104619462CE795EA0C0F06D152EA36
:1009780003353FF4FDAE1046194622E750EA41061A
:1009880018BF52EA43067FF4C5AE50EA41047FF42B
:100998000DAF52EA43057FF4EBAE12E74FF0FF3C90
:1009A80006E000BF4FF0010C02E000BF4FF0010C61
:1009B8004DF804CD4FEA410C7FEA6C5C4FEA430CDA
:1009C80018BF7FEA6C5C1BD001B050EA410C0CBF29
:1009D80052EA430C91EA030F02BF90EA020F00208B
:1009E800704710F1000F91EA030F58BF994208BFF2
:1009F80090422CBFD8176FEAE37040F001007047AF
:100A08004FEA410C7FEA6C5C02D150EA013C07D105
:100A18004FEA430C7FEA6C5CD6D152EA033CD3D050
:100A28005DF8040B704700BF8446104662468C464A
:100A38001946634600E000BF01B5FFF7B7FF00287D
:100A480048BF10F1000F01BD4DF808EDFFF7F4FFA6
:100A58000CBF012000205DF808FB00BF4DF808ED31
:100A6800FFF7EAFF34BF012000205DF808FB00BF54
:100A78004DF808EDFFF7E0FF94BF012000205DF876
:100A880008FB00BF4DF808EDFFF7CEFF94BF01202B
:100A980000205DF808FB00BF4DF808EDFFF7C4FF24
:100AA80034BF012000205DF808FB00BF4FEA410277
:100AB80012F5001215D211D56FF47873B3EB6252A8
:100AC80012D94FEAC12343F0004343EA505311F0CF
:100AD800004F23FA02F018BF404270474FF0000061
:100AE800704750EA013005D111F0004008BF6FF09F
:100AF800004070474FF00000704700BF4FEA4102C6
:100B0800B2F1E04324BFB3F5001CDCF1FE5C0DD963
:100B180001F0004C4FEAC0024CEA5070B2F1004FAD
:100B280040EB830008BF20F00100704711F0804FB0
:100B380021D113F13872BCBF01F00040704741F475
:100B480080114FEA5252C2F11802C2F1200C10FA79
:100B58000CF320FA02F018BF40F001004FEAC1235D
:100B68004FEAD32303FA0CFC40EA0C0023FA02F301
:100B78004FEA4303CCE77FEA625307D150EA0133D7
:100B88001EBF4FF0FE4040F44000704701F00040A7
:100B980040F0FE4040F40000704700BF80F0004085
:100BA80002E000BF81F0004142001FBF5FEA41033D
:100BB80092EA030F7FEA226C7FEA236C6AD04FEA3D
:100BC8001262D2EB1363C1BFD21841404840414082
:100BD800B8BF5B42192B88BF704710F0004F40F434
:100BE800000020F07F4018BF404211F0004F41F450
:100BF800000121F07F4118BF494292EA030F3FD01C
:100C0800A2F1010241FA03FC10EB0C00C3F120032E
:100C180001FA03F100F0004302D5494260EB4000BD
:100C2800B0F5000F13D3B0F1807F06D340084FEA28
:100C3800310102F10102FE2A51D2B1F1004F40EB1D
:100C4800C25008BF20F0010040EA03007047490085
:100C580040EB0000013A28BFB0F5000FEDD2B0FA22
:100C680080FCACF1080CB2EB0C0200FA0CF0AABF45
:100C780000EBC25052421843BCBFD04018437047E3
:100C880092F0000F81F4000106BF80F400000132E9
:100C9800013BB5E74FEA41037FEA226C18BF7FEAC0
:100CA800236C21D092EA030F04D092F0000F08BF02
:100CB8000846704790EA010F1CBF0020704712F0E9
:100CC8007F4F04D1400028BF40F00040704712F128
:100CD80000723CBF00F50000704700F0004343F08D
:100CE800FE4040F4000070477FEA226216BF0846C3
:100CF8007FEA23630146420206BF5FEA412390EA86
:100D0800010F40F4800070474FF0000304E000BF7B
:100D180010F0004348BF40425FEA000C08BF70472C
:100D280043F0964301464FF000001CE050EA0102F0
:100D380008BF70474FF000030AE000BF50EA010205
:100D480008BF704711F0004302D5404261EB4101F2
:100D58005FEA010C02BF84460146002043F0B64317
:100D680008BFA3F18053A3F50003BCFA8CF2083A3C
:100D7800A3EBC25310DB01FA02FC634400FA02FC45
:100D8800C2F12002BCF1004F20FA02F243EB02004C
:100D980008BF20F00100704702F1200201FA02FCAE
:100DA800C2F1200250EA4C0021FA02F243EB0200A1
:100DB80008BF20EADC7070477BB972B90029BEBF52
:100DC80000204FF0004106E008BF00281CBF6FF06C
:100DD80000414FF0FF3000F077B8ADF1080C6DE935
:100DE80004CE002909DB002B1ADB00F0A9F8DDF896
:100DF80004E0DDE9022304B07047404261EB4101A1
:100E0800002B1BDB00F09CF8DDF804E0DDE9022391
:100E180004B0404261EB4101524263EB4303704727
:100E2800524263EB430300F08BF8DDF804E0DDE9A0
:100E3800022304B0404261EB41017047524263EB28
:100E4800430300F07DF8DDF804E0DDE9022304B097
:100E5800524263EB4303704753B94AB9002908BFAC
:100E680000281CBF4FF0FF314FF0FF3000F02CB8C6
:100E7800ADF1080C6DE904CE00F062F8DDF804E08D
:100E8800DDE9022304B07047D0B5FFF71DFB00224F
:100E98000B4B06460F46FFF76FFB00F017F80446AA
:100EA800FFF7F0FA0022074BFFF766FB02460B46F6
:100EB80030463946FFF7A8F900F008F82146D0BDBA
:100EC8000000F03D0000F041704700BF4A0011D219
:100ED80012F5001211D20DD56FF47873B3EB62528C
:100EE8000ED44FEAC12343F0004343EA505323FA98
:100EF80002F070474FF00000704750EA013002D10D
:100F08004FF0FF3070474FF00000704710F8012B8A
:100F180011F8013B012A28BF9A42F7D0D01A70472E
:100F2800034611F8012B03F8012B002AF9D1704769
:100F3800034613F8012B002AFBD1181A0138704711
:100F48002DE9F0478C468E46089E154604461946FC
:100F5800002B40F0D080724547D9B2FA82F74FB1E2
:100F6800C7F120030EFA07FCBD40BC4020FA03F38A
:100F780043EA0C0C4FEA154EA8B2230CBCFBFEF852
:100F88000EFB18CC08FB00F943EA0C43994528D915
:100F9800EB1808F1FF3204D2994502D9A8F10202F0
:100FA8002B44A3EB0903A4B2B3FBFEFC0EFB1C33DA
:100FB8000CFB00F044EA0344A04214D92C190CF1AC
:100FC800FF3304D2A04202D9ACF102032C44241A04
:100FD80043EA02401EB1FC40002334607360BDE860
:100FE800F0874246DDE76346F1E7002A79D0B2FA96
:100FF80082F3002B3FD01946C1F1200302FA01F514
:1010080000FA01F42EFA03F20EFA01FE20FA03F3B5
:10101800AFB243EA0E034FEA154EB2FBFEFC0EFBDD
:101028001C201A0C0CFB07F842EA004290455AD9DA
:10103800AA180CF1FF3004D2904502D9ACF1020095
:101048002A44A2EB08029BB2B2FBFEFC0EFB1C2258
:101058000CFB07F743EA02439F4246D9EB180CF111
:10106800FF3204D29F4202D9ACF102022B44DB1BAF
:1010780042EA004202E0AEEB020301224FEA154EBB
:10108800AFB2200CB3FBFEFC0EFB1C330CFB07F8C5
:1010980040EA034398452AD9EB180CF1FF3004D2F3
:1010A800984502D9ACF102002B44A3EB0803A4B283
:1010B800B3FBFEFC0EFB1C330CFB07F744EA0344AE
:1010C800A74216D92C190CF1FF3304D2A74202D932
:1010D800ACF102032C44E41B43EA00400F461146DE
:1010E80078E71F2188E76046ABE76246BFE76046BE
:1010F800DBE76346EFE7734506D916B900210846D2
:101108006DE7C6E9000EF9E7B3FA83F787B97345C7
:1011180001D3824207D8841A6EEB030301209C4650
:101128001EB900215BE73846FAE7C6E9004CF8E744
:10113800C7F1200CBB4000FA07F422FA0CF520FA9C
:101148000CF1BA401D432EFA0CF30EFA07FE4FEAD3
:10115800154941EA0E011FFA85FEB3FBF9F809FBB0
:1011680018300B0C08FB0EFA43EA00439A4540D9A5
:10117800EB1808F1FF3004D29A4502D9A8F1020011
:101188002B44A3EB0A0389B2B3FBF9F809FB183324
:1011980008FB0EFE41EA03418E452CD9691808F177
:1011A800FF3304D28E4502D9A8F10203294443EA49
:1011B8000040A1EB0E01A0FB02984145CE464346F4
:1011C80002D306D14C4504D20138B9EB020E68EBC4
:1011D8000503002EA5D0B4EB0E0261EB030101FA62
:1011E8000CFC22FA07F3F9404CEA0303C6E9003184
:1011F80097E74046C5E74346D9E7000000000000EE
:101208002DE9F04F984685B000F15803C0E9163330
:10121800129B0026838104239FED257B073222F051
:10122800070A0374119B01EB0A090F4680ED087B3E
:101238004946C0E9066686608373C6730446DDF8CE
:1012480038B002F03BFA109BC51D25F00705C4F81D
:101258008850C4E9207A02930F9BA9EB0505CDE9D4
:1012680000B32A4643463946204602F031FD0F9B1B
:10127800C4E91B8B6367109B6665A367EFF3118254
:10128800102383F31288BFF36F8F0B4B596A5C628C
:10129800E16782F31188BFF36F8F9B680BB1D3F8B6
:1012A8008C302846C4F88C3005B0BDE8F08F00BFFC
:1012B80000000000000000009C3B0020000000002F
:1012C8002DE9F0412DED028B90F8A5300446B0EEE3
:1012D800408A86B01BB9F7EE007A37EEC08AD4F898
:1012E80084202F4B9A4213D118EE100AFFF7ECF81E
:1012F80029A3D3E90023FFF7CFFB011E18BF012163
:1013080004F184000EF05EFB84ED268A012005E0DE
:10131800B4F89C30B3F5807F05D1002006B0BDEC51
:10132800028BBDE8F08104F15008404627F0A2FE88
:101338000028F2D0DFED1B7A68EE277AFCEEE77A18
:10134800CDED037A94F8806094F89C209DF80C30D9
:10135800276E206D6EB18DF8153002238DF814209C
:1013680000210122009305ABB847404653F0EDFD3C
:10137800CAE7012531468DF813208DF814302A4626
:101388000DF113030095B847009532462946276E9C
:10139800206D05ABE8E700BFAE47E17A14AEEF3F3A
:1013A8009CC1070800007F432DE9F04F044685B033
:1013B80008466160062190461D469DF838709DF8E4
:1013C8003CB011F035F8A060067C16F0010602D09A
:1013D8007D4812F0D5F99DF8403005FB08F084F8F7
:1013E8002A309DF844307D3084F828307E2390FBE5
:1013F800F3F0C0010430C4E90485277360624EF03D
:101408006FFA0DF1080A0622C4E907066F4920465B
:10141800A66160F0AFFF022251462046ADF8088071
:1014280060F0A8FF022251462046ADF8085060F04F
:10143800A1FFF623032269462046ADF800308DF857
:10144800026060F097FF7B1EDBB2082B05D840F2E4
:101458005515DD4015F0010501D15D48B9E7052FA7
:1014680009D0072F06D0032F73D1012384F8293020
:10147800002502E02E4684F82960002646F34F1026
:10148800C0EB0020FFF70EF80022524BFEF7BEFE1D
:101498000022514BFFF79AF9FFF708FB5FFA80F833
:1014A800C6F38200C0EB0020FEF7FCFF00224B4B86
:1014B800FEF7ACFE00224A4BFFF788F9FFF7F6FA71
:1014C800C7B206F00300C0EB0020FEF7EBFF0022D6
:1014D800404BFEF79BFE00223F4BFFF777F9FFF7E3
:1014E800E5FAC0B2002D5ED08DF808008DF80980AD
:1014F8008DF80A70032251462046013660F03AFF03
:10150800802EBBD1BBF1000F1AD0364D01A92A8815
:10151800AB782046ADF8042003228B7060F02AFFD8
:101528000B222046304960F025FFD5F80300EB79FF
:1015380002900522514620468AF8043060F01AFFCE
:10154800204660F005FFA06960F026FF05B0BDE801
:10155800F08F092F84F829608AD10FF25C09D9E944
:101568000089354616A7D7E900672846FEF79AFF8F
:1015780042464B46FEF74AFE32463B46FFF726F9FF
:10158800FFF794FAC0B28DF808008DF809008DF8BD
:101598000A00032251462046FF3560F0EBFEB5F500
:1015A800FF4FE2D1AEE78DF808808DF809708DF80D
:1015B8000A009FE7AFF300800000000000C04F4022
:1015C8000000000000C05F40C5860808B56A08082A
:1015D8000A7E08080000F83F0000084000000C40A0
:1015E80000001C4012400708A96A08080000000013
:1015F80010EE103A33F0004210B52DED028B06D1F3
:101608000120BDEC028BBDE8104042F0B5BF002BB5
:1016180005DABDEC028BBDE8104042F0BBBFB3F168
:10162800FF4F06DB30EE008AB0EE480ABDEC028BB5
:1016380010BDB3F5000F6049BBBFDFED607A6FF0F6
:101648001802002260EE277AB8BF17EE903AF7EE3C
:10165800007ADC15C3F316037F3C1944144401F4E3
:10166800000282F07E5204EBD15403F10F011A43B9
:1016780007EE102A524A0A4037EE678AB2BBB5EE27
:10168800408AF1EE10FA0FD1002C00F08C8007EEA2
:10169800904A9FED4C0A9FED4C7AF8EEE77A27EED8
:1016A800808A07EE878ABFE741A1D1E90001FFF7E9
:1016B80025FAB6EE007A07EE900A07EEC87A68EEC9
:1016C800087A27EE277A14B938EE478AACE707EE8E
:1016D800904ADFED3C6AF8EEE77A07EEE67A37EEF5
:1016E800488A9FED397A17EE878A9DE7F0EE007AEF
:1016F8009FED365ADFED364A364A78EE277A1A4495
:10170800C3F5571388EE276A07EE904A03F522734C
:101718001343F8EEE76ADFED307A002B66EE065ADF
:1017280025EEA57A07EE275ADFED2C7A45EE077AE3
:101738009FED2B5A07EE875ADFED2A7A47EE274AA4
:10174800DFED297A44EE877A67EE877A45EE257AC7
:101758001ADDB6EE007A28EE077A27EE087A77EED9
:10176800877A67EE867A14B937EE677AACE79FED29
:10177800156A46EE867A37EE677A37EE488ADFEDE5
:10178800127A16EEA78A4FE778EE677A67EE867ABE
:1017980014B938EE678A47E79FED0A7A46EEC77AAA
:1017A80037EEC88AEBE79FED118A3DE7AFF300807B
:1017B800555555555555D53F20FB4A000000004C5E
:1017C800F0FF7F00D1F717378071313F25333A3E5C
:1017D800298E633E305CCFFF9788173E2549923E9D
:1017E800ABAA2A3F4FD01C3ECDCCCC3E0000000017
:1017F800F8B510EE904A10EE103A34F000472DED8F
:10180800048BB0EE609A0DD183F480035B0013F56E
:10181800000F40F2AA8230EE098AB0EE480ABDEC09
:10182800048BF8BD23F000411846B1F1FF4F02D8F0
:10183800B7F1FF4F08D9B3F17E5FECD184F480048F
:10184800640014F5000FE4E7002B25DAB7F1974F91
:1018580080F09482B7F17E5F39D3FA15C2F196020F
:1018680047FA02F505FA02F2BA4229D105F0010554
:10187800C5F10205B7F17E5F2AD1002C80F27B8288
:10188800B5EE400AF1EE10FA1CD1D80FBDEC048B6E
:10189800BDE8F84042F070BEB7F1FF4F10D1B1F18A
:1018A8007E5F00F0628205D9002CDFEDD17A29FE37
:1018B800278AB2E7002C80F25B82B1EE498AACE756
:1018C8000025D7E7B7EE007A87EE008AA5E700255E
:1018D800B4F1804F0A4640F05782B1F1BF4F0CD2A5
:1018E800B1F1D05F02D920EE008A96E7B0EEC08A47
:1018F80059BB012D00FE088A8FE723F04046B0EE61
:10190800C08AB6F17E5F17D1002CBCBFB7EE007A53
:1019180087EE088A002B80DAA1F17E51294305D190
:10192800BDEC048BBDE8F84042F034BE012D7FF4D5
:1019380074AFB1EE488A70E739B9002CD9DA002BB8
:10194800A4D06B1E58425841A0E7DE0F013E55EA6D
:101958000600E5D0B7F19A4F71D9A64B994208D83D
:10196800002C0BDA0020BDEC048BBDE8F84042F0F7
:10197800F5BDA14B994208D9002CF3DC0020BDEC41
:10198800048BBDE8F84042F0DBBDB7EE007ADFED2E
:101998009B7ADFED9B9A38EE478A93A1D1E9000143
:1019A80068EE278AFFF7AAF8B5EE007A07EE900AE4
:1019B800DFED946A68EE299A48EE477AB6EE007A27
:1019C80007EEC87A68EE087A27EE277AF0EE687A8A
:1019D80047EE667A39EEA77A17EE103A6FF30B03E3
:1019E80007EE103A77EE699A77EEE97A013DF7EE5D
:1019F800006ABFEE008A6FF30B04354367EE890A6D
:101A080008FE268A06EE904A39EE666A67EE267A5E
:101A180046EE070A30EEA77A17EE101A002921F0D1
:101A2800004340F31381B3F1864F40F2CC80B5EE0A
:101A3800C08AF1EE10FA4CBF0120002093E713F0A2
:101A4800FF4F05BF9FED707A6FF01701002168EE18
:101A5800077A08BF17EE902AD315C2F316027F3B08
:101A680042F07E500B4469498A4206DD68498A4241
:101A780040F3A7800133A0F500000021654A06EE77
:101A8800100AF7EE006A02EB8102D2ED005A75EEF9
:101A9800867A36EE657AC6EEA74A27EE245A15EE00
:101AA800102A6FF30B0206EE902A5B4A02EA6002E4
:101AB80042F0005202F5800202EB415207EE902AF2
:101AC80006EEE77A77EEE57ADFED545A36EE676A86
:101AD80065EE057A06EE667A9FED516A47EE865AFC
:101AE8009FED506A27EE247A66EEA64A05EEA76AAD
:101AF800DFED4D5A46EE275A9FED4C6A05EEA76A70
:101B0800DFED4B5A46EE275A36EE856A67EEA77A1E
:101B180026EE076A05EEA76AF0EE085A74EEA57A73
:101B280077EE867A17EE902A6FF30B0207EE902A6B
:101B380077EEE55A27EE277A66EEA76A75EEE45A3D
:101B480036EE656A06EE057A9FED3A6A76EE877A92
:101B580017EE902A6FF30B0207EE902A364A77EEBB
:101B6800E66A02EB810227EE866A37EE667ADFEDD7
:101B7800336A67EEA67ADFED326A47EE267A92ED8F
:101B8800007A77EE877A07EE103A2E4BF8EEC76A9E
:101B980003EB810336EE277AD3ED005A37EE257A28
:101BA80037EE267A17EE103A6FF30B0307EE103A6A
:101BB80077EE666A76EEE56A76EEC66A77EEE67ADC
:101BC80014E701215AE755D1DFED1F6A37EE677A2E
:101BD80070EEA66AF4EEC76AF1EE10FA3FF727AF87
:101BE80086234BE0AFF30080E13D55555555D53F71
:101BF80000000000F3FF7F3F0700803F70A5EC3630
:101C080000AAB83F3BAAB83F0000804B71C41C0033
:101C1800D6B35D00A8FF070800F0FFDF55326C3E21
:101C280042F1533E05A38B3EABAAAA3EB76DDB3EFD
:101C38009A99193F0040763F98FF0708C623F6B8DF
:101C48004F38763FA0FF07083CAA3833534A9342DF
:101C580007D9B5EEC08AF1EE10FA4CBF012000207A
:101C68008DE607D137EE677AB4EEE07AF1EE10FA36
:101C7800B6DBEEE7B3F17C5F72D9DB157E3B4FF440
:101C88000000474A002940FA03F00844C0F3C7534C
:101C9800A3F17F0342FA03F2C3F1170302EA000239
:101CA800C0F3160040F4000007EE102A40FA03F0D3
:101CB80077EEC77AB8BF404237EEA07ADFED396ACF
:101CC800DFED395AB7EE000A9FED386A17EE103A81
:101CD8006FF30B0307EE103A77EE677A67EE266A22
:101CE80070EEE70ADFED327A27EE277ADFED317AF8
:101CF80000EEA77A76EE877A77EEE66A37EE667AAE
:101D080067EEA76A07EE877A16EEA56ADFED2A5A0C
:101D180046EE265A9FED296A15EEA66ADFED285A87
:101D280046EE265AB0EE676A05EEE66AF0EE006AFD
:101D380067EE865A36EE666AC5EE866A36EEC77A6A
:101D480077EE677A30EE670A10EE103A03EBC0536D
:101D5800B3F5000F06DA42F077FA20EE088A5CE560
:101D68000020A9E700EE103AF7E7B7EE008A54E53D
:101D78009FED148A51E5B0EE408A4EE5B7F1FF4F6A
:101D88003FF48DAD0A460225B4F17C5F7FF4B5AD12
:101D9800002BFFF6B2ADB1EEC08A3EE50000164357
:101DA800000080FF0072313F4CBB31330EEADD3555
:101DB8008CBEBF351872313F55B38A38610B363B3C
:101DC800ABAA2A3E0000000010EE103AB3F1FF4F14
:101DD80010B52DED048BB0EE408A06DB30EE008A9C
:101DE800B0EE480ABDEC048B10BD774A934276DC0E
:101DF80023F00042B2F17E5F13D3FFEE007AB4EE17
:101E0800670AF1EE10FA06D10120BDEC048BBDE89B
:101E1800104042F0B1BBBDEC048BBDE8104042F06D
:101E2800B9BBB2F1645F0FD2B2F14A5F24BF20EEB2
:101E3800007AF6EE007ABDEC048B28BF07EE670A3D
:101E4800BDE8104042F0BAB9604A134493424ED8F4
:101E5800F7EE007A38EE277A17EE103ADC157F3C59
:101E6800002CD5BF77EE677A37EE488A78EE677A26
:101E780077EEC87A87EE879AC3F31603544A9342DB
:101E8800CCBF43F07C5243F07E52F7EE007AC8BFD5
:101E9800C3F5000307EE102AC4BF01349B1037EEC8
:101EA800678AF6EE008A68EE288A68EE888A002B30
:101EB80044D1B5EE408AF1EE10FA1DD1002C7AD04B
:101EC80007EE904AB0EE498A9FED427AF8EEE77A3B
:101ED80007EE878A9FED407A07EE878A80E7B3F19D
:101EE800B44FB5DBDC159FED3D9A7F3CC4E7012379
:101EF80000249FED3A9AD4E731A1D1E90001FEF719
:101F0800FDFDB7EE007A07EE900A07EEC87A27EED5
:101F1800287A14B938EE478A62E707EE904ADFED6F
:101F28002D6AF8EEE77A07EEA69A37EE497A37EE89
:101F3800488A9FED297A17EE878A51E7F0EE007AF2
:101F48009FED276A9FED277A78EE277AC8EE276AF1
:101F580066EEA67A07EE867A9FED236A07EE276A71
:101F68009FED227A06EE277A9FED216A07EE276A0F
:101F78009FED207A06EE277A9FED1F6A07EE276A03
:101F8800B0EE687A06EE277A27EE267A24B978EE3C
:101F9800C78A38EE688A23E707EE904ADFED0D6AB4
:101FA800F8EEE77A07EEA69A39EE079A78EEC98A2C
:101FB80038EEC88ABDE79FED098A11E7AFF30080C4
:101FC800555555555555E53FD613D43EE0096A4158
:101FD800F6043500D1F717378071313F0000000053
:101FE8009788173E4FD01C3E25333A3E298E633ED4
:101FF8002549923ECDCCCC3EABAA2A3F2DE9F047ED
:102008000546884600AF42F006FFA9680646B1F5C6
:10201800004F36BFA8F10403002303F00703B1F50E
:10202800004F34BF0420082002F0070407341C4482
:102038000444E40804EBD2048C4228BF0C46012275
:102048003146284642F0A1FE10EA020A16D1E946B6
:1020580088B06A46504BCDE90538032342F8103F53
:102068004FF4C25153464D4800F09EFECD468AF3C8
:102078001188BFF36F8F0423184602DF31462846C4
:1020880042F099FE06EB000949460022284642F034
:102098007CFEA9EB00094E4518D0E94688B0694690
:1020A8003F4BCDE90538032341F8103F3B48134621
:1020B8000A464FF4C25100F077FE0023CD4683F361
:1020C8001188BFF36F8F0423184602DF3146284674
:1020D80042F071FE8442804623D028D234443146EF
:1020E8002246284642F029FF01223146284642F07E
:1020F80068FE214642F05FFE261801223146284636
:1021080042F043FEC30708D43146284642F0C5FED4
:1021180032462146284642F037FF2146284642F0FB
:1021280051FF4FF001094846BD46BDE8F08706EB70
:10213800000A01225146284642F027FE10EA020909
:1021480027D15146284642F036FE40448442EAD818
:102158005146284642F0A1FE5146284642F02BFE41
:10216800A4EB0808804509D2344451462846224643
:1021780042F0E3FE2146284642F024FF524631460B
:10218800284642F001FF01223146284642F019FE56
:10219800C7E74FF00009C6E7A40908080C3F07087D
:1021A800C80908082DE9F843884600AF00297DD002
:1021B80005680122284642F02EFE014604462846BC
:1021C80042F0E3FD10EA020616D1E94688B06A46F5
:1021D800384BCDE90538032342F8103F4FF4C2517C
:1021E8003346354800F0E0FDCD4686F31188BFF34D
:1021F8006F8F0423184602DF2146284642F0DBFD94
:10220800261831460022284642F0BFFD361AB4424D
:1022180018D06E4688B06946284BCDE905380323A7
:1022280041F8103F244813460A464FF4C25100F0C3
:10223800BBFD0023B54683F31188BFF36F8F0423DA
:10224800184602DF00222146284642F0BAFD214600
:1022580042F0B1FD261801223146284642F095FD8C
:10226800C20708D43146284642F017FE32462146B6
:10227800284642F089FE00222146284642F085FD84
:10228800261A01223146284642F07FFDC30709D4A9
:102298003146284642F001FE22463146284642F0A1
:1022A80073FE34462146284642F08CFEBD46BDE802
:1022B800F88300BFF10908080C3F0708C809080897
:1022C80008B5024843F019FA002008BD1E0A08089C
:1022D8000E4A0346904202D30D4A904211D30D4A4A
:1022E80022B1934202D30C4A93420AD30B4A52B109
:1022F8000B48834234BF01200020934238BF00209E
:102308007047012070471046704700BF30390708F2
:10231800E89D080800000000000000000000000020
:10232800000000002DE9F04F9BB000AF04468B463B
:10233800D7F890A0FA637B6349B903784678807828
:1023480000EB830020445E4522D8A0EB040B0AF082
:10235800010394F80280FB62E378B8F1000F0CBF28
:102368004FF000090AF001093B6313B11AF0020F9C
:1023780017D1B9F1000F14D1FB6B1BB15946204698
:102388007A6B98475D4628466C37BD46BDE8F08FA6
:10239800451C2846FEF7CCFD013028440BF1010B03
:1023A800D1E7CAF3C003FB612378BB629B00BB6122
:1023B80063683B62BB6A04EB8301FB6B002B7DD136
:1023C8005D468844B9F1000F1DD08B469946A94E49
:1023D8001BF8013B54F82300002808BF3046FEF7DD
:1023E800A7FDD7F8943001304BB1D7F898304B455A
:1023F80082BFD7F8943023F8190009F10109C345C1
:102408000544E5D1D8461AF0050F0CBF4FF0020B72
:102418004FF0010B00260AF00203FB633B6B9E4260
:10242800B1D298F8013008F1020854F823A05046B8
:10243800FFF74EFFFA69034602B3B86318F8021CA7
:10244800386A43F03BF9BB6BC0B1EA468AB06A46CA
:10245800894B05933B6ACDE906314FF40073ADF81B
:102468002030864B42F8103F00234FF41251844825
:1024780000F09AFCD546023D0136CFE723B1FB6A4E
:102488002BB9A5EB0B05F7E7FB6B002BF4D07948CC
:10249800BAF1000F18BF5046FEF74AFDD7F894303E
:1024A80053B1D7F8983099453FBFD7F89420431CCB
:1024B80022F8193009F101090544DDE7B9F1000FE7
:1024C8006DD04346102B28BF10230026BB6397F816
:1024D800389007F14800BA6B796260F04CFF796A6E
:1024E80000227A620AF0020201EB08033A610AF05C
:1024F80004027B61FA6002337A6A396B8A4267D3D5
:102508006378F96A1AF0020F7B624B4418BF002205
:10251800DBB208BF7208002940F0A9801AF0040F46
:1025280014BF314600216370A170E27020467A6BB7
:10253800B969FB6B9847051EFFF625AFBB6A3146A4
:1025480023707B6A7A6B63703B6B84F80280E3705C
:1025580007F15800FB6B9847061EC0F2C5803A6B1E
:10256800BB69386B03EB4203ABEB0301D7E90D23DF
:10257800C91A7B6903EB4000FB6B98470028C0F23F
:10258800B5804FF000082E44351807F1480AC845B1
:1025980078D300217A6B0846FB6B9847F3E6B8F1CD
:1025A800000F0CD01AF0040F0ED04346102B28BF92
:1025B8001023BB6397F8386007F158008BE746464D
:1025C800C146C7F838808BE74E46C7F8388087E79A
:1025D80013F8015C13F8021C54F82500BB60FFF7E0
:1025E80077FE0246F869BB6838B1386AC7E9013234
:1025F80043F064F8D7E90132F0B912B3FA6A72B15C
:10260800B9F10F0F18D809F1280107F1400009F1B5
:102618000102014401F8205C5FFA82F90CE0FA68D3
:1026280052B10F2E08D806F1280107F14000721C9C
:102638000E1806F8105CD6B27A6A023301327A6252
:102648005AE73A69002ADBD10F2EF5D806F128009F
:1026580007F1400C6044721C00F8101C07F1680177
:10266800023651FA82F2F6B202F8105CE4E7002171
:1026780059E700BF4C0A0808530A0808040000017B
:10268800643E070818F80A3054F823B087F8473032
:10269800D7F8943033B3D7F89830984522D2D7F882
:1026A800943033F8186001217A6BFB6B07F147000F
:1026B800984700281ADB0E4B0544BBF1000F08BFF2
:1026C8009B4626B95846FEF733FC461CB6B231463F
:1026D80058467A6BFB6B9847002807DB054408F1DE
:1026E800010854E70026DEE735464CE605464AE68B
:1026F8004C0A0808014B1860704700BF8001002091
:10270800044608B5EFF31183102383F31288BFF34F
:102718006F8F46F08DFC204601F03EFA024842F0E9
:10272800ECFF43F0EEFDFCE7070B0808034A002026
:10273800536823F002035360704700BF004004E071
:1027480008B5094A136943F0005313614168074803
:102758000C3183681B681BB1984700EAE07008BD1C
:102768006FF05700F9E700BF00080246403A070833
:10277800082810B502D90024204610BD044B53F890
:102788002040204647F00EF90028F5D1F3E700BFB6
:10279800CC43070810B5EFF31184102383F3128894
:1027A800BFF36F8F084803683BB9084A916A41F044
:1027B80001019162916AC907FCD50133036084F372
:1027C8001188BFF36F8F10BD7C37002000080246C8
:1027D80010B5EFF31184102383F31288BFF36F8FC2
:1027E80011490B68A3B90122104BD3E8EF1F002948
:1027F80003D1C3E8E02F0028F7D104D102210C4A05
:102808000C4843F0C9FB84F31188BFF36F8F10BDE8
:10281800012B08BF084803F1FF3302BF826A22F088
:10282800010282620B60EEE77C37002078370020D7
:10283800CC0B0808343F07080008024607B505F026
:10284800E9FC0E4B0E4A1A600E4BD3F8942042F066
:102858000402C3F89420D3F8943003F004030193DE
:10286800019B094BDA6A42F00102DA629A6822F0A7
:1028780002029A6003B05DF804FB00BFC80600209E
:1028880000093D00000C0246000802462DE9F04709
:10289800044607464FF00109DFF84C8094FAA4F586
:1028A800B5FA85F509FA05F32E0108EB05156FEA67
:1028B800030A24EA03042B7B63B158F806301B692A
:1028C8006BB94644736802222846196807EA0A0762
:1028D80043F0F2FA002CE1D13846BDE8F0872846EB
:1028E80098470028F6D1ECE7D43F070810B5002236
:1028F80088B00E490E4847F0AEFC002200230024A1
:10290800CDE906230E234FF44072CDE90334CDE917
:102918000144084B08490094084809F0D5FC0849C7
:10292800064847F0F6FA204608B010BD4D290108C0
:1029380068280020592C010800520020802300201C
:10294800140C0808014809F009BA00BF5411002006
:102958002DE9F047804620480F4643F089FA06469D
:10296800002832D000252846BDE8F087237B83B1B4
:102978002368DB680BB120469847636883F80690A4
:1029880023681B69CBB9636802222046196843F0A3
:1029980093FA013610345445E8D3B8F1000FE2D069
:1029A800002DDFD02846FFF771FF0546002FF7D02E
:1029B8000021642047F0AFFBF2E720469847002843
:1029C800E1D009FA06F31D43E3E705464FF0010994
:1029D800024CDFF80CA0DEE790370020D43F070850
:1029E800E43F0708014B53F82000704704440708E8
:1029F80008B5034608462BB1044A136000F044FCAE
:102A0800002008BD6FF01500FBE700BF840100201F
:102A180010B5044C237813B9034809F09FF9012332
:102A2800237010BD7E4900205411002010B50446C3
:102A3800094843F01DFA3CB1084BD3E8EF1F0139B0
:102A4800C3E8E21F002AF8D105480AF05FFABDE89A
:102A58001040044809F082B9883700208C370020DC
:102A680068280020541100200022044BD3E8EF0FFF
:102A7800C3E8E12F0029F9D1704700BF883700204B
:102A880070B5FFF7F1FF0546074C084EB44200D376
:102A980070BD63685B792BB123685B6813B1294605
:102AA800204698471034F1E7D43F0708E43F070869
:102AB80010B5044C0449204642F02DFF034B1C601E
:102AC80010BD00BF6C100020F043070880370020BD
:102AD80000230D4A10B513700C4A4FF47A71136035
:102AE8000B4A0C481360FFF783FFFFF7E1FF0A4B1F
:102AF8000A4918468B4200D310BD1A1A5C68121195
:102B0800013222711033F5E77F4900208837002011
:102B18008C3700208B5E0508D43F0708E43F070880
:102B2800014642F210720023014842F015BF00BF6F
:102B38006C100020014842F0ABBF00BF6C100020B1
:102B4800024B0146186842F0FEBF00BF80370020E4
:102B5800014843F033B800BF6C10002070B5254B16
:102B68001B78002B43D0FFF7E5FF044600283BD134
:102B7800214B224D1B68002B12DD47F024FB0A2253
:102B88000023FEF769F9D5E90032C01A40F2E933AB
:102B980061EB0201984271F1000101D3FFF770FF68
:102BA800D5E9003213F57A7342F10002C5E9003223
:102BB800ECB1BDE87040FFF7CBBF6B685B7923B120
:102BC8002B68214628461B6898471035B542F4D330
:102BD8002046FFF7B5FF0A4BD3E8EF1F0139C3E8DA
:102BE800E21F002AC4D0F7E7064D074EEEE70020A3
:102BF80070BD00BF7E490020883700206028002073
:102C08008C370020D43F0708E43F070870B50D4D06
:102C1800297861B90120FFF79BFE0B4C0B4EB4429B
:102C280006D3FFF79BFF0028FBD101232B7070BD53
:102C380063685B791BB1236820469B68984710340A
:102C4800EDE700BF7F490020D43F0708E43F0708AD
:102C580000212DE9F8430846FFF77AFE044648B3F9
:102C68004FF4FA784FF0000901F03EF91A4B1B4A6D
:102C78001B58136033B11A4B1B68092B02DD194826
:102C880009F06CF80025184F44B12046FFF7FEFD07
:102C9800044618B94FF0FF384FF0FF39FFF75EFFD1
:102CA800064628B9B5B90F4842464B4609F092F88E
:102CB8003546E9E74FF0FF384FF0FF39D4E72B6886
:102CC8009B691BB100222846114698471035BD4222
:102CD800F5D3E8E7054DFAE708000000843700203F
:102CE8008C37002054110020E43F0708D43F070820
:102CF80013B5184843F0BCF8174B1B7873B1EFF3C2
:102D08001184102383F31288BFF36F8FFFF726FF18
:102D180084F31188BFF36F8F02B010BD0F4B1B688F
:102D2800002BF9D050B9002200230D48CDE900232B
:102D380042F2107200230AF0C3F8EDE70928EBD13C
:102D480007480AF0E3F8074802B0BDE8104009F068
:102D580005B800BF8C3700207F4900208437002049
:102D6800682800205411002010B5064B04461B6843
:102D780098472146A060044842F06BFEBDE8104029
:102D8800FFF7B6BF840100206C100020044A054BF1
:102D98009B1AB1EBD30F34BF52F8310000207047B3
:102DA800543E0708D43F07082DE9F04F8FB0C1F310
:102DB8004A2604AF0D469046B8607B600C0D002E85
:102DC80061D04FF000090A234FF0040B07F1140AF1
:102DD800FE60C7E90799C7F824900093CDF808B0BA
:102DE800CDF804A007F11C034A464046F968FFF7EE
:102DF80099FAB0F5006F03461CD36C468AB0D8F830
:102E0800041004AB24481A46C3E9050140F2FF71D7
:102E1800D9614FF400711984204B42F8103F4FF4E8
:102E280012514B461E48FFF7BFFFA5462C37BD463B
:102E3800BDE8F08FC0F30A0604F11700184420F02B
:102E4800070080083B60FFF76BFE66F353250446D6
:102E580080B13B6800F11001C7E908390A23F9611C
:102E6800CDE901AB009340460E4AF96807F11C030F
:102E7800FFF758FA66F353252A4620467B68B96857
:102E880043F03AF8D2E704F1170020F00700800871
:102E9800FFF746FE0446EDE7250C0808040000018C
:102EA800D43E0708D35E05082DE9F04F87B00546E4
:102EB800DDE9106BDDE9127A884614469946BFB100
:102EC80010213B465A460020CDF800A0CDF814A0AA
:102ED80042F01BFAB0F5006F01460BD340F2FF73C6
:102EE8000221184A184807B0BDE8F04F43F05DB812
:102EF8003946384604F0070305F00704E40044EABD
:102F0800831444EA402444EA065406F117000844AE
:102F180020F0070080080391FFF702FE054640B144
:102F28003FB13B465A460399CDF800A0103042F015
:102F3800ECF94B4622464146284607B0BDE8F04F1B
:102F480042F0DABF640C0808D43E0708406820B194
:102F5800034BC01A40F3CF0070474FF0FF30704763
:102F6800543E07080EB403B503AB53F8042B0146CF
:102F78000448019301F0ECF902B05DF804EB03B0EA
:102F8800704700BF15600508CA0605D48B064CBFFC
:102F980002490349FFF7E6BF704700BFC53208087A
:102FA8005A2A08082DE9F04F8BB099469DF85880A9
:102FB800179B044607930D46DDE918A31A9F06924E
:102FC8000593B8F1000F00F0BC80834B07F0020BAB
:102FD80013F80830089307F48073099342F06AFFE6
:102FE800024600287AD020467C49FFF7BBFF0646F8
:102FF800BBF1000F08D017F0440F71D12A462046C4
:103008007749FFF7AFFF064407F0010353B1754B4B
:10301800204653F82820744B7449002A08BF1A46E2
:10302800FFF7A0FF07F48073002B07F0080318BF11
:103038004FF00009002B7FD06D4B204653F8282015
:103048006C49FFF78FFF0546069B2BB11A462046B1
:103058006949FFF787FF0544B9F1000F0DD0089BB8
:10306800002B6CD06549664BB8F1040F18BF1946A0
:103078004A462046FFF776FF054462483544079BD9
:103088001BB12246604942F0E8FA059B002B00F08C
:103098008E80059B3946102B28BF10232046994661
:1030A8000026FFF771FFB54252DC00263346204662
:1030B8001AF803205549FFF755FF0136102E4DD059
:1030C800710703D120465249FFF74CFF4E4533465E
:1030D800EDD320464F49FFF745FFEEE7064687E761
:1030E8004D4B186800288ED04C4B4FF47A7B1B68E8
:1030F8004FF03C0CB5FBF3F5B5FBF0F14FF4616311
:1031080000FB11550BFB05F5B1FBF3F2B5FBF0FE27
:1031180003FB121100FB1E55B1FBFCF30BFB05F57D
:10312800B5FBF0F50CFB131120460091CDE901E544
:103138003B49FFF717FF66E707F0080584E73049C2
:1031480096E7B9F1010F45460CBF2E48354896E77A
:1031580020462F49FFF706FF0136A4E70026204640
:103168003149FFF7FFFE33461AF803202046A2F143
:1031780020035F2B28BF2E222C49FFF7F3FE0136D0
:10318800102E0DD0720703D120462149FFF7EAFE21
:10319800B1453346E8D820461D49FFF7E3FEEEE780
:1031A800059BCA44B3EB090305937FF472AFB8F1EA
:1031B800000F0AD0FB0704D520460B4A0B49FFF73E
:1031C800D1FE39462046FFF7DFFE20460BB0BDE8AA
:1031D800F04F42F00EBF00BFE46A0808AA0C0808C6
:1031E800AE0C0808144407089C0C08087E3108082F
:1031F80028440708D40C0808DA0C0808A10C0808A9
:10320800A50C08081560050859430108DE0C0808D4
:1032180089690808876908089837002094370020CA
:10322800B80C080843600508E40C0808C53008080D
:1032380042F20F7373B58B4228BF0B4605680446EC
:10324800052168460D4A3DF07BFE06466368284620
:103258000B225B680A4942F0BEFE63683246694643
:1032680028465B6842F0B7FE63681B2228465B6805
:10327800044942F0B0FE02B070BD00BFD520080876
:10328800D86A0808BC6A080800210123064A904247
:1032980006D8064A01B901231360054B1860704728
:1032A800012140085B00F2E740420F0094370020FC
:1032B80098370020F8B50D460446064F4618B44224
:1032C80001D12846F8BD14F8011BBB6801485B68AA
:1032D8009847F4E71C3C0708014B0360002070473F
:1032E800704407082DE9F34205460E4600244FF0C6
:1032F8001409084B084F1B680193019BA34202DC89
:1033080002B0BDE8F0823868314609FB0400A847DE
:103318000134F2E7704407089001002070B5104BA3
:103328000D461C68B4B10F4B196800238B4202DBB1
:103338006FF0010070BD224612F8146B864202D06D
:1033480014460133F2E7E06846F02CFB28B1002070
:103358002C60EFE76FF00C00ECE76FF01200E9E784
:10336800900100207044070810B5436888B00293A4
:1033780083680C46CDE9033200230A68C068CDE9AA
:103388000623054901AA059344F0DBFF079808B90D
:10339800059B236008B010BDD56105082DE9F843E9
:1033A8000646FDF7C5FD0546EFF31188102383F3A4
:1033B8001288BFF36F8F114B1C68D3F804909C429E
:1033C80008BF002434B988F31188BFF36F8F2046F3
:1033D800BDE8F883A7683846FDF7AAFDA84206D1DC
:1033E8002A463946304660F011F80028EBD04C45A3
:1033F80001D02468E6E70024E5E700BF9401002037
:103408002DE9F0410E461546FFF7C8FF044628B3DC
:10341800C3681BB35F690FB3062E07D0072E20D0F1
:103428002A4631463B46BDE8F0411847838A3BB9F6
:103438002A463146B84750B9A38A0133A38206E029
:103448004FF6FF72934204D00133A3820020BDE8F7
:10345800F0810121114A124842F09EFD6FF01500DB
:10346800F5E745B12A7832B10022828231462A46F0
:103478005B699847EAE7A38A012B08D12A46072106
:103488002046B8470028E2D1A38A013BD6E70BB112
:10349800013BDAE70221034ADDE700BF380D0808DF
:1034A800743E07085A0D080810B5044608B180682C
:1034B80038B9104A1048012142F06EFD6FF015002E
:1034C80010BDFFF76BFF08B10C4AF3E7A082EFF3DA
:1034D8001181102383F31288BFF36F8F084B5A684A
:1034E800C4E9003214605C6081F31188BFF36F8F08
:1034F800E6E700BF780D0808743E0708910D080834
:103508009401002080B505460E461746984609F0F6
:10351800FBF9034600F0E8FC0446DFF81890424641
:1035280049F8003039463046A84754F8090000F0F9
:1035380055FC00BF0800000008B50348034A0021F5
:10354800121A42F0B5FE08BDC0130020FC4D002041
:10355800074808B5074A0849121A42F0ABFEBDE809
:1035680008400648064A0749121A42F0A3BE00BF9F
:1035780000000020C0130020E89D0808000000207B
:1035880000000020E89D08082DE9F84F80460C4609
:1035980000AF00296AD0D1E90012E9468AB0A368D1
:1035A8006D464FF0050A6E463948CDE90723CDE947
:1035B800050146F810AF002332464FF42151354833
:1035C800FFF7F2FBD4E90312CD466369AD463248F2
:1035D800C5E90723C5E90501C5F810A0002332464F
:1035E8004FF421512B48FFF7DFFBCD46E36901215A
:1035F8002A4A284842F0D9FC0121294A254842F0A4
:10360800CBFC264600254FF00A0ADFF8A4B0E946AD
:10361800D6E908C0D6E90A138EB06A46CDF81CC0B0
:1036280005F1010CCDE908C0A81CCDE90A01E91C87
:10363800CDE905B5CDE90C1342F810AF002345F2EA
:10364800400114480435FFF7AFFB102DCD4606F1B5
:103658001006DCD1236E0121124A0E4842F0A5FC67
:10366800A3690121104A0B4842F09FFCB8F1010FF1
:1036780007D1EFF305830D4A41460648103B42F057
:1036880094FC2146404607F0A1FFBD46BDE8F88FEF
:10369800C90D0808043F0708F80D0808270E080890
:1036A800360E0808B30E0808C20E0808F00E0808FF
:1036B800700E080830BFFFF7FDBF00BF2DE9F041CD
:1036C80005460B4EDFF83080324606EB0807CC1B68
:1036D800204608495FF04FFEA01942460021083CE9
:1036E8005FF06FFEC5F8904007F10800BDE8F08173
:1036F80000000000E43F07080800000010B5244C53
:103708002449254842F0E3FDA36A99013ED52248A1
:10371800224942F0DCFD1E20A36ADA0104D51E48C6
:103728001F4942F0D4FD1F20194CA36ADB0204D5BF
:1037380019481C4942F0CBFD0220A36A1C0304D59A
:103748001548194942F0C3FD2120114CA36A5903B9
:1037580004D51148154942F0BAFD2220A36A9A03FC
:1037680004D50D48124942F0B2FD2320084CA36A43
:10377800DB0304D508480F4942F0A9FD2420A36AB9
:103788006FEA03436FEA1343A36210BD1D20C3E72A
:1037980000ED00E0030F0808043F07081B0F0808A6
:1037A8002E0F0808480F0808720F0808900F08081D
:1037B800B50F0808CF0F080870B506460D46294C06
:1037C80029492A4842F083FDA36ADB0647D52748E2
:1037D800274942F07CFD1120A36A1C0704D5234821
:1037E800244942F074FD12201E4CA36A990712D591
:1037F80021491E4842F06BFD636BA26A120609D587
:1038080001211E4A194842F0D0FB1EB1A36A23F0D9
:103818008003A3621320134CA36ADE0704D5134860
:10382800174942F054FD1420A36A9C0604D50F489A
:10383800144942F04CFD15200A4B9A6AD10658BF2C
:103848009A6A9A6A920642BF5A6A22F400525A62E7
:103858009A6A42F0FF029A6200232B7070BD102012
:10386800BAE700BF00ED00E0FA0F0808043F0708B8
:103878001010080843100808561008086E100808A9
:1038880084100808A310080870B506460D46284C91
:103898002849294842F01BFDA36AD9043CD526488B
:1038A800264942F014FD1720A36A1A0504D52248B8
:1038B800234942F00CFD18201D4CA36A9B0512D524
:1038C8001D48204942F003FDA36BA26A100409D5E4
:1038D80001211D4A184842F068FB1EB1A36A23F46F
:1038E8000043A3621920124CA36A590504D5124853
:1038F800164942F0ECFC1A20A36ADA050ED50E48E8
:10390800134942F0E4FC1B20094A936A43F47F43BD
:10391800936200232B7070BD1620C5E7A36A9B0431
:10392800F2D505480B4942F0D2FC1C20ECE700BF59
:1039380000ED00E0D2100808043F0708E810080866
:1039480043100808F9100808121108082711080878
:1039580042110808A3100808F0B59DB0664B05464B
:103968005868002600AFC0F3080386F31188BFF338
:103978006F8F02F07F44B4F17F4F07D102F00C043F
:10398800082C0ED15D495E4842F0A1FC5D495C48B7
:1039980042F09DFC00210846FFF7F6FD7437BD464E
:1039A800F0BD14074CBF0D460126002DEED00022B5
:1039B800FA71DA1E092A7ED8DFE802F005757871F7
:1039C8007D7D7D7D7D7B50494D4842F080FC002304
:1039D800494CFB71E36A9A0705D54C49484842F0BF
:1039E80076FC00242DE0E36A002B01DA4849F5E76C
:1039F800E36A5B00F5D54749414842F068FC6369D2
:103A0800AA6943F480736361BFF34F8FBFF36F8F6D
:103A180032F8023C626922F480726261BFF34F8F10
:103A2800BFF36F8F03F47F42B2F55F4F21D1DBB252
:103A3800022B1ED12B680121374A314842F0B5FAD2
:103A48002C68FB79002BA9D16822294607F10800C8
:103A58005FF091FC7B6A002E4AD0C3F3080222B9BA
:103A68006FEA53236FEA43237B62204607F108017C
:103A780092E7214B9A6AD2B222B10120F91DFFF7D1
:103A88009BFE0EE09A6A12F47F4F04D00120F91DC4
:103A9800FFF7FAFE05E09B6AB3F5803FA1D3FFF775
:103AA8002DFE0446CDE70020F91DE8E70020F91DAA
:103AB800EEE71A4992E71A4A6C4610F4F87F8AB082
:103AC800184918BF11466A46103B07934FF4007314
:103AD8001548ADF82030154BCDE9050142F8103FE7
:103AE80000234FF411510648FFF75EF9A54678E721
:103AF8006FF30803B8E700BF00ED00E0881108087D
:103B0800043F0708B3110808EF110808061208084F
:103B180027120808351208085412080870120808F5
:103B28006F1108085A1108089412080804000001C7
:103B3800064B5A6942F010025A615A6942F480628F
:103B48005A615A6922F008025A61704700ED00E094
:103B5800EFF30880EFF3098101B57246FFF7FCFE29
:103B680001BD00BF0A4880F30888102080F311883F
:103B780008484FF40061401880F30988EFF3148077
:103B88000221084380F31488BFF36F8F00F07AF89E
:103B980020C9002000610020BFF34F8F0549064B64
:103BA800CA6802F4E0621343CB60BFF34F8F00BFD3
:103BB800FDE700BF00ED00E00400FA051EF0040F69
:103BC8000CBFEFF30880EFF30980816911F8021C3C
:103BD8000229FFD001B5724642F06EFB01BD00BF5D
:103BE8000028ACBF00F16040064B4FEA0111C9B292
:103BF800ABBF00F5614000F00F0080F800131954C6
:103C0800704700BF14ED00E040B2002807DB012335
:103C18004109034A00F01F00834042F821307047F1
:103C280000E100E040B200280CDB0122064943090C
:103C380000F01F008240203341F82320BFF34F8F4C
:103C4800BFF36F8F704700BF00E100E0054B4209EA
:103C580053F82220012300F01F0003FA00F010405F
:103C6800704700BF00E100E0044B054A23F07F03E2
:103C78009360BFF34F8FBFF36F8F70470000010849
:103C880000ED00E008B5FFF7EFFF104BD3F88820F0
:103C980022F47002C3F88820D3F8882042F4A002E6
:103CA800C3F888204FF04042C3F83422BFF34F8F47
:103CB800BFF36F8F0023E1EE103AFFF73DFCFFF7EB
:103CC80047FC00F0F3F807F0ADFD00BF00ED00E0A1
:103CD8008189203A41F0020181814FF47D41C0F889
:103CE800DC101360009B08495360019B21F001011F
:103CF8009360029B9161D3604FF08073D36100237E
:103D08000265C0F8943070470D350108104B9B6868
:103D180083421AD1EFF30580B8B9EFF3118110226D
:103D280082F31288BFF36F8F9A8922F002029A8178
:103D3800EFF3148323F0040383F31488BFF36F8F26
:103D480081F31188BFF36F8F70476FF015007047CC
:103D58009C3B00200E461546002300B5E1EE103AC4
:103D6800EFF3148323F0040383F31488BFF36F8FF6
:103D7800BFF36F8F0C4BD0F8902098600B4B1A60F4
:103D8800D0F8803083F30B882C4686F3098800200E
:103D9800034B98472046002100220023014C20476E
:103DA800FD6205080D3501089C3B0020C83700203E
:103DB8001022014B1A61704700ED00E0054B9A692B
:103DC8009B689A421FBF044A536843F0805353606C
:103DD800704700BF9C3B002000ED00E0084B9B684B
:103DE80083420BD1EFF3058343B1064B5A6842F087
:103DF80080525A605A6A22F400425A6246F08EB8DB
:103E08009C3B002000ED00E025498A6882F8DDE04F
:103E18004FF030001044EFF3098C80E8F01F1EF0DB
:103E2800100F03D102F19C0080EC108A102080F35F
:103E38001288BFF36F8F1B4F4FF000668A698A6044
:103E48003E60D2F89000184C206092F9DDE0D2F87C
:103E580094000023C2F8943080F311881EF0100FEC
:103E680003D00023E1EE103A03E002F19C0090EC4D
:103E7800108AEFF3148323F0040383F31488BFF349
:103E88006F8F02F1300090E8F01F8CF3098802F17F
:103E9800000004B542F027FABDE80440704700006E
:103EA8009C3B002004ED00E0C837002000231021CF
:103EB8000348C2180133722B82F80013F9D17047F6
:103EC80000E100E008B5EFF30583064A103B02EB7A
:103ED800C30152F8330049688847BDE80840FFF736
:103EE8006DBF00BFAC0C002001480068704700009F
:103EF800C83700201FB50121094B0A4A0A4800F0BB
:103F08000FF90023064A0393084B0121019301A8E6
:103F1800D31A029300F00EF905B05DF804FB00BF58
:103F280000000C2000000020C4440708C013002033
:103F38000A7A0B6810B562F304031C46CB68520971
:103F480023F01F0343EA4203044A43F00103C2F883
:103F58009800C2F89C40C2F8A03010BD00ED00E007
:103F680010B50A4BD3F89030C3F30723013B9842AE
:103F780008D901210346064A064842F016F86FF0B0
:103F8800150010BDFFF7D4FFFBE700BF00ED00E010
:103F9800AB120808EC3E07082DE9F04F8946144695
:103FA80006464FF000084F4D85B0C84527DAD6F8C9
:103FB80004A0BAF1000F44D0BAF11F0F17D91AF0B4
:103FC8001F0F14D1D6F800B01BF01F0F0FD15846A1
:103FD80042F0A4F907460AEB0B00013842F09EF9BB
:103FE800874210D06FF015073F4A3B4601E0434631
:103FF8003E4A01213E4841F0D8FF6FF015042046A3
:1040080005B0BDE8F08F17F1160FEDD0BC42EBDD1F
:10401800C5F89870D5F89C10C5F89870D5F8A030F8
:1040280021F01F0143F01F0BD6E900321A449942D0
:1040380002F1FF3A1AD1D34507D13146F8B242F01E
:1040480076F908F101080C36AFE73146C5F89870E3
:10405800D5F89C30E0B263F30402C5F89C2042F026
:1040680066F910F1160FC8D0441CEAE7C5F8987035
:10407800D5F8A020013B23F01F0302F01F021343D1
:10408800D3453146E0B2C5F8A030E8D042F04FF948
:1040980010F1160FB1D0C5F89870D5F89C209DF88E
:1040A80008300BF1FF3B62F304038DF80830D5F8B4
:1040B800A0309DF808205B0863F347128DF80820AC
:1040C800D6E900321344009323F01F035B44A3EBAB
:1040D8000A03013023F01F036946C0B20393FFF7B8
:1040E8003FFFBEE700ED00E0F7120808D11208080C
:1040F800EC3E07080522044BC3F89420BFF34F8F0A
:10410800BFF36F8F704700BF00ED00E0BFF35F8F14
:104118000022024BC3F89420704700BF00ED00E076
:1041280010B5034C2278FFF737FF207010BD00BF91
:10413800814900202DE9F74F294D8A4606464FF060
:104148000008AB46274FD0451BDAD6F80490B9F1E2
:10415800000F3FD031680846019142F0DFF801991D
:10416800044609EB0100013842F0D8F884424FF0C8
:1041780014021D4B08D002FB08F36FF015024BF830
:10418800032003B0BDE8F08F14F1160F2C60F8D0AF
:104198001978A142F5DD02FB08B0C7F89840C7F8C6
:1041A8009840D7F89C4000F10801007B64F30400B4
:1041B8000871D7F8A0000C79400860F347140C7117
:1041C800D7F89C1021F01F016960D7F8A01021F0E2
:1041D8001F01296108F1010814350C36B3E700BF47
:1041E800CC37002000ED00E081490020F0B55349AC
:1041F800534DD1F890302C68C3F307239C4287B005
:1042080000F299800020FFF781FF4E4BC1F8C030C3
:10421800844216D14C4D01A82C70FFF75DF800269A
:1042280007464A4CB74213D100202B784349D1F8AE
:104238009020C2F30722934277DBFFF75BFF002051
:1042480046E0696801EB0011FFF772FE0130DFE715
:104258000199300101EB0613DA682240B2F1807F40
:1042680052D00AD8B2F5001F34D0B2F5800F3ED034
:10427800B2F5801F12D00136D4E7B2F1006F43D0F7
:10428800B2F1805FF7D15A689B680958013B22F068
:104298001F00034423F01F03012032E05A689B6883
:1042A8000958013B22F01F0003440120844623F0F3
:1042B8001F0340EA4C10CDE902218DF8100002A935
:1042C80028780593FFF74CFE00282ADA6FF01500CE
:1042D80007B0F0BD5A689B680958013B22F01F00DF
:1042E80003444FF0020C012023F01F03E1E75A6852
:1042F8009B680958013B22F01F000344022023F069
:104308001F034FF0000CD4E75A689B680958013B1B
:1043180022F01F0003444FF0030C012023F01F0379
:10432800C7E72B7801332B70A5E7C1F89830C1F89F
:10433800A00001337BE74FF0FF30C9E700ED00E054
:10434800D0440708AAFF4400814900200000F0FF7C
:10435800F0B587B007460E4614460021102268467D
:104368001D465FF02EF802238DF80230054B2A46D1
:1043780021466846CDE9047601933CF073FF07B007
:10438800F0BD00BF6F63050808B5024B1B6898476E
:10439800002008BDE0370020034B044A18609378DA
:1043A80043F0020393707047E03700209C0100201F
:1043B80008B5054841F0A1F9002383F31188BFF33C
:1043C8006F8F0423184602DF2913080808B5064929
:1043D800064821F00701C1F1005202F5402240F0E1
:1043E80042FF002008BD00BF13EA0020E437002088
:1043F8004FF0FF324FF0FF33014807F0B7BB00BF63
:10440800AC010020014807F023BC00BFAC0100202C
:1044180038B50546FFF7ECFF2A460821074840F063
:1044280068FE044628B925B1FFF75EFD0C22044B4F
:104438001A50FFF7E7FF204638BD00BFE4370020D9
:104448000C00000038B504460D46FFF7D1FF2146A1
:104458002B460822074840F0CEFE044628B925B16D
:10446800FFF742FD0C22044B1A50FFF7CBFF204602
:1044780038BD00BFE43700200C00000010B504462A
:10448800FFF7B6FF21460348FDF78CFEBDE8104054
:10449800FFF7B8BFE437002070B541690446867A53
:1044A8000A4D59B1437ADB0706D42C2303FB065384
:1044B8005B6A1B689B689847002363612C20214630
:1044C80000FB0650BDE8704045F049BCA81100202B
:1044D8002C22024B02FB0030704700BFA8110020BD
:1044E8002C21827A054B01FB02339A6A1B7F801AC2
:1044F8001B3323F00303B0FBF3F07047A81100202F
:1045080038B52C24827A064B04FB02335B6AD3E964
:1045180001240C601568FFF7E3FF04FB005038BD69
:10452800A81100202DE9F04385B00546684690465D
:104538001C46039145F049FEDDE90067EFF3118958
:10454800102383F31288BFF36F8F6B8B002B41D03E
:104558002A8B9A4225D900220023284607F0C8FB57
:104568000446F0B189F31188BFF36F8F039B002BCA
:1045780041D032463B46684645F04CFE2C21A27A93
:10458800254B204601FB02335B6A03A91B681D68A3
:10459800DDE90023A847606170BB2046FFF77CFF78
:1045A80024E0698B4B1E6B8389F31188BFF36F8FEF
:1045B8002B7F2A8BAC6A1B3323F00303521A02FBAE
:1045C8000344154B154AEB1A9B105343A3722B7FD8
:1045D800E372CBE789F31188BFF36F8F2346424616
:1045E800284607F085FB04460028BFD10024204652
:1045F80005B0BDE8F0836361012300252381039B97
:1046080029466382E27A656004F118005EF0D9FEFB
:1046180063692582E360EAE7A8110020A38B2EBA1C
:10462800F8B500242C260F4D00B9F8BD476800F1F5
:104638000802D2E8EF3F591EC2E8EC1FBCF1000F98
:10464800F7D1DBB2012BF0D1837AC46006FB0353A8
:1046580044601B6A13B198473846E5E7FFF71CFF2B
:10466800FAE700BFA8110020F7B506460D46144624
:10467800124F384645F096F9E0B1BB6831463846E6
:104688001B68AAB29847002802DB002003B0F0BDDF
:10469800002CFBD1AC42F8D22F1B042F28BF0427D3
:1046A80005F0F0FF3A46019001A930195EF063FE6B
:1046B8003C44EFE76FF01200E8E700BFC83B07088B
:1046C80038B5044608F0FCF8204641F0C8FEA06959
:1046D800C8B194F86C30DB070DD50221154A16488D
:1046E80041F0BBFE6FF07705201D41F0BFFE08F0DA
:1046F800FBF8284638BD45F055F938B901210F4A6D
:104708000D4841F0AAFE6FF01205EDE7204600F0D3
:10471800ADFF05460028E7D10146242204F1280010
:104728005EF04FFE94F86C3043F0010384F86C306F
:10473800DAE700BF411308089C3F07086B13080815
:1047480070B5044608F0BCF8204641F088FE94F89D
:104758006C30DA070DD40221254A264841F07DFE47
:104768004FF0FF35201D41F081FE08F0BDF82846C6
:1047780070BDC3F340019B0707D502211E4A1D489F
:1047880041F06BFE6FF07705ECE7A06943F0E6FABD
:104798000646A06943F072FB054628B10121174A75
:1047A800144841F05AFEDDE7A36F4BB1314620466D
:1047B80042F036F80546A0B1A06943F087FBD1E77F
:1047C800A06943F003FBA0670028EFD101210C4A40
:1047D800084841F042FEA06943F078FB6FF00B05F2
:1047E800C0E794F86C3043F0020384F86C30B9E702
:1047F8008E1308089C3F0708B4130808DA13080842
:10480800F613080838B590F86C3004469B0708D4AE
:104818000221144A144841F020FE6FF0770528461B
:1048280038BD41F01CFE0021204601F0B9F820B146
:1048380001210E4A0C4841F010FEA06943F046FBE6
:10484800054620B101210A4A074841F006FE94F8BE
:104858006C30201D23F0020384F86C3041F006FE12
:10486800DDE700BF121408089C3F07083914080840
:10487800571408082DE9F04385B006460C469046C3
:1048880041F0F6FD0546B8F1000F07D0304641F07B
:10489800F4FD012810D1B5FA85F56D0901342946D2
:1048A8003046E2B241F0D5FF814650B90121234696
:1048B800324A334841F079FB0024204605B0BDE870
:1048C800F0834768B8F1000F09D03868796801AB00
:1048D80003C33A7A01AF1A7007238DF80530F18DBA
:1048E8007B883046994228BF194642F004F90446AD
:1048F8000028E1D0038A428A4169D21AC36800F1CC
:104908000C085B1AD21A3B7839469A4228BF1A46D5
:10491800404641F077FDD9F80C90B9F1000F08D165
:10492800218AF38D9942C8D94046C91A41F085FDBC
:10493800C3E7D9F8040083681B6B13B9D9F8009052
:10494800EBE7294698470028F8D0071F57F8041FB7
:104958000029F3D008780028F0D0628A238AA2EBD5
:10496800030C6269E3689B1AACEB0302904294BFA4
:10497800024692B2404641F045FDE7E78714080831
:104988007C3F070838B50446806F41F01CFD05469A
:1049980041F0FDFC2046294601F04AFA044638B1A8
:1049A80004480121044A41F0F7FA2846FFF738FE87
:1049B800204638BD7C3F0708AD14080838B580216B
:1049C8000446806943F025FA054678B10146204639
:1049D80001F02EFA044638B106480121064A41F092
:1049E800DBFA2846FFF71CFE204638BD6FF00B04A3
:1049F800FAE700BF7C3F0708CC14080800232DE91C
:104A0800F04F93B005930B7E044633F080060F46B3
:104A180015460AD00121AD4AAD4841F0BDFA6FF004
:104A28000406304613B0BDE8F08F82B10846FFF7A0
:104A3800F7FD7B7EDA0704D49D07F2D53B7E002B79
:104A4800EFD1204613B0BDE8F04FFFF79BBF4A7E79
:104A580000F12809900705D5802B09D13846FFF7C2
:104A6800DFFDDEE7910700F03184002B40F02E8453
:104A7800D3071ED53B8A082B12D1FA68394613682A
:104A88000020A3625368C9F8043041F0A3FC0590E4
:104A980080B18F4801218F4A41F07EFA059805E0E0
:104AA8008B4801218C4A41F077FA3846FFF7B8FD68
:104AB8001EE00597FFF718FA002394F82850874A54
:104AC80015F0600F8350C5F341131CD0032B40F041
:104AD80064836FF08505FFF707FA804B1B58002B9E
:104AE80000F09A83002D00F0698305980028DDD135
:104AF800484641F0F5FD0346A069002B00F02184EB
:104B0800802100F027BC484641F0EAFD94F829309E
:104B1800002840F02C81013B0A2BDAD801A252F878
:104B280023F000BF6B4C0108DB4A0108F14C010877
:104B3800DB4A0108594B0108DB4A0108DB4A010836
:104B4800DB4A0108BF4B0108DB4A0108334C010866
:104B5800A069618D03697F2993F88030B9D8A28D47
:104B6800002AB6D1E28D002AB3D1EE06B1D194F86D
:104B78003020022A02D14FF0FF35ACE71D070BD5D4
:104B8800C9B241F0E3FD054648B1638D0121544A9D
:104B98004F4841F00AFA9EE7012384F8393094F827
:104BA8003030012B05D1638D1BB984F830300025D6
:104BB80091E70123F9E7204641F05AFC628D01464E
:104BC800FF2A86D8E38D002B83D194F82830D806A5
:104BD8007FF47FAF94F83030002BCCD092B9618D40
:104BE80094F838308B42E2D02046C9B200F0D8FEA3
:104BF800638D054668B1012100903A4A344841F076
:104C0800DEF968E72046D2B241F049FE0028E6D135
:104C1800B1E7002B14BF02220122052184F83020BD
:104C280020461A4641F0B0FFC1E705F01F05012DE7
:104C38007FF44FAFE38D002B7FF44BAF628DFF2ADB
:104C48003FF647AFA18DFF293FF643AF94F83030C8
:104C5800022B90D12046D2B2C9B241F0D0FE05460F
:104C680039E7E38DA68D002B7FF433AF94F830300D
:104C7800002B80D0012B02D1002E7FF47CAF15F0E1
:104C88001F0515D0022D92D1B4F82A80B8F1000F73
:104C98008DD1F6B23146204601F032F9421C054664
:104CA8003FF419AF42463146204641F01FFD12E756
:104CB800002E7FF460AF638D012B7FF478AF94F8FA
:104CC8006C3066F3C30384F86C3070E7EF1408089F
:104CD8007C3F070827150808101508080C00000075
:104CE800491508086B150808A38DE28DDEB2002A65
:104CF8007FF4EFAE628D022A11D105F01F0535430E
:104D08004FEA13217FF4E5AE0122A06941F0FEFCD1
:104D180000287FF4DEAE012384F8393047E794F8A1
:104D2800301000293FF427AF012902D1002B7FF46E
:104D380022AF15F01F050FD0022D7FF438AF002ADF
:104D48007FF435AF3146204601F0B8F8431C0546DC
:104D58003FF4C1AE0122A6E7002B7FF40CAF012A75
:104D68007FF425AF94F86C3043F00803ABE70A2BC7
:104D780063D8DFE813F00B00620062006200620093
:104D880062003A006200DD016200F201E38D022B4D
:104D980053D194F83030002B4FD0012BA18D01D185
:104DA80000294AD115F01F050ED0022D17D0002674
:104DB8000221204641F09FFE054618B131460C30CD
:104DC80041F031FB0595F2E6002936D194F86C30B4
:104DD8009E0806F00206C3F300131E43E8E72046C8
:104DE800C9B241F0ACFE0646E2E7618DED064FEA36
:104DF8001123C9B207D0002320460AA90A9341F01B
:104E0800BEFC0A9DDEE7013B0E2B16D8DFE813F047
:104E18000F003000380015001500D20036001500CC
:104E28001500150015001500150015000F01204686
:104E380041F01EFB18B1012818D00025C2E7266FE3
:104E4800002EFAD0B4F82E8033782046984528BF33
:104E58009846414641F04FFE05460028B2D04246EA
:104E6800314605F10C0041F0CDFAABE7666FE7E794
:104E780000222046FFF7FEFC0546A3E70122F8E7DB
:104E88000A462046032141F07FFB80460028D4D003
:104E980041F021FCE58D98F81530B8B998F8146000
:104EA8008DF82930AE428DF8286028BF2E46D8F8F4
:104EB800103031461B882046ADF82A3041F01BFEE1
:104EC80005460028B9D032460AA9CAE74FF0000AB9
:104ED800B44A8DF81130D8F808308DF810A01A406F
:104EE800B14B9A4255D1102106A804F09DF8061E30
:104EF80036DB0AAB102E984628BF1026AB4806AA08
:104F0800564503F1020334D8B6000236F6B28DF8DE
:104F18001060AE4228BF2E462046314641F0EBFDD8
:104F28000546002889D0022EB34628BF4FF0020B51
:104F38005A46A6EB0B06C34600F10C0A504604A9D4
:104F480041F060FA730808EB56025A4528D1F00779
:104F58007FF538AF504618F8031041F05CFA31E796
:104F680058367FF46AAF0121914A924841F014F80B
:104F780063E712F8011B0AF1010A4FEA111C01F05C
:104F88000F0110F80CC0415C03F802CC03F8011CB7
:104F9800B6E798F81460D8F810808DF81060B8E774
:104FA80050461BF8011BCDE9022341F03CFADDE92C
:104FB8000223CAE7204641F05BFAD4E91C530028D3
:104FC80008BF1D460A2300268DF8283006232046F0
:104FD800CDF82A60CDF82E608DF8293041F04DFAD1
:104FE80001287FF42AAF002D3FF4ECAE6B882046F1
:104FF800ADF82A302B798DF82C306B798DF82D305F
:10500800AB798DF82E30EB798DF82F306B7C8DF8DD
:105018003030E68D9DF828309E4228BF1E46314626
:1050280041F069FD054600287FF44DAFCAE62046E9
:1050380041F01EFA20B101287FF4FFAE636F00E053
:10504800236F002B3FF4F9AE5B88B3F5007F7FF642
:10505800F4AE594B04F14C060A9300238DF82C301A
:10506800E36C9E4208BF0023BDF82A2093B1597D06
:105078000F2908D1197D0A44ADF82A209DF82C2063
:1050880001328DF82C20226D9A4201D01B68EBE783
:10509800BDF82A20B4F82E802046904528BF9046B7
:1050A800414641F028FD054600283FF4C6AE9DF86C
:1050B800282000F10C0A424528BF424650460AA95A
:1050C80041F0A0F99DF82830434594BFA8EB0308A8
:1050D800A8EB0808B8F1000F3FF474AED4F84CB050
:1050E800B3453FF46FAEBBF1000F3FF46BAE9BF8D6
:1050F80015300F2B15D19BF814205046424528BF78
:105108004246DBF8101041F07DF99BF81430434516
:1051180094BFA8EB0308A8EB0808B8F1000F3FF408
:1051280051AE236D5B453FF44DAEDBF800B0DAE7D6
:1051380094F83030002B3FF480AEE18D01297FF4E4
:105148007CAE94F83860204641F0D5FC054600282E
:105158003FF438AE31460C30FFE605F01F05012D4F
:105168007FF46BAE204641F088FB00283FF465AE23
:10517800A38D4268FF2B3FF660AE12799A42FFF486
:105188005CAEDAB20F2A3FF658AEE18D01297FF402
:1051980054AE234493F83A60D5E7204605A941F078
:1051A800EEFA5CE500FF020000030200E96A080865
:1051B8008E1508087C3F0708050F050045F003F821
:1051C8000A220023FBF748FE644BD3E8AF1F41F2E5
:1051D8008732461A9642624A39D9D3E8EF6F8E422F
:1051E80004D1C3E8EC0FBCF1000FF6D12FD1D2E8FF
:1051F800EF3FC2E8E15F0029F9D123B10221594A02
:10520800594840F0D2FE0221584A574840F0C4FE9F
:10521800FEF76AFE564B1D58002D7FF466AC7B7E68
:10522800E28DD9071BD5484641F05AFAB8B9BAB148
:105238002946A06942F0D9FD0146059000283FF4AF
:1052480057AC204613B0BDE8F04F00F0F1BDD2E8EE
:10525800EF3F0133C2E8E13F0029D9D0F7E73AB977
:105268002046FFF7ABFB00287FF442ACFFF7E9BB11
:10527800484641F035FA059D18B92846FFF7D0F998
:10528800EEE7002D3FF434AC2946204600F0D0FD6F
:1052980008B128460AE4A069036993F8801011F060
:1052A80004017FF4CEAB42F0B4FD054600283FF47C
:1052B8001FAC0146204600F0BBFD00283FF4C1ABFF
:1052C80001212C4A284840F067FEE2E752077FF5A3
:1052D8000FAC002B3FF4C2AB3846FFF7A1F994F8A6
:1052E8003930002B3FF49DAB94F82930052B0CD1B5
:1052F800618DA069C9B241F029FA054628B1638DCC
:1053080001211D4A184840F050FE94F82930032B1B
:1053180011D1638D022B0ED1A18D00220E0A3146C8
:10532800A06941F0F3F9054628B101213346134A33
:105338000D4840F03AFE00232E4684F83930FFF736
:1053480070BBE38D002B3FF4DBAB0599003918BF28
:105358000121C90142F060FCFFF773BBF43700205C
:10536800F0370020B01508087C3F0708C415080866
:105378000C000000ED150808491508081116080862
:105388000B7810B4062B14D10369D3F89C20EFF3E3
:105398001184102383F31288BFF36F8F00204B68AA
:1053A8001860506A60B9C2E9083384F31188BFF302
:1053B8006F8F0022002304485DF8044B44F0F1BBD2
:1053C80003605362F1E700BF2411002030B589B0B3
:1053D800002200230024CDE906236FF007034FF4D1
:1053E8008062CDE90334CDE90144154B1549009499
:1053F800154806F069FF1549134844F08AFD144B17
:1054080014498B4207D30020134B14498B420CD309
:10541800002009B030BD03F11402D2E8EF0FC2E852
:10542800E54F002DF9D11833EBE703F11402D2E868
:10543800EF4FC2E8E50F002DF9D11833E6E700BFBA
:10544800C154010800550020A02800205A3008083F
:10545800001300206013002060130020C0130020F8
:1054680038B50D4641F009FA30B90121BDE8384098
:105478000F4A104840F090BDC46804B938BD2B7875
:10548800032B05D0052B0ED0022B08D02468F4E797
:10549800606883685B69002BF8D09847F6E7606816
:1054A80083689B69F7E760688368DB69F3E700BF97
:1054B800381608088C3F07082DE9FF4110274FF0E0
:1054C800FF334FF0FF32644801A906F0EBFA039B63
:1054D8001B69D3F89C40236A93B1EFF3118287F3D9
:1054E8001288BFF36F8F216A29B1606A0B68814205
:1054F800236208BF636282F31188BFF36F8FC9B953
:105508009DF80430062BDAD0072BD8D801A252F820
:1055180023F000BF61550108555501088955010858
:1055280067550108BD550108AB550108C754010866
:10553800515601080B7E20465D06D1F81E2002D187
:10554800FFF75CFAC7E741F0E8F9C4E70022012158
:10555800204641F019FBB2E700221146F8E794F81B
:105568006C3043F0040384F86C3094F83030022B2C
:1055780003D1204601A9FFF773FF00220321E7E7C3
:1055880094F86C3023F0040384F86C3094F83030CD
:10559800022B03D1204601A9FFF762FF0022022156
:1055A800D6E794F83030022B89D1204601A9FFF7BD
:1055B80057FF84E794F86C30A66923F0040384F855
:1055C8006C30D6F808803369A033D3E8AF3F9A0728
:1055D8001ED53046D8F83C309847D8F824300021FA
:1055E800304698470546D8F840303046984795B138
:1055F8001A4A01211A4840F0CFFC00220421204613
:1056080041F0C2FA002D3FF45AAF2A4607219FE71E
:105618004FF0FF35ECE72946204600F0C1F9054672
:1056280008B1104AE5E7A06942F012FC831E58420F
:10563800584194F86C3084F8305023F0680343EAFA
:10564800401384F86C30D8E70121074A044840F039
:10565800A3FC0621029A7BE724110020671608089C
:105668008C3F070895160808C116080838B5024681
:1056780005460C49806942F049FC044630B10121D5
:10568800094A0A4840F088FC204638BD85F83800A9
:10569800284600F043F904460028F5D0A86942F0EE
:1056A80064FCF1E789530108D11608088C3F070804
:1056B800F8B501231D460C68002C35D063F07F0235
:1056C800D6B202F07F02103224FA02F7FF0716D58D
:1056D800046824FA02F7FF0708D433461348012167
:1056E800134A40F062FC6FF01500F8BD05FA02F2AB
:1056F80024EA020404600C6824EA02040C60DC401A
:10570800E6070ED5026822FA03F4E40700D4E5E7B9
:1057180005FA03F422EA040202600A6822EA040293
:105728000A600133102BC6D10020DEE7BC3F070812
:10573800F81608082DE9F04F0026536891B0D46890
:105748000A900891069202930E96039674B9039BE9
:10575800029A09339BB293701B0AD370069B167189
:10576800DC68002C40F0C780A346AEE04FF0000A8A
:105778006068CDF83CA083681B6B002B00F0AC8000
:1057880008999847002800F0A7803546C4E903AA7D
:10579800A0F1040959F8043F0BB11A789AB9B54237
:1057A80040F29780E3680F9A1343E3606068836868
:1057B8009B6A002B00F0928098478346002800F0EF
:1057C8009080534A7DE05A780B2A08BF9D70D9F81B
:1057D80000305A78042A10D1E2680F990A43E2602F
:1057E800DA78002A5CD101229D702369AA4013430C
:1057F80001352361EDB2CDF83CA0D9F800707B7873
:10580800052BC7D16FF0120B4FF001080A9B9B695B
:10581800099379793A790E9B42EA0122ADF836204C
:1058280097F902205FFA88F1002AACBF424641F09E
:1058380080010493B7BF4BB24FFA88F321F080027E
:105848000793A8BF0793049BB8BF103223FA02F04E
:10585800C0072CD40F9B23FA02F20593D30726D452
:10586800BB79FA78099800930DF136030B9142F051
:1058780049F90B998346D0B9079BB970002B4FF0B3
:105888000103BCBF21F0800110318B4004980599B9
:10589800BDF8362019431843CDE90E01BA8079E7DF
:1058A8006A1E9A700FA90EA8FFF702FFA3E708F176
:1058B8000108B8F1100FACD1BBF1000F3FF46AAF8B
:1058C800144A0121144840F067FB584611B0BDE85E
:1058D800F08F6FF0150BF3E7354667E76FF0850B30
:1058E8006FE76068089940F0E8FF039B2E46034481
:1058F800246803932AE7E36804F10C01A3600EA867
:10590800FFF7D6FE08B924682BE76FF0150BDCE724
:105918003917080815170808BC3F070870B58369C8
:1059280005461B69026F93F88030C3F34113022BBD
:105938000CD0032B0CD0012B0CBF10230823D371E0
:10594800EE6D3EB96E6DBEB9344611E02023F6E720
:105958004023F4E7324601212846FFF7EBFE0446D0
:1059680040B173685B790B4A01210B4840F01DFB7D
:10597800204670BD3668E4E7324600212846FFF726
:10598800D9FE044618B173685B79044AECE73668B7
:10599800D9E700BF5D170808BC3F0708801708084B
:1059A8002DE9F04105460E4640F062FD95F8383085
:1059B800804633B3284640F060FF0746F0B1014601
:1059C800284640F0CAFF10220446002105F13A009B
:1059D8005DF0F7FC002385F83830FF683FB984B1E3
:1059E80019491A4840F028FF2046BDE8F081786838
:1059F80083685B6A03B198473F68EFE76FF03C0440
:105A0800EEE71EB985F838600024EDE732464146D6
:105A1800284640F01EFF074690B10246284640F04F
:105A2800C6FF04460028DFD185F83860FC68002CE2
:105A3800EAD0606883681B6A03B198472468F6E770
:105A48006FF03C04D0E700BF39140808743F07081A
:105A58002DE9F04105460F461446D2F8048040F07F
:105A6800EFFE95F86C30D9070BD54749474840F009
:105A7800E3FE6FF00F07281D40F0E9FE3846BDE849
:105A8800F081012F0AD1284640F0F7FC30B940498F
:105A98003E4840F0D1FE6FF08507ECE798F80730F4
:105AA8009A0607D5AB691B6993F880309B0701D428
:105AB8003849EDE71FB1012F06D03749E8E7EB6D0C
:105AC8002BBB05F1540603E06B6DABB905F15C0621
:105AD800002233680BBB002FD5E91C2308BF1346EF
:105AE8005B7C626803F10103DBB25371D5E91C12D8
:105AF80008BF0A46537422E09C4206D1274923482E
:105B080040F09AFE6FF01507B5E71B68DDE79C4289
:105B180001D12349F3E71B68D2E79C4221D12368CE
:105B2800CAB972683360944200D17360002323605D
:105B380063685B7902211B4A144840F036FAA16871
:105B4800B9B1284640F03AFD074668B116490F48F2
:105B580040F072FE8FE7136073689C4208BF726062
:105B6800E4E71A461B68B5E7A06840F0B4FD88F87A
:105B780006000023236073681BB9C6E900440027A8
:105B880079E71C607460FAE7D1170808743F0708C2
:105B9800F3170808AD17080811180808311808087D
:105BA8004E1808086B18080888180808F8B505463C
:105BB80000AF29B301290BD1184C194E2BE06368AB
:105BC80028461968FBF7A2F9B8B11834B442F6D3DD
:105BD8006C4688B06A46134BCDE905354FF400731F
:105BE800ADF81C30104B42F8103F00234FF4E2513F
:105BF8000E48FDF7D9F8A54600242046BD46F8BD55
:105C08000B4C0C4EE2E7636828461968FBF77EF9EF
:105C18000028F2D01834B442F5D3D9E76013002035
:105C2800C0130020BF18080803000001843F0708BC
:105C3800001300206013002070B5012501F07F03D8
:105C480011F0800F18BF10339D4090F83030044693
:105C5800022B06D001210C4A0C4840F09DF9002087
:105C680070BD90F8386040F003FC3246014620468B
:105C780040F0EFFD0028F2D0C0680028EFD083681C
:105C88001D42EDD10068F8E7DD180808843F0708D1
:105C98002DE9F84305460846114616469846FFF78B
:105CA80085FF0446002843D0284640F0FFFD95F8BC
:105CB8006C30DA0702D5204A012109E0D4F80490B3
:105CC80004F11407D7E8AF3FDB070CD502211B4AC4
:105CD8001B4840F061F96FF00F04281D05F0B8FF6C
:105CE8002046BDE8F883D9F804301BB1AB4201D097
:105CF800144AE1E742463146284640F0AAFDA0B1E1
:105D08000023236003696BB9C0E90344D7E8EF3F78
:105D180043F00103C7E8E23F002AF7D10024C9F89D
:105D28000450DAE71C600461F0E76FF03C04D4E744
:105D38006FF01204D4E700BFD11708080219080849
:105D4800843F0708241908082DE9F04F83B000AFF5
:105D58007B6097F830304C680E463B608146904631
:105D680040F086FBA36801461B6B33B96FF015043E
:105D780020460C37BD46BDE8F08F204698470028DE
:105D8800F4D00024051F06F10C0A55F8041F09B1C8
:105D98000B782BB9002C14BF00246FF03C04E7E704
:105DA8004B78042B0ED1002C3CD18B787A68934227
:105DB800EBD1CB783A689342E7D10B79002BD7D057
:105DC8000124E2E7052BE0D1002CDED0B8F1010F69
:105DD80091F802B009D0B8F1020FF1D152465946F4
:105DE800D9F8180040F071FE04E05246D9F81800BE
:105DF80040F04FFE04460028E2D06D468AB06A465D
:105E0800F368CDE907B3062307490990CDE90518DA
:105E180042F8103F00234FF441510448FCF7C4FFF7
:105E2800AD46A5E70024A3E764190808B43F0708AE
:105E38002DE9F0410B7E0C465906054637D16BB368
:105E480040F056FB40B11B4801211B4A40F0A4F822
:105E58004FF0FF30BDE8F0812846D5F87080268ADB
:105E6800EF8D40F005FBF8B1421E534253419B01B0
:105E7800228A9AB1BE42324628BF3A46E98D9142FB
:105E88000CD9B2FBF3F103FB11223AB994F918309B
:105E9800002BBEBF637E43F0080363762146A869E2
:105EA800BDE8F04141F014BF98F80730E0E76FF023
:105EB8001500CFE7A43F0708A019080870B50646E3
:105EC80080690C4641F0A8FE054638B102212346F8
:105ED800094A0A4840F069F8284670BD012214F0C2
:105EE800800F18BF24F08004736B18BF1034A240D1
:105EF8001A437263F0E700BFB4190808A43F070803
:105F080070B5054680690E4641F0B1FE044638B1C9
:105F180002213346054A064840F047F8204670BD3E
:105F2800314605F1340040F0A6FDF7E7CB19080823
:105F3800A43F070870B50646EFF31181102383F3D9
:105F48001288BFF36F8F1B4D2A6881F31188BFF346
:105F58006F8F526892F86C20D20705D4BDE8704064
:105F68000A22002306F062B9EFF3118283F3128844
:105F7800BFF36F8F2C682CB1696823688C422B6043
:105F880008BF6B6082F31188BFF36F8F44B16068FC
:105F980004F10801C36998472146074843F09EFD6C
:105FA8002B6833B13046BDE870400022002306F06C
:105FB80005B970BDF8370020B010002030B585B0A5
:105FC800CDE90012054600220023144803A905F074
:105FD800CFFC0246E8B9DDE90001039B5D600833A8
:105FE80083E80300EFF31180102383F31288BFF3D3
:105FF8006F8F039B1A600A4A516861B9C2E900337E
:1060080080F31188BFF36F8F00220023054806F044
:10601800D5F805B030BD0B605360F1E7B010002033
:10602800F83700200000002073B5102504698DF8AA
:106038000710EFF3118685F31288BFF36F8F0122E3
:10604800206C0DF107013FF020FE86F31188BFF3A5
:106058006F8F012812D043F056FFC8B10122104BB0
:10606800D3E8EF1F002903D1C3E8E02F0028F7D1B8
:1060780004D102210B4A0C483FF08EFF237F2BB13D
:106088000A22002304F1480006F098F802B070BD17
:10609800A37E002BE2D000210A2044F03CF8C8E798
:1060A80000380020F51908086C3F070838B50024A7
:1060B80005690E492B6C05F14800C3E90144DC6011
:1060C800AB6BC3E90144DC6043F011FF05F17800D4
:1060D800074943F0E0FE074905F1280043F0DBFEDD
:1060E800284640F076FD204638BD00BF21620108F1
:1060F80069630108356401082DE9F341036906461F
:106108000D46D0F804801C690F7E002A32D00B8A15
:1061180071323E480BBF022101213D4A3D4A00939E
:106128003B463FF04CFF30462F7E40F0C6FD87428D
:1061380004D1042104F1880040F073FE30462F7E1C
:1061480040F0C9FD874204D1052104F1880040F0E0
:1061580068FE30462F7E40F0A2FD874203D104F14D
:106168008C0005F05DFE2946404602B0BDE8F041CE
:1061780040F0E2BC40F0A1FDB84214D12A8AE96897
:10618800A06B3FF082FD28B1236A1BB104F12800FF
:1061980005F0A4FF04F18800042140F042FE04F158
:1061A800780005F09BFF30462F7E40F094FD874233
:1061B80015D1236A1BB104F1280005F08FFF0521D2
:1061C80004F1880040F02DFE237F9BB900234FF493
:1061D8007A7204F1480005F0F1FF01232377304675
:1061E8002F7E40F05CFD8742BDD104F18C0005F0A4
:1061F800B5FDB8E7236C5A89DB889A42EFD00022B4
:10620800002304F1480005F0D9FFE8E76C3F0708D0
:10621800141A0808381A08082DE9F04750F8483CBD
:1062280000F140075B68054600213846D3F8009026
:1062380040F02FFD002864D00121384640F029FDA8
:10624800804600285DD155F8083C5A89DB889A4277
:1062580003D115F82D3C002B53D0D7E8EF4F44F06D
:106268002003C7E8E23F002AF7D114F0200448D100
:10627800484640F030FD002282460023224840F084
:106288008BF8064650B93846052140F0CAFD284625
:10629800BDE8F0470A22002305F090BF80F818A057
:1062A80015F82C3C33B1428AC16855F8080C3FF008
:1062B8000CFD0446214606F10C0040F09DF85CB147
:1062C800D9F8040040F08BFDB4FBF0F303FB104455
:1062D800B4FA84F84FEA58183146484605F82D8C28
:1062E80040F012FC68B10121084A09483FF054FE09
:1062F8003046FEF795F93846BDE8F047052140F0ED
:1063080090BDBDE8F08700BFA8110020591A080801
:106318006C3F070838B503461B6940685D68AC6880
:10632800A37A84F8223094F82D3084F82330A376A9
:10633800696849B1237C3BB940F040F930B101218B
:10634800054A06483FF028FE002038BD686840F03E
:10635800C2F92074F8E700BF6B1A08086C3F0708F9
:1063680070B550F8782C00F11004526803460021EB
:106378002046156840F08DFC00284DD001212046AC
:1063880040F087FC002847D153F8402C6868938870
:10639800918916695B1A9BB2F61A40F020FDB0424B
:1063A8003AD8D4E8EF3F43F01002C4E8E12F0029BF
:1063B800F7D1DB0606D5BDE870400221174A184818
:1063C8003FF0EABD284640F078FC0022064600234C
:1063D80014483FF0E1FF0446F0B10676686840F0E3
:1063E800FEFC638A984203D2686840F0F8FC83B2E6
:1063F80021462846638240F087FB68B1284640F072
:106408005CFC034606480121074A3FF0CEFD2046C2
:10641800BDE87040FEF704B970BD00BF951A0808C2
:106428006C3F0708A8110020B51A080838B550F8BD
:10643800083C044633B9BDE8384001212A4A2B48B4
:106448003FF0AABD50F8283C00F160055B680221C6
:106458001A68002383828383284640F01AFCB8B167
:1064680054E9023110699847637D1BB104F150006B
:1064780005F034FE0521284640F00BFC98B9637FEF
:106488006BB10022002304F1200005F097FE0AE01A
:106498000321284640F0FDFB0028E1D1E4E714F889
:1064A8000D3C002BEDD10221284640F0F2FB38B11B
:1064B8002369DA885B899A4202D0204605F00EFEED
:1064C8000321284640F0E5FB60B1A26993889189D1
:1064D80012695B1A9BB29A4204D02046BDE8384044
:1064E80005F0FCBD38BD00BFDA1A08086C3F070884
:1064F800D3B5002600270446CDE9006705483FF0DC
:106508004FFF28B1230658BF0023047658BF0382E3
:1065180002B0D0BD2C1200202DE9F04383B0002337
:106528004FF0010805691C4C1C4E02AF28602B7700
:1065380085F8203005F12409B442234601D3002010
:1065480019E095F820201034CAB16C4688B01B6851
:1065580002AA1349C2E905134FF400739383114B40
:1065680042F8103F104800234FF4E251FCF71CFC9E
:106578006FF00B00A5460437BD46BDE8F08385F8EB
:10658800208054F8043C4846009354F8101C54E901
:10659800032340F012FFCFE7A8B10808B8B10808F4
:1065A8003C1B080803000001C43F07081FB5CDE9DC
:1065B800010103924FF0FF324FF0FF3301A9034866
:1065C80043F0EFFA002005B05DF804FBF41000205A
:1065D8001FB500230190CDE902334FF0FF324FF091
:1065E800FF3301A9024843F0DCFA05B05DF804FB6B
:1065F800F41000202DE9F041044617460E460068C5
:1066080040F043FD31463A468046FFF771FFD4F823
:106618007B300546DB1B0146C4F87B30206840F020
:1066280073FA88B10B4A434601210B483FF0BDFC81
:106638003146204640F0F4FD2846FDF7F1FF20469C
:10664800BDE8F04140F0B8BDA37F0133A377BDE8B2
:10665800F08100BFB51A0808C43F07082DE9F84FB4
:106668000446006840F026FD4FF030090746E37FF6
:10667800012B1ED82368D3F810B0D3F804A09BF8D8
:10668800616009FB06B62436304640F0BCFE314650
:1066980002468046504640F023FD9BF81F300546D1
:1066A80033B1A8EB00023146504640F019FD0546CB
:1066B8000DB9BDE8F88F204640F0CFFC2A460146C8
:1066C80006463846FFF714FF05460146206840F0A5
:1066D8001BFA80B101213B46094A0A483FF065FC94
:1066E8002846FDF79DFF3146204640F099FDBDE85C
:1066F800F84F40F061BDE37F0133E377B7E700BFB0
:10670800B51A0808C43F07082DE9F04FB94F89B0FA
:106718004FF0FF324FF0FF33B74805A905F0C2F933
:10672800059E069D3469002D40F09080257704F180
:10673800240694F820309D42C0F2828004F11803A8
:10674800D3E8EF2F22F00202C3E8E12F0029F7D1A6
:10675800D3E8EF1F21F00401C3E8E21F002AF7D1B4
:1067680004F11803D3E8AF3FDB07D1D5237F022B11
:1067780000F08E81032B00F0878153BBDDF814A055
:10678800DAF81050EB7F23BB504640F093FC81466B
:10679800284640F062FC4FF400720146064648461F
:1067A800FFF7A6FE80460146504640F0ADF90028A6
:1067B80000F0668101214B46904A91483FF0F5FB75
:1067C8004046FDF72DFF3146284640F029FD40F0B0
:1067D800F3FCA37F002B9BD1237F012B40F07D810D
:1067E800302304F1630694F86150304694F862103F
:1067F80003FB054500F060FA24350246314623695B
:10680800284600F077FA0646C4F88400284640F087
:10681800F0FD8146284640F0F1FD8046284640F0CC
:10682800F2FDE26D3044002A40F03B81002840F040
:106838003381284640F00EFE003818BF01202CE1B5
:10684800304640F0CDFD0135303672E7DDF81C806A
:10685800D6F804A095F81890B8F1000F21D02B8A2B
:1068680018F1710F6648009308BF02214B4616BF06
:106878000121644A644A3FF0A2FB304695F818802B
:1068880040F018FC804540F0EF80E37F013BE37760
:106898002046696940F0C4FC2946504640F04CF94E
:1068A8005EE7304640F006FC484540F09580237F7F
:1068B800D5F80C80B5F810B0002B49D1BBF11F0FEB
:1068C80042D1D8F80030BB423ED1414604F15403CE
:1068D80008F11C0251F8040B914243F8040BF9D15A
:1068E8000A881A808A7842219A70552384F873306E
:1068F800532384F8743084F87630A36DE26DC4F8BD
:1069080077300023C4F8803094F86030C4F87B20D6
:106918009A0684F875100FD194F8612094F8203005
:106928009A4209D294F86230013B0F2B04D8012314
:1069380084F87F302377A0E7206840F0B1FB02237A
:1069480084F87F300423F5E7204640F035FC94E7CF
:10695800032B92D1302394F8619003FB0949D4F8B2
:10696800803009F124095B44C4F88030BBF1000F82
:1069780016D0484640F047FD90B141465A46484631
:1069880040F053FD804628B902215B461F4A1C4847
:106998003FF00BFBD4F87B30A3EB0803C4F87B3043
:1069A800D4F88020E36D9A420DD2484640F02BFD82
:1069B80000287FF462AFD4F88020E36D9A4202D2B7
:1069C800206840F083FB484640F044FD003818BF7B
:1069D800012084F87F00B5E7304695F8189040F01C
:1069E80054FB81457FF449AF237F052B10D184F8F0
:1069F8001C8042E755534243F4100020B51A08089A
:106A0800C43F0708141A0808381A0808531B08084E
:106A1800022B7FF432AF4FF030092A8AD4F8803045
:106A280094F861801344C4F8803023681969D3F856
:106A380004B091F8613009FB031124310846039131
:106A480040F0E1FC03990246584640F049FB002813
:106A58007FF413AFD4F87B3013B1206840F020FBEB
:106A680009FB08402430AFE7304695F8188040F01D
:106A78000CFB804502BFA37F03F1FF33A37707E731
:106A8800EB7F0133EB77A4E62046FFF7E7FDA0E6AE
:106A9800204640F0D5FB9CE6022084F87F000423C2
:106AA8001AE094F9601040B90029206802DA40F031
:106AB800F7FABEE640F00AFBBBE6002914DA90427A
:106AC80002D8B9F1000F06D1206840F0E9FA022394
:106AD80084F87F30E3E702232377237F022B0ED14C
:106AE800204640F0ADFB13E6904202D8B8F1000F03
:106AF80003D1206840F0EAFAE9E70323ECE7032B27
:106B080003D12046FFF7AAFD02E6042B7FF400AE6E
:106B1800A37F2BB101211D4A1D483FF03DFAF7E53F
:106B2800206840F0B2FA8046204640F096FA0546C2
:106B3800024604F1730304F17F0153F8040B8B42FE
:106B480042F8040BF9D11B782946137040460D22F0
:106B5800FFF7CEFC0646014620683FF0D5FF78B126
:106B68000C4A434601210A483FF01FFA3046FDF718
:106B780057FD2946204640F053FB40F01DFBC7E572
:106B8800A37F0133A37705232377C1E5791B080881
:106B9800C43F0708B51A0808802938B50D461446B9
:106BA80021D083290DD019BB80235371832303205F
:106BB800117193710023E07023706570A370043025
:106BC80038BD0223137101235371002393710A23E3
:106BD800D37108224168A0185CF02AFC064B0E20ED
:106BE8001B882382E6E7044B02201B889380E1E799
:106BF8006FF08500E4E700BF886908082DE9F041D7
:106C08008769D0F82480BA4228BF3A46B2FBF8F424
:106C18000646C269234600683FF033FB0546C0B903
:106C2800B7FBF8F7A7420BD1002205213068FCF723
:106C3800E7FB28B101210A4A0A483FF0ADF90125CE
:106C4800F3692344F3613DB10020074BB362BDE80B
:106C5800F08100240125E7E7706A6043F7E700BF89
:106C68009A1B0808C43F07080203000C81420B4620
:106C780007B509D302210D4A0D483FF096F96FF088
:106C8800150003B05DF804FB6AB101391144814273
:106C980001D28B4207D90221009305481346054AC1
:106CA8003FF08DF9EBE70020EBE700BFB11B0808C8
:106CB800C43F0708C81B08080C290346084616D114
:106CC8001B78252B12D009D8122B10D8084A42FA63
:106CD80003F313F0010F08BF0620704703F0FD020D
:106CE800282A03D05A2B08BF0A2070470A20704769
:106CF800F6FFFBFF2DE9F041984690F82C3086B05E
:106D080023F00C0380F82C300023C0E9043383619E
:106D1800062A04460F460B7840F010810BBB4B79CE
:106D28005B0724D490F82C309F070DD402234FF42E
:106D380068521946002584F8283084F8291062859D
:106D4800284606B0BDE8F08140F0B9FA0028EDD138
:106D5800002319461A46EDE70223052145F20232BF
:106D6800E8E7032B36D14E7916F0040604D0022347
:106D780005214FF41052DDE790F82C308DF80760AC
:106D880043F0040380F82C307023ADF8043090F8F9
:106D980029300D7903F00F038DF806300A23122DE0
:106DA80028BF12258DF80B30438D2A465BBA404622
:106DB80001A98DF808608DF809608DF80A600396BE
:106DC800ADF81030ADF81260ADF814605CF0D3FA8D
:106DD800A662B5E71B2B00F0898009D8122B1AD0C0
:106DE8001A2B61D00121B24AB2483FF0DEF8BEE763
:106DF8001E2BF7D14B795E07B9D40B7913F0030337
:106E080000F09780012BA3D190F82C3043F00103B8
:106E180080F82C309CE74B795E07A8D490F82C308A
:106E280043F0040380F82C304A7812F002061FD190
:106E3800D5078B7822D5B1F8035042461946FFF79B
:106E4800ABFE6DBAADB285420BDAB7F803506DBA36
:106E5800ADB200231A4684F8283084F82960628588
:106E68006EE742462046B978FFF796FE051EF0DA2F
:106E7800022305264FF410520025ECE72BB102211E
:106E88008D4A8C483FF091F8F2E7B1F8035041463B
:106E98006DBAADB240F049FA232DD6D94146204605
:106EA80040F043FA2425D4E74D7915F004057FF422
:106EB8005EAF90F82C3043F0040380F82C308B78C8
:106EC8003F2B0ED1CE78002ED2D10D790323042D7D
:106ED80028BF042540462A4601A901935CF04BFAD5
:106EE800B7E7022305264FF41052B4E74B79590748
:106EF8003FF53DAF3B791A090CD19A070AD5DB0754
:106F080015D494F82C3003F00303032B3FF424AF7B
:106F1800002305E094F82C209707C2F34003F0D52E
:106F280094F82C2063F3410284F82C2010E7012305
:106F3800F6E790F82C2063F30002F5E70A2A7FF4BD
:106F480051AF2A2B1AD8222B7FF64CAFA3F123027C
:106F5800072A3FF647AF01A151F822F0DB6F01087D
:106F6800ED6D01085D700108ED6D0108ED6D01081A
:106F7800C5700108ED6D01081D7101085A2B7FF4D9
:106F880031AF4D7A15F004057FF4F1AE90F82C304E
:106F980043F0040380F82C308B783F2B40F0DD80E1
:106FA800CE78002E40F0D9804FF4C063CDE9013689
:106FB800B1F8075040466DBAADB2082D28BF082574
:106FC80001A92A465CF0D7F93246334684F82820CE
:106FD80053E07B7A13F004037FF4C9AE01AEADF839
:106FE8000430B370082390F82C208DF8073042F055
:106FF800040280F82C2040F062F90028B5BF4FF059
:10700800FF3302220322236A8DF80C20A8BF1BBA83
:107018000293636A31461BBA8DF80D30C3F3072219
:10702800C3F307438DF80F3094F82C308DF80E20F9
:1070380043F0040384F82C30B7F8075040466DBA83
:10704800ADB20C2D28BF0C252A465CF094F900231C
:10705800A36275E67E7A16F004067FF488AE90F88F
:107068002C3043F004039D0780F82C3009D4022605
:107078004FF46853002584F8286084F829606385F4
:107088005EE640F01CF90028F1D1236A03B1013B08
:1070980094F82C10626A1BBA12BA41F0040184F801
:1070A8002C100825C8F80030C8F804200023E2E7AF
:1070B8000F1C0808C43F0708F21B08087B7A58070A
:1070C8003FF555AE94F82C30D7F8026043F004032E
:1070D8009907B7F8075084F82C307FF527AE20467B
:1070E80040F0EDF800287FF421AE6DBA36BAADB2A3
:1070F8002A463146206AFFF7B9FD20B1022305214F
:107108004FF4045216E6174B2361636AE6616B433A
:10711800A3611DE67B7A5A073FF529AE90F82C301B
:10712800D7F8026043F00803B7F8075080F82C300E
:107138009B077FF5FBAD40F0C2F800287FF4F6AD61
:107148006DBA36BAADB22A463146206AFFF78EFDCF
:107158000028D3D1044B6361D7E7022205264FF4F8
:10716800105333E795730508056C010810B50469D9
:107178000346204640F8143B0122002142F013FE4A
:1071880004F12C00024942F086FE002010BD00BF29
:107198002573010838B503461B6940685C681B699C
:1071A80025685A681AB19A680AB1DA683AB9134870
:1071B8000121134A3EF0F0FE6FF0150038BD103380
:1071C800D3E8EF1F41F00101C3E8E21F002AF7D11D
:1071D800216909B90020F1E72B7A002BFAD13FF099
:1071E800EDF928B10121074A04483EF0D5FEF1E740
:1071F80020693FF070FA2872ECE700BFAC3F07083F
:107208002A1C08086B1A080838B504694068006821
:1072180004F11005D5E8AF5FED071FD40BB15D6829
:107228003DB9104A104801213EF0B6FE6FF0150036
:1072380038BD90F820501DB1DD680DB90B4AF1E753
:1072480085791DB19D690DB9094AEBE7C4E90212B8
:1072580063600274120A42740020E9E76FF0770055
:10726800E6E700BF541C0808AC3F0708731C080871
:10727800921C08082DE9F347D0F804A0066988464F
:1072880015467768DAF8044006F11003D3E8AF3FF3
:107298009B073BD5236960685B68D3F800903FF093
:1072A800E7F800220023012829460CBF99F81B9013
:1072B80099F81490DAF80C00CDE9002342463FF023
:1072C8006FF8054650B90121124A13483EF064FE92
:1072D8006FF00B04204602B0BDE8F087014680F845
:1072E800189020463FF010FC044618B12846FDF7D8
:1072F80097F9EFE7FB69002BECD14FF0FF324FF025
:10730800FF3306F1140004F065FDE3E76FF00C04A9
:10731800E0E700BFB31C0808AC3F070870B550F899
:107328002C3C5C6865681C38D0E8AF3F9B0725D5C6
:107338002B6968685B681E683FF09AF8002201288C
:107348004FF00003A0680CBF96F8296096F82260F9
:107358003FF022F8044630B9094A0121BDE87040DF
:1073680008483EF019BE0146067628463FF0CCFB99
:1073780020B12046FDF754F9034AEEE770BD00BF7F
:10738800CE1C0808AC3F0708E81C080807B5084ADF
:1073980092E80300CDE9000106488268126822B12C
:1073A8006946904703B05DF804FB6FF05700F9E7B2
:1073B800E83F0708403A07081F2808B5034606D9DA
:1073C80009480121094A3EF0F0FD002008BD0120CE
:1073D800074A00FA03F3D16833EA0101F6D01269CB
:1073E800934318BF0020F1E7843E07081D1D0808D5
:1073F80000200246012100F01F021F2808B501FAEB
:1074080002F2034606D90648064A3EF0CEFD6FF062
:10741800150008BD044B0020DA601A61F9E700BFC7
:10742800843E07081D1D0808002002462DE9F0418A
:10743800054600264FF001080E4F6B78F4B2A342C0
:1074480001D8BDE8F0812B781C442046FFF7B4FF33
:1074580068B12046FFF7CEFF57F834303BB107EB51
:10746800C40204F01F04516808FA04F09847013672
:10747800E3E700BF44380020014B1954704700BFB0
:10748800480C0020034670B1B0FA80F2C2F11F0226
:10749800D2B206498856064AD2F880100B43C2F881
:1074A8008030FCF7B1BBFF22F3E700BF480C002097
:1074B80000200246034AD2F8803023EA0003C2F8CB
:1074C8008030704700200246032921D8DFE801F008
:1074D800020C10190F4B1A6822EA00021A605A6847
:1074E80022EA00025A6070470A4B1A680243F5E71D
:1074F800084B5A6802435A601A6822EA00021A6066
:107508007047044B1A6802431A605A68104358605F
:10751800704700BF0020024630B5B0B1B0FA80F322
:10752800C3F11F03DBB20B4850F833408C4204D13F
:1075380000EBC3056D68954205D044B940F8331097
:1075480000EBC3004260002030BDFF23EBE76FF083
:107558000F00F9E74438002060B1B0FA80F3C3F1B6
:107568001F03DBB20021044A42F8331002EBC302C6
:1075780051607047FF23F5E744380020C300074AED
:10758800C0F38100183052F8202003F018000F23B0
:107598008340134023FA00F0704700BF00200246E2
:1075A800F8B504690D4600AFA034D4E8AF3FC3F383
:1075B8008003994218D1164A164B6E4688B00029A6
:1075C80018BF13466A461449CDE905134FF40073F2
:1075D800ADF81C30114B42F8103F00234FF4E45132
:1075E8000F48FBF7E1FBB5464DB1D4E8EF3F43F058
:1075F8000403C4E8E23F002AF7D1BD46F8BDD4E849
:10760800EF3F23F00403C4E8E23F002AF5D0F6E791
:107618005D1D0808651D08086C1D080803000001A9
:107628005C3F07082DE9F0470546894690461F4606
:10763800D0F808A040F09FF90446D0B1067FF307C0
:107648000AD590F8203018480121184A3EF0ADFCC0
:107658006FF07700BDE8F0873B464246494640F068
:1076680048F948B994F820300121114A0E483EF0F3
:107678009CFC6FF01200EDE79DF8203026F006061E
:1076880084F82180678484F824302677DAF8183063
:10769800214628469847B0FA80F3227F5B0963F3B6
:1076A80000022277D6E700BF5C3F07087E1D080866
:1076B800981D080870B50546866840F05CF90446D0
:1076C800D8B1037FDB0709D490F820300C4801219A
:1076D8000C4A3EF06AFC6FF0770070BD0146F36912
:1076E8002846984738B1237F03F00103227F63F3CC
:1076F80000022277F1E70346F8E76FF01200ECE7A3
:107708005C3F0708BA1D08082DE9F3411746D0F871
:1077180008800546D8F83C300E46984700220023DA
:1077280039460B48FCF7FEFE044670B901213B467A
:10773800084A094800963EF042FC2846D8F84030EE
:107748009847204602B0BDE8F0810676F5E700BF0D
:1077580058120020D51D08085C3F070813B50369B7
:107768000C46D3F8A40091F8201041F06DFD94F870
:10777800203048B101210090084A09483EF01FFC1A
:107788006FF0040002B010BD5B0601D10020F9E7DC
:10779800237F43F002032377F8E700BF031E08089E
:1077A800643F0708F8B591F9203091F82060002B64
:1077B80001DB0020F8BD7306FBD047684C8CB7F896
:1077C8004830C4F30A04A34294BF03330334006966
:1077D8008CBFA3089B08D0F8A440402B98BF5B003F
:1077E800D4F8E8049D008AB9A84224BF401BC4F815
:1077F800E80491F820100022204601F07F0141F0B2
:10780800B7FD0028D5D06FF00400D3E7BA68121A84
:10781800AA4207D20A4832460A4940F00EFC6FF0E5
:107828000B00C7E720469AB206F07F0141F0A0FDA1
:107838000028E8D1D4F8E8342B44C4F8E834B8E791
:10784800643F0708311E0808F7B54668036974687D
:10785800D3F8A45064009834A1B20746A40028467F
:1078680041F0A5FDC5F8E84401241022002128466E
:1078780041F07EFDD5F8E8344033C5F8E834736844
:107888009C420ED3284641F0F1FB054680B11749CA
:107898000246174840F0D1FB6FF00404204603B0BD
:1078A800F0BDE1B20022284641F062FD0134E6E76E
:1078B80002460146009040233846FFF7B3FE0446CF
:1078C80028B12A460B490A4840F0B7FBE6E70246CA
:1078D8000090402380213846FFF7A4FE044608B1F3
:1078E8008022EFE73069FCF78FF9D7E7541E0808C4
:1078F800643F0708691E080838B504460369D3F8C9
:10790800A45043681869FCF78DF900212046FFF759
:10791800D1FE38B10C490D4840F094FB6FF00404D7
:10792800204638BD20468021FFF7C4FE04460028C3
:10793800F0D1284641F0B7FB02460028F0D00449B0
:10794800024840F07AFBE9E7831E0808643F07080D
:10795800A61E080838B503690546D3F8A440204692
:1079680041F000FD024630B10D490E4840F065FB7C
:107978006FF0040038BD0021142042F0CCFB2046F3
:1079880041F0F3FC04460028F2D101462846FFF7EF
:1079980007FE22460221284640F027F82046E9E75C
:1079A800BA1E0808643F070870B5036945680446AD
:1079B800D3F8A40041F045FB024618B11A491B4808
:1079C80040F03BFB6668F069D8B1436898470446C5
:1079D800B8B117490246154840F02FFB002C19DBB7
:1079E80000F0F8FB024618B11249104840F025FB98
:1079F8002869FCF72BF910B12869FCF713F9002066
:107A080070BD0D48716983685B6843B90B490748C5
:107A180040F018FB0A49054840F014FBE0E7984796
:107A28000028DDD0F2E700BFDA1E0808643F070827
:107A3800F01E0808431F0808403A07080E1F0808E8
:107A48002A1F08082DE9F04103690646D3F8A45017
:107A5800476800F08BFB044638B12E4902462E4891
:107A680040F0EBFA2046BDE8F08176682B4896F89E
:107A78004A30D0F80880012B13D97169D8F818302A
:107A8800083153B92649244840F0DCFA25492248F0
:107A980040F0D8FA6FF00404E4E72246984700283B
:107AA800F0D1D8F8003071690BB91F49EBE71B48D2
:107AB800984704460028F8D1F06950B10368984700
:107AC800064630B119490246134840F0B6FA002E6E
:107AD800DCDB40F2E442002128465BF072FC3B68A4
:107AE80028462B607B682B7140232B723B6B6B7293
:107AF8007B6BEB7102F06EFE024620B10C49064822
:107B080040F09BFAC6E7284641F0CDFA0028A9D0F4
:107B1800C0E700BF611F0808643F0708403A07082C
:107B28007E1F0808D81F0808A01F0808BB1F0808E0
:107B3800F01F08082DE9F04F064600274FF0280AE5
:107B48004FF0400BD0F810904568D9F8A4808BB05E
:107B58006B68BB4256D800274FF0280A4FF0400BFD
:107B68006B68BB4200F2858099F8803023F06A0385
:107B780043F06A0389F880306B6B2BB999F8803031
:107B880043F0010389F88030C8F8E46408F5C0615F
:107B980008F5BA600823042241F0F0FFD5E9101275
:107BA80008F59E684FF0000A4FF0000B6FF00703CE
:107BB80001200027CDE90330CDE906AB4046CDE9E9
:107BC8000177514B009604F07FFB3168404642F044
:107BD800A0F9EB6898473946A86909AA40F07CFEE5
:107BE800041E07DB099B3A461979186840F086FE9F
:107BF800041E6BDAA31C69D044492246444840F06D
:107C08001CFA30E00AFB07F1EB6B17F0800F0B440E
:107C18009A7E07F07F000CBF42F0400242F020023B
:107C28009A769A7E83F8207050B942F001029A76CB
:107C3800EB6B5FB1EB6BB5F848200B441A8307E098
:107C480022F00E0242F00E029A76F3E7A3F818B07B
:107C5800EB6B304619443FF0A0FE044638B12D497D
:107C68002B4840F0EFF920460BB0BDE8F08F013704
:107C78006EE70AFB07F1AB6B67F07F020B4483F8F2
:107C880020209A7E7C0642F020029A760BD1D2B24E
:107C980042F001029A76AB6B67B1AB6BB5F848203E
:107CA8000B441A8308E09A7E22F00E0242F00E027C
:107CB8009A76F2E7A3F818B0AB6B304619443FF058
:107CC8006CFE04460028CAD1013749E7A86A08B9FA
:107CD8000024C8E7283541F065FE30B90E490C4844
:107CE80040F0B0F96FF01504BDE74FF4B011284625
:107CF80040F062F90028EBD00849054840F0A2F9A5
:107D08006FF00404AFE700BFF17D010820200808E8
:107D1800643F0708042008083E2008085A2008087D
:107D280073B5D0F8A46008460C4615463FF02CFE03
:107D380018BB94F82030298A802BEA680B4602D1B8
:107D4800402928BF4023D018C91AE8602982304644
:107D580094F8201041F05EFA58B194F820300121CF
:107D68000090074A07483EF02AF96FF0040002B075
:107D780070BD012120463FF00BFE0020F7E700BF51
:107D880077200808643F070813B591F820300C469F
:107D9800D0F8A400DBB9537EDB071ED4538AC0F8A1
:107DA800EC34538A402B28BF4023D26894F8201023
:107DB80041F00BFA68B194F8203001210090084A8C
:107DC80008483EF0FCF86FF0040002B010BD538A7A
:107DD800EBE7012120463FF0DBFD0020F5E700BF7F
:107DE800A8200808643F07082DE9F34707460369F8
:107DF800D3F8A4604FF0FF334FF0FF3201A906F526
:107E0800BA6003F04FFE9DF80430012B5FD0022BBF
:107E180007D0002BEED1384606F29C413FF018FE01
:107E2800E8E79DF80590D6F8E48449F0800A5146C1
:107E380040463FF0A0FD054600213FF0A9FD284639
:107E48003FF0C6FD04460028D4D019F07F0F18D1A2
:107E5800038AB3B1402B28BF4023C2688021304633
:107E68001D4641F0D7F9024620B13F493F4840F04E
:107E7800E4F8BFE7238A5B1B2382E3682B44E360B3
:107E8800B8E720463FF0A8FD814660B120463FF0A4
:107E9800A7FDE26800235146304641F0BBF902468F
:107EA8000028A7D0E1E728463FF08EFD4A46014664
:107EB80040463FF0A6FD28463FF08AFD02460028CE
:107EC80098D02946D8F81000FFF72AFF92E79DF8C6
:107ED8000590D6F8E48449464046BDF806A03FF030
:107EE8004AFD05463FF074FD044648B920494A4614
:107EF8001E4840F0A2F8214628463FF049FD79E7A0
:107F080051460C303EF078FAB9F1000F17D1BAF1AA
:107F1800400F14D1228AD6F8EC349A420FD2E06886
:107F2800638A61699B1A411A5B1A402B024428BF75
:107F38004023304695F8201041F047F95AE7284683
:107F48003FF042FD0022014640463FF05AFD2846D8
:107F58003FF03EFD024628B12946D8F81000FFF749
:107F680013FF47E70146C7E7D8200808643F07081A
:107F780001210808F7B591F82150036905F00305B8
:107F8800D3F8A4706B1E022B4FF001020C4688BF79
:107F98000025FFF707FC064698B9628C2B46384641
:107FA80094F82010C2F30A0241F0B3F848B194F8EB
:107FB800203001210090044A04483EF000F86FF098
:107FC8000406304603B0F0BD1A210808643F0708CC
:107FD80013B503690C46D3F8A40041F087F840B103
:107FE8000121009023460448044A3DF0E8FF6FF061
:107FF800040002B010BD00BF643F07084321080811
:1080080037B5036905460C46D3F8A40091F820104B
:1080180041F0B3F8024630B92146284603B0BDE81E
:108028003040FFF7BFBB94F8203001210090044A8C
:1080380004483DF0C4FF6FF0040003B030BD00BF3A
:1080480071210808643F070873B5036905460C46A3
:10805800D3F8A40091F8201041F02DF958B194F804
:10806800203001210090164A16483DF0A8FF6FF015
:10807800040002B070BD237F60F3410323772046DC
:108088003FF0A6FC064608B90020F2E720463FF07C
:108098007BFC94F92030002B07DA0028F4D1324613
:1080A80021462869FFF73CFEEEE70028ECD132466E
:1080B8002146286902B0BDE87040FFF765BE00BFE1
:1080C8009B210808643F070837B50D46044641F070
:1080D80099F801238DF805508DF80430ADF80600A5
:1080E8000022002301A904F5BA6041F05AFD18B135
:1080F800024903483FF0A6FF03B030BDCB21080872
:10810800643F0708002307B5ADF8063002238DF851
:1081180005108DF804300022002301A900F5BA608B
:1081280041F03FFD18B1034903483FF08BFF03B00E
:108138005DF804FBCB210808643F0708002307B556
:1081480001930022002301A900F5BA6041F029FD3E
:10815800002803DA034904483FF074FF03B05DF8D0
:1081680004FB00BFCB210808643F070838B54FF06F
:10817800FF324FF0FF33124803F02CFE0446C0B91B
:10818800104D2B685A1C2A6083B90F4BDA6802F429
:108198004032B2F5003F0ED26FF0040401210B4AC1
:1081A8000B483DF0F9FE2B68013B2B60044803F0B7
:1081B800D5FD204638BD1A6942F080521A61F5E7AC
:1081C80084110020A43A002000080246FE21080875
:1081D800443F070810B54FF0FF324FF0FF330A480D
:1081E80003F0F8FD044660B9084A1368013B1360C0
:1081F80023B9074A136923F080531361024803F037
:10820800ADFD204610BD00BF84110020A43A002017
:1082180000080246074B1A6822F004021A605A68DE
:10822800D207FCD40222DA601A6842F001021A600E
:10823800704700BF00040340044B1A6822F0010293
:108248001A601A68D207FCD4704700BF00040340C4
:108258000D4A0E49936813F4000308D0936813F489
:1082680000030CD1D2F8F42051F82300704790682D
:10827800000207D4D2F8F430C3F30333F4E7936869
:108288001B0FF1E79268EFE7000C0246E848070881
:1082980038B50B880D46C3F30B03122B144636D89A
:1082A80013B96FF0850031E0013B112BF9D801A219
:1082B80052F823F0378301086B830108058301080E
:1082C800AB820108AB820108538301084D83010882
:1082D800AB820108AB8201083183010831830108B0
:1082E8003183010831830108318301083183010892
:1082F8005783010837830108378301084FF4FA4090
:1083080020602B68B3F5805F2ED2002038BD882B03
:108318000AD003F67473C3F30B031C2BC1D8164A97
:1083280022FA03F3DB07BCD5144B1868E8E7FFF71C
:108338008FFF4FF42023A0FB0303400B40EAC34008
:108348004008DDE7FFF784FFDAE70D48D8E7FFF7D5
:108358007FFF4FF42023A0FB0303400B40EAC340F8
:10836800CEE74FF40040CBE7C3F313330133B0FB40
:10837800F3F02060C9E700BF11011111C806002001
:10838800006CDC0237B5A84CA84BE26902F00C027D
:108398001341D80700F14381FFF75AFF236AA44A23
:1083A80003F00F03D35C20FA03F5A24BDA6842F41A
:1083B8004032DA60DA681104FCD59F48854201D260
:1083C80003F072F8984CD4F8943043F00403C4F8DE
:1083D8009430D4F8943003F004030093009BFAF728
:1083E800D9F9D4F8F03023F0180343F01003C4F897
:1083F800F030D4F8F03043F00103C4F8F030D4F88A
:10840800F0309A07FBD5D4F8F03043F08003C4F875
:10841800F030854CD4F8F0301B05FBD5FAF7D8F9C5
:10842800A36843F40003A360A36823F0704343F0F8
:108438008043A360236843F040032360236843F02C
:1084480008032360236843F001032360764B1A680E
:108458005407FCD5D3F8942050070BD4D3F89420B4
:1084680042F00402C3F89420D3F8943003F00403D4
:108478000193019B6C4CFAF78DF9D4F8F03043F076
:108488008063C4F8F030D4F8F0301901FBD5FAF75E
:108498009FF9236843F480532360634B1A6892045E
:1084A800FCD5DA6902F00C020C2A1AD11A685405B4
:1084B80007D41A6842F480721A605B4A1368580538
:1084C800FCD5594BDA6922F0030242F00102DA6165
:1084D800DA6902F00C02042AFAD11A6A22F00F02B1
:1084E8001A62514B1A6822F080721A609A6A22F056
:1084F800030242F001029A624E4AD16821F48021B7
:10850800D160D46814F48044FBD19A6A464922F4B5
:1085180070429A62494B4A4A1B699342B6BF494A1C
:10852800102393FBF2F38A6A03EBD37322F47042AD
:108538005B1042EA03338B623E4BDA6842F48022D6
:10854800DA60DA685104FCD5FFF782FE3E4AA0F5EE
:108558007413A3F51063934205D93C4B394A03447D
:1085680093425ED20C24304B9A6A22F470629A626B
:108578009A6A22F00C0222439A625A6B6FF308023D
:1085880042F04F025A639A6A22F010029A625A6BBA
:1085980022F4FE0242F480325A639A6A42F40032AC
:1085A8009A625A6B22F0FE4242F080725A639A6ACB
:1085B80042F480229A621A6842F080721A601A683D
:1085C8009201FCD5DA6A22F00302DA621A6B22F011
:1085D80003021A631A6A22F00F021A621A6A22F058
:1085E80070021A621A6A22F4E0621A625A6A22F067
:1085F80070025A62DA6942F00302DA610A4AD36900
:1086080003F00C030C2BFAD10B4CA54202D32046E5
:1086180002F04AFF00200E4B1C6003B030BD002062
:10862800BCE66FF02100F8E7000C0246FEEFFFFF02
:108638005A6B08080008024600688909E8480708D4
:108648000020A10700127A0000093D00FFED85FF18
:10865800C8060020192808D8054BC34013F0010F9D
:108668000CBF6FF08500002070476FF085007047E1
:10867800CEFC060208B5074841F094F938B106481F
:10868800FBF78AFE0448FAF735F8002008BD6FF0BA
:108698001200FBE71C3C0708A58601080A2838B524
:1086A8000446074D04D1AB680D2128465B689847FE
:1086B800AB6803485B68E1B29847204638BD00BF05
:1086C8001C3C0708064A11680B6823F004030B607A
:1086D8005068044B196883685B6803B11847704792
:1086E80078050020E405002010B5094BD3E90040C7
:1086F800084B196883681B6803B19847236843F0DF
:1087080004032360236843F00803236010BD00BFFF
:1087180078050020E405002008B5EFF31181102347
:1087280083F31288BFF36F8F0120094B93F8482019
:1087380083F8480081F31188BFF36F8F32B9FFF7D0
:10874800D3FFBDE808405E20FBF75EBA08BD00BF56
:108758007805002038B543680569394868601968A4
:1087680083681B6853B19847044650B101212346DA
:10877800344A35483DF019FC204638BD6FF057049F
:10878800F4E7012205F10800114641F00CFB012233
:10879800214605F1200041F006FB05F138002B4980
:1087A80041F079FB072385F86130042385F86230AE
:1087B8000F2385F84C300C23224685F84D3021468E
:1087C8005E2085F85E4085F85F4085F8604085F852
:1087D800494085F84A4085F84B403DF07CFD1C4BEC
:1087E8001C491B681A681D6922F07C4222F07F022E
:1087F8008A42D86806D14AF2B0218D4202D1164980
:10880800884211D0196821EA0201144A0A431A6001
:108818004AF2B0221A61104ADA601A6822F08042DD
:108828001A601A685200FCD41A6842F004021A60EE
:108838001A6842F008021A60FFF76EFF9CE700BF53
:10884800403A0708492208087C3E0708A78205081D
:1088580078050020000DF000BB7C0100000DF04001
:10886800F8B58378C678EFF3118E102484F3128854
:10887800BFF36F8F057890F801C05B1B33409A42B5
:1088880088BF9AB2AF1837402C4607708EF311880C
:10889800BFF36F8F8F188F421BD165450CD1EFF353
:1088A8001181102484F31288BFF36F8F0478447009
:1088B80081F31188BFF36F8F01799B1A994294B2A3
:1088C80005D341F020FB68B1084803F007FC2046B7
:1088D800F8BD00EB040E9EF805E0013401F801EB49
:1088E8003440D8E7FFF718FFF1E700BFB0050020D4
:1088F80070B50D4614460CB9204670BD4FF0FF32D6
:108908004FF0FF330B4803F065FA224629460A4820
:10891800FFF7A6FF064630B94FF0FF324FF0FF339E
:10892800064803F057FA0348A41B03F017FAA4B249
:108938003544E0E780050020D60500209805002092
:1089480010B51D4B01461B68EFF31184102282F30A
:108958001288BFF36F8F5A68500605D45A68D20739
:108968001DD46FF00A0015E01A6842F080421A60C0
:108978001A6822F080421A600A221868400005D45A
:108988005868400602D458684007E7D5013AF4D140
:108998006FF0040084F31188BFF36F8F10BD5A681D
:1089A8009207F5D4586810F04000F1D19B680B602D
:1089B800002BEFD1D5E700BF780500202DE9F7435C
:1089C800D8078846144605D43148FFF749FF03B055
:1089D800BDE8F083002A37D0EFF31185102383F325
:1089E8001288BFF36F8F5E20FBF730F906465E20D2
:1089F800FBF718F985F31188BFF36F8F0EB9FFF7EE
:108A080073FEDFF89490D9F800305A68510713D4F0
:108A18005B685A0610D44FF0804325461D4FC7F8AF
:108A28008831D9F800305B68DB070FD4BFF34F8F6C
:108A380020BF40BF20BFF4E701A8FFF781FF002453
:108A480016B35E20FBF7E0F82046C0E701A8FFF761
:108A580077FF4FF080420346C7F8882188B9291F5D
:108A6800019A89B2002DEBD0A94203D1002BD8D0AE
:108A78000192D6E7013DADB208F805200123120A9C
:108A8800F0E7002DCDD1DBE7FFF71CFEDCE700BFE8
:108A9800C105002000E100E0780500202DE9F7433A
:108AA80001A8FFF74DFF002843D10427804601465F
:108AB800264C019A94F84B3094F84CC094F84AE04C
:108AC800A3EB0E053CEA05055FFA82F91ED194F87E
:108AD800601094F85F6094F861508E1B35EA0606C2
:108AE8002AD108B184F84B30B8F1000F00D00192B8
:108AF8005E20FBF797F8FFF7E5FD002384F8483080
:108B0800134803B0BDE8F04303F028B9E01880F833
:108B18004E90012001330CEA0303013F4FF0010896
:108B28004FEA1222CCD108B184F84B3001920029C7
:108B3800E6D103B0BDE8F083661801310D4086F830
:108B48006390012184F86050E7E700BF78050020B2
:108B580098050020004870478C460708044BB3F876
:108B6800A0379B020B60002318464B60704700BF7C
:108B78000000FA0B07B50346054A00910548012194
:108B88003DF01DFA6FF0150003B05DF804FB00BF5F
:108B9800AF220808943E070873B5064664220023EE
:108BA800684641F012FBDDE9004533691B681A6A23
:108BB80012F0FA0212D01A6A02F0FA021A626FF080
:108BC800040002B070BD22462B46684641F022FBE5
:108BD800DDE9003213430CBF0122002233691B6810
:108BE800186A10F48030ECD0002AECD00A23012156
:108BF800024A03483DF0D9F9E1E700BFD922080845
:108C0800943E070838B5036905461C6849B1FFF763
:108C1800C3FF58B12869043003F0A0F86FF00400CE
:108C280038BDA36A002B06DB0020F9E7A36A43F0EE
:108C38000043A362F8E7034BA36003F18833A36002
:108C4800F2E700BF2301674573B5012306460D46C9
:108C580014463FF0F3FB50B90A482B4601210A4A53
:108C680000943DF0ACF96FF0150002B070BD3CB156
:108C780022462946304602B0BDE870403FF0BBBBF3
:108C88002046F2E7943E0708ED220808F7B51C468F
:108C980017460123224605460E463FF0CFFB58B93A
:108CA800012100943346154A15483DF088F96FF0C4
:108CB8001504204603B0F0BD002CFAD028693FF017
:108CC8006CFB00212846FFF79DFF98B931462346E3
:108CD8003A46284600F0B8F8064601212846FFF72C
:108CE80091FF002E14BF344604462869043003F06F
:108CF80035F8DEE76FF00406EFE700BF1823080831
:108D0800943E07082DE9F84F494B17461B680D4656
:108D1800824603F001084FF0000BFFF78DFA013F80
:108D2800DFF82091434E2F44AF420CD3DAF81030CD
:108D38001C68A36A002B0EDA01213F4A3F483DF028
:108D48002BF96FF0040BB8F1000F01D0FFF762FAAE
:108D58005846BDE8F88F5046FFF71EFFB0F1000BEC
:108D6800F1DBDAF810301B681B6C9B0252D54FF60A
:108D7800FD70B9F8A010226C4B1E9BB2834202F41E
:108D8800801250D8B5EB412F2CD26B0B002A43D15F
:108D9800A26A22F40062A262A26A504642F002026B
:108DA800A262A26A22F47E72A262A26A42EAC303A3
:108DB800A362A36A43F48033A362A36AFFF7ECFEBD
:108DC800DAF8103083461B681B6C13F4001FA36A83
:108DD80014BF334023F002030028A362B3DB05F578
:108DE8000055A1E7B5F5801F0BD332B1A36A23F470
:108DF8000063A3626B0B803BCEE7A36A43F4006376
:108E0800F7E701212B460E4A0C483DF0CEF86FF0EB
:108E1800150B98E76B0BBFE7B5F5801FE6D2A26A82
:108E280042F40062B7E7B5F5801FAED3DDE700BFB7
:108E380000040340FDF7FFFF692308089C3E07086C
:108E4800762308080007FA0B2DE9F84F0024984606
:108E5800324B0D461F6806469146A346FFF7ECF9CC
:108E680007F0010705F10065D8450DD93369D3F836
:108E780000A0DAF82830002B0CDA0121284A29480A
:108E88003DF08AF86FF004040FB1FFF7C3F92046EC
:108E9800BDE8F88F3046FFF77FFE041EF4DB2BF0A9
:108EA80003024A44111F0B460C3253F8040F00BB4F
:108EB8009342FAD1DAF8283043F00103CAF828308F
:108EC800DAF828302B4651F8040F914243F8040B86
:108ED800F9D13046FFF760FEDAF82830041E23F097
:108EE8000103CAF8283005F11005CDDB0BF1100B92
:108EF800BAE7284600230468013408D005F178450C
:108F08000121094A07482B443DF04FF8BAE70133DD
:108F1800042B00F10400EED1CCE700BF00040340AD
:108F2800692308089C3E07088F23080830B5104CB1
:108F3800104D0C60236813B12B68136030BD0369B2
:108F48001B68196C1B6C9B020FD54FF6FD700A4B02
:108F5800B3F8A030591E89B281428CBF4FF4807398
:108F6800DB0823604FF40053636001232B60E4E7C0
:108F7800AC3A0020A83A00200007FA0B2DE9F84384
:108F8800D0F8049090460746D9F808000D461E46CA
:108F98003EF07FFCB8F5001F044616D12846D9F8E4
:108FA8000840FEF7EBFA84420CD129463EF071FCEA
:108FB8000446FEF77FFA2046FEF7CEFA0021204647
:108FC800FEF782FA0020BDE8F883B8F5800F20D0BC
:108FD800B6F1806F19D0B6F1C06F18D0B6F1007F26
:108FE8001AD102263A4620460E49FEF795FAB0B93C
:108FF8002846D9F808103EF051FC20463146FEF7C5
:1090080063FA2046FEF73EFADCE70126EAE7032684
:10901800E8E76FF08500D6E76FF01500D3E76FF04B
:109028000F00D0E7AD8505080C291FB528BF0C2116
:109038000C460A4BD3F8082712BA0192D3F8042732
:1090480012BA0292D3F800370A461BBA01A9039351
:109058005AF091F9204604B010BD00BF0000FA0B89
:10906800174AD2F8F430D2F8F410C3F30073490168
:10907800D2F8F4104FEA4303D2F8F42048BF43F083
:109088000103890048BF43F0100352000C4A48BF4F
:1090980043F01003D2F8F410D2F8F420090148BFC5
:1090A80043F00403002A074AB8BF43F08003926BD9
:1090B800520748BF43F0800303600020704700BF99
:1090C800000C02460008024680B500AF8AB06A4626
:1090D800094B0791CDE905304FF40073ADF8203006
:1090E800064B42F8103F00234FF411510448F9F79A
:1090F8005BFEBD4680BD00BFBD230808040000011B
:10910800CC3E07082DE9F74398460B7A164643F0FC
:109118000403046907460B720D460B460122B2424E
:109128001AD904F118094FF0FF324FF0FF334846BF
:1091380002F050FE38463FF096FA041E2DDA01215F
:1091480023461A4A1A483CF030FF484602F006FE09
:10915800204603B0BDE8F0830AD2197A187D81EA67
:10916800000C1CF0010F01D040071CD589071AD448
:1091780001320C33D2B2D2E7012E0CBF002305F125
:109188001403CDE90038384695E80E003FF00EFB91
:10919800041E04DB013E0C35F6B2002EECD1384635
:1091A8003FF063FAD1E76FF01504D1E7D12308083F
:1091B800CC3E070808B50121034A04483CF0ECFE00
:1091C8006FF0040008BD00BFED230808CC3E070877
:1091D8000023F7B542680446066923480F46D56858
:1091E8005168926801938368012ADB6833D9083192
:1091F8004BB91E4A01211E483CF0CEFE6FF0040414
:10920800204603B0F0BD01AA98470028F1DB376378
:1092180006F118074FF0FF324FF0FF33384602F0DF
:10922800D9FD2B68204623F001032B6096F86210C5
:109238003FF0DCF92046019900F0BEF8041E06DB79
:1092480096F861301BB12B6843F001032B60384658
:1092580002F084FDD4E70BB9064ACBE701AA984788
:109268000028D4DAF8E700BF403A07080B240808BA
:10927800CC3E070839240808F8B50446466805694D
:1092880000274FF0FF320021284640F08CFD204691
:109298003368984785F8607085F86270012205F197
:1092A8001800114640F07FFD204600F051F8B368E1
:1092B800012B25D831691F4B994230D014D81E4B49
:1092C80099422ED01D4BCB1A59425941890020464C
:1092D80041F01001FFF77CFF041E26DA0121184A2D
:1092E80018483CF059FE13E0174B99421BD003F580
:1092F800C31303F5206399420CBF0A210021E6E756
:1093080012487168836808319B691BB96FF00404BF
:109318002046F8BD3A4698470028CBDAF6E70621FA
:10932800D5E70221D3E70821D1E70123002485F8F6
:109338006030EDE740420F00A0860100801A060069
:1093480067240808CC3E070840E13300403A070884
:1093580037B545680021286A01AA3FF0BDFA041E06
:1093680007DB019B0022197918683FF0C7FA041E31
:1093780008DA012123460C4A0C483CF016FE204628
:1093880003B030BD0A48696883681B683BB901218E
:10939800084A06483CF000FE6FF00404EFE79847DF
:1093A80004460028EBD0F2E78B240808BC3E0708E7
:1093B800403A0708A92408082DE9F04F4FF00C0E91
:1093C80044680369002085B00393A36AE568DFF861
:1093D8002881DFF82891DFF828A1DFF828B1029367
:1093E800029B8342039B1B6B01930DD1C3F3420283
:1093F800012A39D0022A66D03A4A3B4801213CF07A
:10940800CBFD6FF015001DE00EFB00F7D4F824C06B
:10941800364A0CEB0706736893421DD015D853459E
:109428001CD0A3EB0B02534253419B00019A5340BB
:1094380013F00E0F16D15CF807308B4212D1B368C7
:1094480000202B6105B0BDE8F08F434508D04B459F
:109458000CBF0A230023E9E70623E7E70223E5E731
:109468000823E3E70130BBE741F25C2E4FF47A6C46
:1094780040F2E2474FF4FA7602201D4B421EB1FB40
:10948800F2F2B3FBF2F2BCFBF2F4013CFF2C23D85E
:10949800BEFBF2F808F1FF38B8F1FF0F1CD8B6FB95
:1094A800F2F9B9F10F0F17D8B7FBF2F2013A0F2A08
:1094B80012D8023848EA094343EA007343EA0253E0
:1094C80043EA0423BCE740F2145E4FF4167C4FF4E1
:1094D800FA7740F27716CFE701301128CED1054A46
:1094E8008BE700BFF3240808C43E070840420F007A
:1094F80000CA9A3B6E25080840E13300404B4C00F7
:10950800A0860100801A060043681B6803F1080260
:1095180052E8002F42F0010203F1080040E8002160
:109528000029F3D1174A93421ED002F18052934288
:109538001AD0154A934217D002F18052934213D0A1
:10954800124A934210D002F1805293420CD0104A32
:10955800934209D002F18052934205D00D4A9342BA
:1095680002D0B3F1502F03D15A6842F040025A603A
:1095780053E8002F42F4807243E800210029F7D114
:10958800704700BF003801400044004000480040D8
:10959800004C00400050004043681B6803F108027B
:1095A80052E8002F22F0010203F1080040E80021F0
:1095B8000029F3D1174A93421ED002F180529342F8
:1095C8001AD0154A934217D002F18052934213D011
:1095D800124A934210D002F1805293420CD0104AA2
:1095E800934209D002F18052934205D00D4A93422A
:1095F80002D0B3F1502F03D15A6822F040025A60CA
:1096080053E8002F22F4807243E800210029F7D1A3
:10961800704700BF00380140004400400048004047
:10962800004C0040005000400129034608461AD06B
:1096380002290BD0C9B91B680D4A934217D002F111
:1096480080529B1A18BF0123180370471868084BEB
:1096580098420AD003F1805398420CBF4FF400504F
:109668004FF440507047002070474FF40050704747
:109678000024004638B51D46094B6C0833F8122003
:109688000023F7F7E9FB090241EA106100022018FC
:109698002A464FF0000341F10001F7F7DDFB38BD22
:1096A800800308082DE9F04782B0436880460C46DD
:1096B8001D6800AF002945D0586819698368DB68C0
:1096C8006BB13A1D9847061E0CDA0121344A354819
:1096D8003CF062FC30460837BD46BDE8F0876FF0C5
:1096E8005706F2E7304B9D4203D003F180539D4269
:1096F8002BD10026D7F80490DFF8BCA023464846B3
:109708000021B2B2FFF7B6FFA0F5407050452BD943
:109718000136102EF2D16D468AB0D8F800306A466C
:1097280022490794CDE905134FF40073ADF82030B2
:109738001F4B42F8103F00234FF411511948F9F715
:1097480033FBAD466FF01506C4E72B6823F40043DE
:109758002B607B6803EB5403B3FBF4F30F2BDAD9CC
:109768009BB2EB600026B5E7EB6A484623F00F038F
:109778003343EB620F4B33F8162000231946F7F7F3
:109788006BFB002306464FF4807C1946600822468E
:10979800E6FB0C01F7F760FBC0F31300E860E1E7B4
:1097A80039240808543F070800240046B225080851
:1097B8000400000180030808FFFC0F002DE9F843AE
:1097C80007460E7940683B69012E0D460468D3F8B8
:1097D800008014D0B31ED3F1000949EB03094FEA06
:1097E80089296979FFF720FFAA790346022A09D057
:1097F800042A01D0002E6AD04FF4805005E04FF4BF
:10980800C069EEE7002E5FD00020A6F1030CBCF182
:10981800010F04D86FF085031846BDE8F8830EB130
:10982800042AF7D0B3F5805F53D0B3F5405F52D028
:10983800002B0CBF012303239942EBD149463FF08B
:10984800B1F88242E6D1EB7953B3012B45D1244BD1
:109858009C4225D003F180539C4221D0214B9C424D
:109868001ED003F180539C421AD01F4B9C4217D044
:1098780003F180539C4213D01C4B9C4210D003F13F
:1098880080539C420CD01A4B9C4209D0B4F1502F03
:1098980006D0184B9C4203D003F180539C42B9D1A7
:1098A8002368294623F00103236038463FF0FCF97A
:1098B80003460028AED1226842F00102226095E8F2
:1098C800030088E80300A7E74FF08050AAE7304676
:1098D800A8E70023B0E70223AEE7032BB7D099E748
:1098E800003801400044004000480040004C00405F
:1098F80000500040002400462DE9F04383B0D0F822
:1099080004908046D9F80400D9F81010836800AF95
:109918001B687BB19847054670B90021D9F8240027
:109928003A1D3EF0D9FF051E0EDA28460C37BD4613
:10993800BDE8F0836FF057050121644A64483CF0A4
:109948002BFB002DF1DBE8E77B680022197918680A
:109958003EF0D4FF051EE8DBD8F80460D8F81030D4
:1099680034681D68236823F001032360B06840F061
:1099780019F838B90121574A55483CF00DFB6FF0EA
:109988001205D2E7D6E902018368DB6803B198477C
:1099980054E8003F43F00C0344E80032002AF7D1B2
:1099A800294640463FF080F9054610B16FF015058D
:1099B800BBE7337E1BB1A36843F00803A360737E43
:1099C8001BB1636843F400436360B37E1BB16368F3
:1099D80043F480336360F37E1BB1636843F4003360
:1099E8006360337F002B5AD03B4B9C423CD003F141
:1099F80080539C4238D0394B9C4235D003F1805378
:109A08009C4231D0364B9C422ED003F180539C426D
:109A18002AD0344B9C4227D003F180539C4223D058
:109A2800314B9C4220D0B4F1502F1DD02F4B9C427B
:109A38001AD003F180539C4216D06C4688B06A460F
:109A4800D8F800302A49CDE905134FF40073ADF872
:109A58001C30284B42F8103F00234FF4E2511C48B9
:109A6800F9F7A2F9A546A1E7D8F804301A6893686F
:109A780043F4804393602368727F23F0787343EA4A
:109A8800425323602368B27F23F4F81343EA024366
:109A98002360F37F1BB1A36843F40043A36096F8E7
:109AA80020301BB1236843F000532360236843F040
:109AB80001032360E3699A02FCD5E3695B02FCD5E4
:109AC8004046D9F8283098472FE700BFC92508082D
:109AD800543F0708E92508080038014000440040C1
:109AE80000480040004C0040005000400024004660
:109AF800042608080300000170B50B68064698881C
:109B08003FF0AEF904280C46D1E91B15034610D0E6
:109B180002280AD1012A01D9012D0AD8328E92B21F
:109B280009B105B10A80022508E0032A12D9032DDC
:109B380012D9326B09B105B10A600425B5FBF3F5FA
:109B4800226F2AB1954213D9164917483FF0C4F934
:109B5800284670BD012A02D9226F012ADED896F85C
:109B68003020D2B201B10DB90125E9E70A70FBE74F
:109B7800521B22677AB9A26D04F15C010832A26512
:109B8800E26D04F15800013AE26504F170023FF019
:109B980043F9E066DCE7E26E002AD9D005FB032230
:109BA800E266D5E761260808243F07082DE9F8434F
:109BB80006460C4604274FF0020891F87C9023686B
:109BC80098883FF04DF904280346626E17D00228A2
:109BD8000FD1B9F1010F02D9A16E01290FD8002ABE
:109BE80039D0A16E01B1118889B2B8FBF3F531847F
:109BF8000CE0B9F1030F1FD9A16E03291FD9CAB10F
:109C0800A16E01B11168B7FBF3F53162A26E2AB1FA
:109C1800AA4224D21F4920483FF05EF9636F5B1BBC
:109C2800A9EB050515F0FF09636701D0002BC6D124
:109C3800BDE8F8831146E6E7B9F1010F02D9A16E34
:109C48000129CCD84AB1A16E01B11178C9B2012558
:109C580086F82010DAE71146C6E71146F6E7521BE8
:109C6800A2667AB9226D04F1540108322265626D48
:109C780004F15000013A626504F168023FF0CCF843
:109C88006066CBE7626E002AC8D005FB03226266D5
:109C9800C4E700BF61260808243F070808B502B9D1
:109CA80033B1044804493FF017F96FF0850008BD47
:109CB8001846FCE7243F07087F2608082DE9F047E7
:109CC800044600AF00693FF047F9012160683FF0A2
:109CD8002EF9002802DA10F1860F15D165680021E7
:109CE800284626693FF023F9041E0BDB3248A96891
:109CF80083681B685BB19847044658B12F493048C0
:109D08003FF0EAF804EAE470BD46BDE8F0876FF07A
:109D18005704F3E74FF00108B5680835D6E9023271
:109D280003EBC203A5F108029342EBD955F8080CDE
:109D38003FF038FE034615F8041C55F8080CBBB96B
:109D48006C468AB06A46006807914FF400711D4D51
:109D5800ADF820101C49CDE9055042F8101F4FF40A
:109D680011511748F9F720F8A5466FF01204C9E712
:109D780035F8023CD0F810E0DA0754BF43F4B013CA
:109D880083F4D013DEF800C023F4801208FA01F936
:109D9800DB074CBF4CEA09032CEA0903D0F808A0FA
:109DA800CEF80030DAF800309847002805F10805A9
:109DB800B4DA0446A6E700BF403A0708AD2608080B
:109DC800243F0708C8260808040000012DE9F04FC1
:109DD80087B080460E469B469146056900AF32B96A
:109DE8002BB9002630461C37BD46BDE8F08FB38836
:109DF8009A0400F123814FF0FF324FF0FF3305F151
:109E0800100001F0E7FF6E600023C5E9113385F803
:109E18004C30D8F81030D8F804A0FB601B68DAF88A
:109E280000409E42B28840F01581130508D5B9F16B
:109E3800000F00F00C814FF4C12120463EF0DDFFF9
:109E4800B0883FF00DF80346B9F1000F40F0758176
:109E5800C5F8509000226A6505F1540105F16802C1
:109E680005F15000FB603EF0D7FFFB686866BBF168
:109E7800000F40F06B81C5F858B00022EA6505F183
:109E88005C0105F1700205F158003EF0C5FF0021A4
:109E98000B46E866686D2964834240F060810023C0
:109EA8001A46D5F85CC0624540F0608199422CBFE3
:109EB80029662B66AB6E3BB92B6F2BB96B6F1BB941
:109EC800AB6F002B00F03F8223687B60E3683B6048
:109ED800D8F80430BB601B68FB60FA681B68D2685E
:109EE80003F4006302F4C022134340F0468149465C
:109EF80030463EF0CFFF5946814630463EF0CAFF15
:109F080081454E46B8BF0646002EC0F2B580BB68F4
:109F18001B6AB342C0F03B81FB68D8F810101B687D
:109F2800DB0702D5F8683EF08DFFFB68FA685B68CE
:109F38006FF30F0333435360C1E91D66D8F804304B
:109F48001B681A6842F001021A60DA68500200F1D0
:109F58002581D8F810603068002840F028817B6897
:109F680003F400693B6803F4C02349EA0309AB6EB4
:109F78002BB92B6F1BB96B6F0BB9AE6F3EB329466C
:109F880020463FF00BF8636913F4787300F01C81E6
:109F98006E468AB06A46934905919349CDE90613FE
:109FA8004FF40073ADF82030904B42F8103F002377
:109FB8004FF411518E48F8F7F7FE6369B5465A0613
:109FC80003D5A36943F04003A3616FF00406D8F8F2
:109FD8000430D8F810901C686369D90700F15F81D4
:109FE800E3685A0240F17281824920463EF043FFFD
:109FF800002800F057812368D80740F1538163682F
:10A008009BB26BB9D9F800309B88C3F34513192B61
:10A0180006D821FA03F3DB0702D520463EF012FFEB
:10A028002368E26803F4006302F4C0221343B3F523
:10A03800C02FDAD120463EF005FFD6E7AB69002BEA
:10A048007FF4D9AE6B689E427FF4D5AEDCE64FF460
:10A05800C021F2E6DAF81010C2F34513022918D02D
:10A06800032919D0012931D1043B1C2B8CBF0023B3
:10A078000123ABB96FF0850695F84C3013B1002E6B
:10A088003FF4AFAE00236B6005F1100001F066FEEF
:10A09800A8E6043B0C2BE9E7082B01D0102BE9D1EB
:10A0A800100448BFE368544842BF23F4601343F4E4
:10A0B8000023E3608368DAF80810DB685BB94F496E
:10A0C8004B483EF009FF6FF00406D5E74C49484875
:10A0D8003EF002FFCEE707F1140298470028EEDBB6
:10A0E80000217B69306823FA01F2824240F22D8117
:10A0F80001310929F7D16C468AB06A4607931B0AD1
:10A10800089305233F49CDE9051042F8103F002385
:10A118004FF421513648F8F747FEA5463BE04FF487
:10A12800C02143E11BB1E36823F0105366E1E36803
:10A1380023F0105343F0005360E1D9F800202A655A
:10A14800002A3FF487AED9F8042084E6DBF8002023
:10A15800AA65002A3FF491AEDBF804208EE62A6D4A
:10A1680002EBC30252680133114495E6A86D00EB77
:10A17800C20040680132034495E6B3F5C12F30466A
:10A188000CBF494659463EF085FE0646BCE61E49C8
:10A1980017483EF0A1FE6FF015066DE71A6842F405
:10A1A80000721A601A6891053FF5D3AEFAE7037D8D
:10A1B800002B3FF4D4AE012108303EF0A5FE3368F1
:10A1C80018693FF0C9FBCAE6B9F5C12F7FF4CFAED5
:10A1D800AB6EDBB100212268E36800295CD102F490
:10A1E8000069C0E66C270808486B080804000001ED
:10A1F800243F070800020202403A0708142708080B
:10A20800EC26080877270808402708082B6F002B3A
:10A21800E0D0DAF8006030463EF02DFE0146002816
:10A22800F9D130463EF00EFE2B689888C30712D449
:10A238000B46D5F85CC0634524D13EF011FE91FB76
:10A24800F0F300FB131323BBB1FBF0F173686FF35A
:10A258000F03194371604FF4C02130463EF0CDFD25
:10A26800336843F001033360F3685A02B2D53368A8
:10A2780043F40073336033689B05ABD473691807E4
:10A28800A8D4F8E7AA6D02EBC3025268013311445F
:10A29800D1E76FF015019EE76FF0150697E694F881
:10A2A800303099E6D8F810A0DAF8003073B11A7D8A
:10A2B80062B1998811F4805B08D118693FF04CFBB2
:10A2C800DAF80000594608303EF01EFE6369990529
:10A2D80042BFA36943F40073A361A36943F0100369
:10A2E800A361A36943F04003A361A36943F0080392
:10A2F800A36163686FF30F036360D9F800309B882C
:10A30800DA0402D420463EF09DFD99F84C3033B96A
:10A31800C9F8406009F1280001F020FDACE6D9F841
:10A32800443023B131464046D9F848209847D9F8F7
:10A3380000309B8813F400537FF49EAEC9F80430B4
:10A3480009F11000E8E71E4696E620463EF07AFD41
:10A358004B4AA36852F8212023F070431343A360AB
:10A368009AF82530DB0703D5E36843F40043E3603C
:10A37800B38813F0020FE36814BF43F0007323F0AF
:10A388000073E360B38813F0040FE36814BF43F06D
:10A39800807323F08073E360B18811F4006105D005
:10A3A800B9F1000F3FF4BBAE4FF4C12120463EF097
:10A3B80024FDB38813F0100FE36814BF43F40003BF
:10A3C80023F40003E360A36823F48003A360B38845
:10A3D800327D03F0010322B99AF8252091077FF511
:10A3E800A1AE33B9E368DA005EBF236843F4805353
:10A3F8002360E36823F0105343F08063E360B3887D
:10A40800204913F0010FE36814BF23F4800343F4D9
:10A418008003E360B288A368C2F34512043A51F896
:10A42800222023F01F031343A360E368DAF81C20FB
:10A4380023F00F031343E360E368DAF8182023F0EE
:10A44800F00343EA0213E360B288DAF81430C2F387
:10A4580045120732D20893FBF2F3012BB8BF012350
:10A46800FA68094982F87C30DBB2A268013B51F8EE
:10A47800233022F4F0721343A360FB681E60DFE40C
:10A48800BC47070874480708344807084FF0E0231A
:10A4980010B599691C699B6900B103600B4A0C48A7
:10A4A8001268002908BF1146002B08BF134614F490
:10A4B800803F01D1994205D20168114401604FF0F3
:10A4C800E021096900681044C01A10BD983B0020BB
:10A4D8008C3B002010220B4B002083F823204FF4E4
:10A4E800C862094B1A604FF47A52084B1A60084B3D
:10A4F80043F67F6218604FF0E0235A6107229861A3
:10A508001A61704700ED00E0943B0020983B002062
:10A518008C3B0020684620F007018D46F1B53EF0DF
:10A528007FFD04460020FFF7B1FF1348134A036874
:10A53800D2E900515B1941F10001C2E9003100275D
:10A548004FF47A520E4D0760D5E900619B1BB3FBAF
:10A55800F2F002FB00F39B1941F10001C5E900315B
:10A56800084B21461F6002F0A7FBF9F727FCBDE85E
:10A57800F1408546704700BF8C3B002088300020A2
:10A5880080300020903B00202DE9F341804601A84F
:10A59800FFF77CFF00272849284AD1E90034C3186F
:10A5A800274844F100041760D0E90020B3EB020CFF
:10A5B800C1E90034234E64EB0004234BBC423568E8
:10A5C80018681ADB4FF47A5E204B1B6813EB0803FC
:10A5D800A3FB0E3247EB07080EFB0822B3EB0C0374
:10A5E80062EB04029842974107DAB3F1807F72F177
:10A5F8000002A8BF6FF07F4318464FF0E023002207
:10A60800306001389C6958619A61114A536803F0B7
:10A61800807343F000735360019BD1E90020A3428B
:10A6280038BF5B191B1B9A1840F10000C1E90020D4
:10A6380002B0BDE8F08100BF883000208C3B0020CC
:10A6480080300020983B0020943B0020903B002065
:10A6580000ED00E010B5084B00201C68074B1B6894
:10A66800E41AFFF713FF4FF47A532044B0FBF3F0DA
:10A67800034B186010BD00BF8830002080300020D8
:10A68800903B002038B53EF0CBFC064B044600203A
:10A698001D68FFF7FBFE84F31188BFF36F8F284412
:10A6A80038BD00BF8830002030B53C4AD369916A74
:10A6B80013F00C0305D00C2B3FD101F00301012945
:10A6C8003BD19168090254BFD2F8F420926834490A
:10A6D80054BFC2F30332120F51F82200002B5AD094
:10A6E8002E49B7EE006A8C6A8B6A8D6AC3F303231E
:10A6F8008A6B013307EE903AC2F3CC03C5F300121C
:10A70800534306EE903A04F00304022CB8EEE77ABD
:10A71800FAEEE96A1FD0032C1DD04B6BC3F3080374
:10A7280007EE903AF8EEE77A77EEA67A06EE900A08
:10A7380077EE867AB8EE666A1AE0D26902F00C0201
:10A74800042A06D0082B27D000200C2B23D1002068
:10A75800C6E71448F9E74B6BC3F3080307EE903AD2
:10A76800F8EEE77A77EEA67A77EE867A9FED0E6AAC
:10A778000A4BC6EE076A5B6B67EEA67AC3F30663FD
:10A78800013307EE103AB8EEC77AC7EE876AFCEED7
:10A79800E67A17EE900A30BD0248FCE7000C024644
:10A7A800E84807080024F4000024744B08B5FFF7B4
:10A7B8007BFF054B054A1B6A03F00F03D35CD840A7
:10A7C800034B186008BD00BF000C02465A6B08080E
:10A7D800C8060020F7B5044610B390F8953405680C
:10A7E80003F0FF021BB980F894243EF028FC0323F1
:10A7F80084F89534324B20689D4204BF0023A3712E
:10A808003EF031FE237C251D8DF8003095E80E00C2
:10A8180020683EF0E4FD014630B1022384F8953407
:10A828000125284603B0F0BD20683EF022FE00282E
:10A83800F3D101270246267904F11403C1B28E42EE
:10A8480003F1240321D800210A4604F51573C8B280
:10A85800864203F1240326D8237C8DF8003095E83E
:10A868000E00206800F00AFC05460028D5D1012317
:10A87800607484F89534237B012B02D120463EF086
:10A888009AFD20683EF0FEFFCBE723F80A0C43E967
:10A89800072203F8237C03F8241C03F8202C43F830
:10A8A800142C0130CAE743E9072203F8232C03F8E4
:10A8B800240C03F8202C43F8142C0131C7E700BFFF
:10A8C800000004422DE9F04F066889B0044630467E
:10A8D8003FF014F80390002840F06F8120683EF0A4
:10A8E800DFFF002800F06981D6F808382068C3F334
:10A8F8000D23C4F8D4343EF0D3FF870748BF22683D
:10A9080006F5006542BF536903F0020353612068EE
:10A918003EF0C6FFC0062DD52268936923F01003C8
:10A928009361D6F8208008F4F013B3F5802F08F06F
:10A938000F0740F0458147F6F07318EA030F14D06B
:10A94800242303FB0747C8F30A194A463046D7F8B9
:10A9580060123EF036FFD7F860324B44C7F86032D9
:10A96800D7F868324B44C7F868322268936943F0D5
:10A978001003936120683EF093FF010300F13381D7
:10A9880020683EF08DFF42030CD520683EF094FF0E
:10A9980027464FF0000A049006F5106B049B002B25
:10A9A80040F0EB8120683EF07BFF002813DA6B68EB
:10A9B80023F001036B6094F8CC34012B40F08582BE
:10A9C8000021204684F8CC143EF008FD2268536923
:10A9D80003F00043536120683EF062FF03050AD587
:10A9E800AB68DF0702D520463DF0A1FB226853691A
:10A9F80003F40063536120683EF052FF000115D54F
:10AA08002268536903F00063536194F8CC34002B37
:10AA180040F05F820121236884F8CC145B6D2046E6
:10AA2800C3F38303C4F8D0343EF0D8FC20683EF06A
:10AA380037FFC10433D56B68102123F001036B6025
:10AA480020683EF044FD4FF67F3106F51063227909
:10AA58000398824200F24182EB6943F00113EB61F3
:10AA6800E37B002B00F05682D5F8843043F00B03CB
:10AA7800C5F884306B6C43F00B036B64D6F8003870
:10AA880004F29C4223F4FE63C6F80038A1792068DA
:10AA980000F0E4FC2268536903F480535361206892
:10AAA8003EF0FEFE820416D520683EF02BFF20689B
:10AAB8003EF058FDE0712768FFF778FEE27901461D
:10AAC800384600F06BFA20463DF0F9FA22685369DF
:10AAD80003F40053536120683EF0E2FE030707D5F4
:10AAE80020463DF042FB2268536903F00803536196
:10AAF80020683EF0D5FE070600F1178220683EF078
:10AB0800CFFEC0020CD5A046012706F512692379AD
:10AB1800BB4200F228822268536903F48013536110
:10AB280020683EF0BDFE81022AD523464FF0010C75
:10AB380006F53261207960451DD993F87C72086862
:10AB4800012F40F02682002880F22382D4F8D424F2
:10AB580082EA1040C20700F11C8283F87B72B06958
:10AB680040F08000B0617069000600F112826B68E5
:10AB780043F400736B602268536903F40013536154
:10AB880020683EF08DFE410007D520463DF0C3FA0F
:10AB98002268536903F08043536120683EF080FEC9
:10ABA80042070AD523685D686B0702D520463DF049
:10ABB800B8FA226853682B43536009B0BDE8F08F98
:10ABC800B3F5402F7FF4D1AE0822304604F29C4101
:10ABD8003EF0F7FD242303FB0747D7F86832C8F394
:10ABE8000A184344BFE620683EF05EFEA2460027EE
:10ABF800049006F53068049B002B3FF4C1AE049B1B
:10AC0800DB0779D55FFA87FB594620683EF05CFE82
:10AC180010F0010F81461FD00123C8F808302068C2
:10AC280094F806C000F5306303EB4713BCF1010F3D
:10AC3800016C9A6840F08B8012F0080F07D0B34877
:10AC4800814209D9120407D54FF4004203E012F0FB
:10AC5800200F5AD020229A6019F0080F21D008231B
:10AC6800C8F808302368A9491A6C03F5306303EB68
:10AC780047138A42986804D9000444BF4FF400403F
:10AC8800986020460592FDF759FA059A9F498A422D
:10AC980007D9A179012904D1206804F29C4200F067
:10ACA800DDFB19F0100F1CBF1023C8F8083019F08D
:10ACB800020F14D07369190642BF6B6843F48063AE
:10ACC8006B609AF85732012B06D10023594620466B
:10ACD8008AF857323EF008FA0223C8F8083019F00B
:10ACE800200F1CBF2023C8F8083019F4005F1CBFD0
:10ACF8004FF40053C8F80830049B01375B080493ED
:10AD080008F120080AF1240A75E7DFF800C2614556
:10AD180001D9120498D41A69DAF87432C2F312020B
:10AD28009B1ACAF868326FB9D4F864222AB901218B
:10AD380004F29C4200F092FB04E0D4F860221A442A
:10AD4800C4F8602259462046FDF7BEF984E7DFF8CB
:10AD5800C0C1614507D111043FF576AF9206F1D520
:10AD680020229A60EEE7002FECD1D4F86432002B51
:10AD7800E8D1394604F29C42DCE7049BDA0740F14B
:10AD88009B805FFA8AF31946206807933EF0A5FD79
:10AD980010F0010F804620D001216B6B0AF00F02E2
:10ADA80001FA02F223EA02036B63CBF80810A179D7
:10ADB80001290DD1D7E9072313443B62BAF1000FEB
:10ADC80006D1636A23B9206804F29C4200F046FB6E
:10ADD80020465FFA8AF1FDF795F918F0080F1CBFB5
:10ADE8000823CBF8083018F0100F1CBF1023CBF83D
:10ADF800083018F0400F1CBF4023CBF8083018F07B
:10AE0800020F10D0514630463EF061FBFB7D012B0E
:10AE180006D100232046FB755FFA8AF13EF065F9FA
:10AE28000223CBF8083018F0800F45D0D7E9093253
:10AE38009A4241D8A3EB0208FB692168984528BFCC
:10AE4800984601F5106308F1030803EB4A130591CE
:10AE58004FEA98080693069B9969D7E9093289B29F
:10AE6800414527D393420BD80121059B0AF00F00D7
:10AE7800D3F83428814022EA0102C3F834281BE0C1
:10AE8800A3EB0209FB69079A994528BF9946A3795C
:10AE980005980093396A1FFA89F33EF07FFC3B6AF4
:10AEA80009F103084B443B62BB6A4FEA98084B44DC
:10AEB800BB62D0E79342D7D9049B0AF1010A5B0829
:10AEC800049324370BF1200B68E520463DF03EF94A
:10AED8007CE520463DF02BF9A8E599601A682033F7
:10AEE80022F4001243F8202CC3F8E811D3F8E0212B
:10AEF80022F40012C3F8E021D3F8E02142F0006206
:10AF0800C3F8E021039A01320392A0E50A30544FB6
:10AF18000A31544F6B6943F4005343F02B036B61C0
:10AF28002B6943F00B032B61A8E501222427B369A1
:10AF380004F2572023F08003B36106F532632179C8
:10AF480091427FF6DBAD07FB02F1415C012907D195
:10AF5800196841F000611960196841F08041196071
:10AF680001322033EBE798F83C30D9F80020012B68
:10AF780009D1002A07DA67F07F01204688F83B30BC
:10AF8800C9B23EF0C8F9013708F1240809F12009CF
:10AF9800BDE50CF1010C24332031CBE5022A4AD15E
:10AFA800274B284A0B44934239D9274B274A0B444D
:10AFB800934236D9264AA1F57403A3F51053934258
:10AFC80031D9244AA1F18373A3F5E74393422CD3E3
:10AFD800214B224A0B44934229D9214B214A0B4445
:10AFE800934226D3204B214A0B44934223D3204A31
:10AFF800A1F1B773A3F5585393421ED31D4B1E4AB4
:10B008000B4493422CBF06230723C26822F47052D4
:10B01800C260C26842EA8323C360002070470F23DE
:10B02800F3E70E23F1E70D23EFE70C23EDE70B23FE
:10B03800EBE70A23E9E70923E7E70823E5E700BF89
:10B04800405327FFFF340C00401E1BFF3F420F00F8
:10B058007F4F120020D6130060B6E5FE5FE31600AE
:10B0680000D3CEFE40771B00C05BB3FEC091210029
:10B0780020753800E05459FEE09C410084B02DE969
:10B08800F843044609A880E80E00002319469DF8F5
:10B0980024809DF82E7003F14002013304EB8202F4
:10B0A8000F2B5160F7D104F50066002F64D1736847
:10B0B80043F002037360A36B23F40013A3632368B4
:10B0C80043F040032360236843F080032360002596
:10B0D80003212046C4F8005E3EF03DFA10212046C8
:10B0E8003EF0F5F9014620463EF014FA0843C0B296
:10B0F800401B18BF01202A464FF090414FF0006CCA
:10B108004FF67F3E356104F510637561F561A8451A
:10B1180037D800224FF0904511464FF0006C4FF69B
:10B128007F3E04F5306390453DD8336923F480733E
:10B1380033610023A3616FF0804363619DF826307B
:10B148001BB9A36943F01003A361A2691F4B134302
:10B15800A3619DF82A301BB1A36943F00803A361DA
:10B16800012F01BFA36943F0804343F00403A361A7
:10B17800BDE8F84304B07047A36B43F40013A3631E
:10B18800A5E7D3F80090B9F1000F0ADA3DB9C3F882
:10B1980000C01A610135C3F808E02033B7E7196029
:10B1A800F7E71A60F5E7D3F80090B9F1000F0ADA6B
:10B1B8003AB9C3F800C019610132C3F808E0203376
:10B1C800B1E71D60F7E71960F5E700BF00383C807C
:10B1D80030B54A780B78012A00EB431300F500607C
:10B1E80029D1D3F80029002A0BDAD3F8002942F034
:10B1F8000062C3F80029D3F8002942F08042C3F85E
:10B20800002901240A78C56B02F00F0204FA02F241
:10B2180025EA0202C2630978C26901F00F018C4075
:10B2280022EA0402C261D3F80019174A0A40C3F897
:10B238000029002030BDD3F8002B002A0BDAD3F800
:10B24800002B42F00062C3F8002BD3F8002B42F029
:10B258008042C3F8002B01240A78C56B02F00F0264
:10B2680004FA02F225EA0242C2630978C26901F0CF
:10B278000F018C4022EA0442C261D3F8001B034A42
:10B288000A40C3F8002BD4E7007833EC0078F3EFDA
:10B29800F7B54B7891F800C0012B6D4D6D4E00EB62
:10B2A8004C1440F089800F6904F510633FBB1F6997
:10B2B8003D401D611D6945F400251D611D6935402E
:10B2C800012A1D614DD1CA6902B15A610B79012B5E
:10B2D8000CD1D0F8083813F4807FD4F800390CBFAB
:10B2E80043F0005343F08053C4F80039D4F80039D0
:10B2F80043F00443C4F80039002003B0F0BD1F69CF
:10B308003E401E611E6935401D610D698E68BCF1A5
:10B31800000F0CD1B54288BF0E611D6945F40025A8
:10B328001D610D691E69C5F312053543C8E735442B
:10B33800013DB5FBF6F5484FD3F810C0AEB207EAA9
:10B34800C54545EA0C051D610D79012DE9D11D6939
:10B3580025F0C0451D611F69750705F0C0453D43CF
:10B36800DEE7D4F8003943F00443C4F800390B7918
:10B37800012B0DD00B69002BBED001230A78D0F821
:10B38800344802F00F0293402343C0F83438B3E73F
:10B39800D0F8083813F4807FD4F800390CBF43F094
:10B3A800005343F08053C4F8003900920B8A0A789E
:10B3B800C9683EF0F3F99FE7D4F8107B04F53063D1
:10B3C8003E401E611E6935401D610E698D68BCF1E5
:10B3D800000F27D106B10D610D621E69C5F3120574
:10B3E80035431D611D6945F40025012A1D6102D1FF
:10B3F800CA6802B15A610B79012B0CD1D0F8083810
:10B4080013F4807FD4F8003B0CBF43F0005343F0A3
:10B418008053C4F8003BD4F8003B43F00443C4F81D
:10B42800003B69E7002ED8D02E44013EB6FBF5F666
:10B43800B6B275430D62084D1F6905EAC6453D431E
:10B448001D610D6A1E69C5F312053543CDE700BFBE
:10B45800FFFF07E00000F8FF0000F81F30B5114CAF
:10B46800056C00F53063A54203D9D0F8004B002CD9
:10B4780016DB00241C611C69012944F400241C61AA
:10B488001C6944F018041C611C6944F0C0441C6128
:10B4980001BF5A61D0F8003B43F08023C0F8003B5D
:10B4A800002030BD0A30544FA8B1304BDA6802F49E
:10B4B8004032B2F5403F10D12D4B984250D92D4B18
:10B4C80098424FD92C4B984235D92C4B984216D9D3
:10B4D8002B4B984231D901207047DA6802F4403288
:10B4E800B2F5003F0DD1274B984239D9264B9842E7
:10B4F80038D9264B98421ED9254B9842EBD80323BE
:10B508001CE0DB6803F44033B3F5803F0AD1214BDC
:10B51800984225D91B4B984224D91F4B98420AD9E7
:10B52800194BEAE71D4B98421AD91D4B984219D975
:10B538001C4B9842CFD8022300E004231A490A681A
:10B5480022F00F021A430A600A6802F00F029342BF
:10B558000AD0086800F00F00C01A18BF0120704711
:10B568000023EBE70123E9E70020704700080246C3
:10B578000048E8010090D00300D8B8050020A107D2
:10B588000068890940787D0180F0FA02C068780473
:10B5980000E1F50520BCBE0060343C0200127A00D0
:10B5A8000024F40000366E010020024010B5044665
:10B5B800F7F72CFB03480121034A3AF0EDFC20463B
:10B5C8003EF0FBF9043F0708BD2708082DE9F843BA
:10B5D80004460D4600AFEFF31188102383F3128859
:10B5E800BFF36F8F04282A4A98BF2A4BE9468AB0CE
:10B5F8009668117C98BF53F820306A4688BF264B5E
:10B60800CDE9073140F201332448ADF82430244B0A
:10B61800CDE9050442F8103F00234FF43151214889
:10B62800F7F7C2FBCD4645B1EB69C3F3080323B175
:10B6380001211D4A1B483AF0AFFC2EB130463EF0BE
:10B648006BFC08B1037803B91848E9468AB06A4622
:10B65800174B0790CDE9053640F20133ADF820309D
:10B66800144B42F8103F00234FF411510D48F7F7DF
:10B678009BFB2946CD462046FFF798FF88F31188A3
:10B68800BFF36F8F3046F8F7A9FBBD46BDE8F883D6
:10B698009C3B002028490708CD270808E32708080D
:10B6A80005000001043F07080B280808DB270808E5
:10B6B8002C2808080400000138B50A4B53F820402C
:10B6C800013053F82050A54200D838BD606830B129
:10B6D800037EDB0701D43EF04DF90834F3E7236815
:10B6E8009847FAE73C490708012270B52C4B2D4CC6
:10B6F8002D4D86B01A70AC421CD30320FFF7DCFF37
:10B708000420FFF7D9FF294C294D2646AE4204F103
:10B71800300413D301F0D4F8244CAC422AD301F0FE
:10B72800E3F839F030FB234A938923F0010393812E
:10B7380006B070BD54F8043B9847DCE754F80C3C5D
:10B74800059354F8103C049354F8143C039354F8AC
:10B75800183C029354F81C3C019354F8203C009385
:10B7680054E90A2354E90C01F5F74AFD54F8303C32
:10B778005E65CAE7D4E90A23B3F1FF3F08BFB2F117
:10B78800FF3F05D052EA0301206803D100F078FD9D
:10B798003034C2E70849183001F0A6F9F8E700BFCD
:10B7A80082490020E43C0708E83C0708E83C070811
:10B7B800183D0708703100203FA00508E02370B548
:10B7C800134E012203FB0066002386B0CDE9042353
:10B7D8000F220193CDE9023218234FF4A0720D4DC8
:10B7E8000D4903FB0055044602FB00110B4B304684
:10B7F8000095F5F705FD337C2C7423F004033374AE
:10B80800074B013403EBC423EE606B6006B070BDD8
:10B81800903000209C3B002000690020559B0508C3
:10B82800006100207FB50020FFF746FF2D4B03F590
:10B83800006282F3088883F30A88F0232A4C2B4D90
:10B8480084F822300023E37723766376A37684F89E
:10B858002030636A43F4E0236362F8F769F9F8F784
:10B86800A7FA4FF0FF33A362E362F8F7BFFCF8F7DB
:10B8780041FBF7F72DF91E4800F0DEFCF6F7DEFF76
:10B888001C4CAC422AD30120FFF716FF02201A4CA9
:10B89800FFF712FF01F00CF8184B00259C61184BBC
:10B8A80045F6E062059301231649CDE90353204686
:10B8B800154BCDE901550095F5F7A2FC0646237C0A
:10B8C800204623F0040323743EF05BFB2846FFF771
:10B8D80075FF314620460C4AF8F73CFA54F8043B09
:10B8E8009847CEE70061002000ED00E0E43C07083F
:10B8F80050320020E03C0708703100209C3B0020BB
:10B90800040C0808406A0020F1B6010838B5064C56
:10B91800064DAC4201D3002038BD2046D4E90112BF
:10B928003EF095F81434F4E7CC100020E010002025
:10B9380030B5054B85B0DDE908450293CDE90045F2
:10B948003EF043F805B030BDFB50050838B5064C4D
:10B95800064DAC4200D338BD20463EF09DF8002885
:10B96800F9D11C34F5E700BFB0100020CC1000203E
:10B9780073B50C46EFF31181102585F31288BFF3D8
:10B988006F8FC5685DB125602B68C360836901331B
:10B998008361002081F31188BFF36F8F11E052EAB1
:10B9A800030603D16FF00B002560F3E7CDE9002310
:10B9B8000246083000F088FE18B9034B9B685B69A3
:10B9C800236002B070BD00BF9C3B0020F7B50E4657
:10B9D80004469DF82010EFF31187102080F3128899
:10B9E800BFF36F8F256AE068854245D22568AC426F
:10B9F80019D0C5B128463EF0B4F805F1180001F099
:10BA080003F93146A268686957F0B5FC0023284657
:10BA1800C5F8983000F0D4FC04F10800394600F06D
:10BA2800DBFD002036E0A268D9B13146E06957F065
:10BA3800A2FCE369A26813446269E361934201D1FD
:10BA48002369E361236A10210133236204F124008E
:10BA58003EF058FC0028DFD187F31188BFF36F8FC1
:10BA680018E0A06923693146984208BF6069801AC6
:10BA7800A06157F080FCE5E752EA03010CD00849C1
:10BA880004F1080089684E61CDE900233946224651
:10BA980000F01AFE03B0F0BD6FF02200DCE700BF33
:10BAA8009C3B0020F7B504460846EFF311861021A9
:10BAB80081F31288BFF36F8F216A00293BD0A268F7
:10BAC800A16957F058FCA369A26825681344626904
:10BAD800A361934204BF2369A361236AAC4203F1C3
:10BAE800FF33236236D02846002D34D000273EF09D
:10BAF80038F805F1180001F087F86969A268E0696B
:10BB080057F039FCE369A268284613446269E36187
:10BB1800934204BF2369E361236A01332362C5F8B2
:10BB2800987000F04DFC04F10800314600F054FD17
:10BB3800384603B0F0BD52EA030111D00A498968BA
:10BB48004861CDE900233146224604F1080000F09F
:10BB5800BBFDEEE7002086F31188BFF36F8FE8E79F
:10BB68006FF02200F7E700BF9C3B00202DE9F3416E
:10BB7800044617461E46EFF31188102383F31288F4
:10BB8800BFF36F8F304BC2689B6872B18068984270
:10BB980017D057EA060216D188F31188BFF36F8FC2
:10BBA8006FF00F0002B0BDE8F08193F90E1001327A
:10BBB8002161C4E9023288F31188BFF36F8F002036
:10BBC800F0E72169F3E793F90E1090F90E309942E6
:10BBD80030DA9942A8BF19463EF01BF805462246BE
:10BBE8004146CDE90076194800F06EFD0028E6D000
:10BBF800EFF31186102383F31288BFF36F8FA068C9
:10BC0800D0B1236821699C420AD04BB193F90E3018
:10BC18009942A8BF19466FF07F039942B8BF1946E9
:10BC28003DF0F7FF40B13146084800F0D5FC6FF011
:10BC38000A00B7E70025D2E7002DF4D186F3118872
:10BC4800BFF36F8FF3E700BF9C3B002083490020C0
:10BC5800F8B583680546002B40D0234A9268934282
:10BC68003FD1C368012B03D9013BC3600020F8BD55
:10BC7800EFF31187102383F31288BFF36F8F0169E5
:10BC880080683DF0C6FF2C68A54207D10023C5E9AE
:10BC9800023387F31188BFF36F8FE7E7002CF5D0E5
:10BCA800D4E90032002613605A60237CC4E9006698
:10BCB80023F002032374A66004F1180000F0A4FF27
:10BCC800AC6094F90E3020462B61C4F8986000F0FF
:10BCD80077FB3946054800F07FFCC7E76FF0150091
:10BCE800C5E74FF0FF30C2E79C3B002083490020A6
:10BCF80073B51546EFF31186102282F31288BFF34D
:10BD08006F8F0468B4B12368426823F00303944238
:10BD180008BF4360036023689B0704D0656820461A
:10BD28003EF01CFB2C4686F31188BFF36F8F20462C
:10BD380002B070BD55EA0302F5D000F108023146A1
:10BD48001046CDE9005300F0BFFC0028EFD1024BAC
:10BD58009B685C69EBE700BF9C3B002070B5EFF384
:10BD68001186102383F31288BFF36F8F0468A042F3
:10BD78001CD0DCB1D4E90032002513605A60237C62
:10BD8800C4E9005523F002032374A56004F11800E8
:10BD980000F03AFF2046C4F89850656100F010FBA7
:10BDA8003146BDE870400A4800F016BCD0E90232BE
:10BDB8009A4218BF01330221836010303EF0A2FA84
:10BDC8000028EDD186F31188BFF36F8F70BD00BFD7
:10BDD8008349002013B5EFF31181102484F31288EE
:10BDE800BFF36F8F846844B1013C846081F311888C
:10BDF800BFF36F8F002002B010BD52EA030406D1D2
:10BE080081F31188BFF36F8F6FF00F00F3E7CDE96F
:10BE180000230246014800F057FCECE78349002064
:10BE2800F8B50546EFF31187102383F31288BFF3A3
:10BE38006F8F00262C68A5421AD0CCB1D4E9003205
:10BE4800002613605A60237CC4E9006623F00203CD
:10BE58002374A66004F1180000F0D6FE6FF00A0300
:10BE680066612046C4F8983000F0AAFA0126E1E796
:10BE780000230221AB6005F110003EF043FA28B917
:10BE880026B987F31188BFF36F8FF8BD3946BDE82F
:10BE9800F840014800F0A0BB834900202DE9F04F8D
:10BEA80004464FF0FF3A4FF0FF3B614E85B0EFF389
:10BEB8001187102383F31288BFF36F8FD4F8E450EF
:10BEC8005DBB022104F1FC003DF07DFF00287FD01E
:10BED80004F1F409D4F8F4504D4500F08680002DA3
:10BEE80000F08380D5E900324FF0000813605A60F3
:10BEF8002B7CC5E9008823F002032B74C5F8088061
:10BF080005F1180000F080FE01232846C5F8983096
:10BF1800C5F8148000F054FADCE7D4F8E8202B6860
:10BF28009542C4F8E43008BFC4F8E830D4F8FC30CF
:10BF380043F00203C4F8FC30EB6823F0040343F039
:10BF48000103EB606B6887F31188BFF36F8F284696
:10BF58009847EFF31187102383F31288BFF36F8F8D
:10BF6800EB68D80623F001024AD4EA60EB689A0726
:10BF780017D5306823F00203EB6090B10022036804
:10BF880078B141688D4249D10368002A40D172686E
:10BF98003360904200D17360002340F8083BFFF7FC
:10BFA800DDFED4F8FC3023F00203C4F8FC30DB05D6
:10BFB8003CD4D4F8E430003B18BF012387F3118840
:10BFC800BFF36F8F002B3FF472AF3DF0C6FF6EE7F3
:10BFD800D4F8FC30D90608D5C4F8FC0087F31188DA
:10BFE800BFF36F8F05B0BDE8F08F00233946CDE968
:10BFF80000AB029304F1EC020E4800F08BFC56E70C
:10C0080023F01103EB6005F11000FFF7A7FEADE781
:10C0180013607368984208BF7260BDE702461BB19F
:10C02800196818460B46ABE71946FAE70023C5E737
:10C03800C43B002083490020F8B5C36804469A072A
:10C048000E46C3F3400542D45F0742D40B680BB9D0
:10C0580083680B60E368D80742BFA3680225336092
:10C06800376858BF012557B31B4B9A68D7F8E0309B
:10C078009A421ED13DF047FF80F00100C0B2D7F8C8
:10C08800FC30D907C3F380021CD5F2B1F8B1002304
:10C098002360D7F8E83073B9C7E9394438463DF02A
:10C0A800BCFEE36843F00403E3603368A3602846FA
:10C0B800F8BD0020E3E71C60C7F8E840EEE76FF042
:10C0C800150506E06FF0120503E01B07DFD56FF0DA
:10C0D8000F0500233360EAE79C3B00200146014836
:10C0E8003DF0F5BE50330020F0B50446002089B07D
:10C0F8000E9DC4E9390004F1EC00C4E93B0004F1E9
:10C10800F400C4E93D0055B32879002840F2011035
:10C1180008BF0120C4F8FC0000204FF0FF364FF0A4
:10C12800FF37CDE90330CDE90100CDE906672046A8
:10C138000C4B009400F0C8F855B1296811B120469D
:10C148003DF0E7FE6B791BB1A38943F00103A3819E
:10C15800204600F095F8C4F8E04009B0F0BD012091
:10C16800D8E700BFA5BE010837B501900846EFF330
:10C178001184102181F31288BFF36F8FC16811F009
:10C188001E0F16D153EA020508D101A9FFF754FF83
:10C1980084F31188BFF36F8F03B030BD41F00801FD
:10C1A800C160019910308161034900F09DFC0120B4
:10C1B800EEE70020ECE700BF639E05080146014852
:10C1C800FFF7D2BF50330020F0B585B00C461746B4
:10C1D8001D460190EFF31183102181F31288BFF3FC
:10C1E8006F8F204603A903933DF0F8FD55EA070336
:10C1F800039E09D1204601A9FFF71EFF86F3118887
:10C20800BFF36F8F05B0F0BDE3683A4643F008030B
:10C21800E360019B0449A36204F110002B4600F07F
:10C2280063FC0120EAE700BF639E05080146014858
:10C23800FFF7CABF50330020012303748381002312
:10C24800C0E92033C0F88C30014B9860704700BFBC
:10C258009C3B002008B500F069FA70B1074B9B6859
:10C26800DB7B53B9EFF31180102383F31288BFF3FC
:10C278006F8FBDE8084000F0C5BA08BD9C3B0020A0
:10C2880038B50446EFF31185102383F31288BFF302
:10C298006F8F037C5B070FD5183000F0B5FC237C4B
:10C2A800204623F00403237400F08AF82946BDE8E9
:10C2B8003840044800F090B985F31188BFF36F8FB8
:10C2C80038BD00BF83490020F0B5002587B005952B
:10C2D800109DDDE9127604950F9D044603950E9D89
:10C2E80002950D9D01950C9D0095F4F789FFB6F117
:10C2F800FF3F08BFB7F1FF3F05D056EA070305D156
:10C308002046FFF7BDFF204607B0F0BD3A4633464A
:10C3180004F11800014900F0E7FBF4E73FA0050825
:10C328006FF00A01094A9368C3F898100849C3F8DE
:10C3380094004B6843F080534B60002383F31188CB
:10C34800BFF36F8F9368D3F8980070479C3B002029
:10C3580000ED00E038B5184CA168206A0B688142EE
:10C3680014BF1A46002249680B605960A368216A05
:10C378002AB9124AC3E900210B6023620AE092F944
:10C388000E5093F90E00854212DD5168C3E9002171
:10C398000B605360E569094B9D4200D005B9E5681B
:10C3A800A3689D4202D028463DF002FFA56138BD32
:10C3B8008A42DED01268DBE79C3B0020B83B0020B5
:10C3C80070B590F91020037C002A2FDBD9062DD1F7
:10C3D8001A4C63F07F032246037452F81C3F216A0B
:10C3E800934207D1C0E90021086020620FE099421A
:10C3F800F8D01B68002BF5D093F90E6090F90E5019
:10C40800AE42F4DD5968C0E9003108605860E5695A
:10C41800954200D005B9E568A3681A7CD20606D112
:10C42800DA897F2A03D9AA690AB9A36170BDAB4228
:10C4380002D028463DF0BCFEA561F7E79C3B0020F2
:10C4480038B590F910200146002A037C04DA03F07D
:10C458007F0303743DF083FD0D4D2A4652F81C4FAF
:10C46800AB68944200D004B9EC688B4207D01A7CC0
:10C47800D20604D1DA897F2A01D9A2692AB1A34256
:10C4880002D020463DF094FE2346AB6138BD00BF84
:10C498009C3B0020002A2DE9F8430CBF4FF0100800
:10C4A8004FF00808027C044618EA020F0D4665D1D1
:10C4B80048EA0203D2090CD10374B8F1080F7ED1FF
:10C4C800A36813B120463DF052FD102704F1180669
:10C4D8000FE003F07F0303743DF041FDEDE785F3C2
:10C4E8001188BFF36F8FEFF3118587F31288BFF3BD
:10C4F8006F8F304600F088FB0B30F0D0A66D04F14A
:10C508005807B74211D04FF0000976B130463DF0D8
:10C518002EFDC6F8989006F1180000F075FB30461D
:10C52800FFF74EFFA66DB742EFD1294B9B689C429F
:10C5380045D1EFF30587003F18BF0127DFF890903A
:10C548004B4653F81C6F9E4200D00EB9D9F80C60C8
:10C55800D9F80830B34202D030463DF029FEB8F190
:10C56800100FC9F8186009D0204639F0C1FE2046DE
:10C5780000F066FA17B11748FFF75EFE144B9B6888
:10C58800A3421ED1EFF30583DBB9A289D20711D5E7
:10C5980085F31188BFF36F8F83F31188BFF36F8F13
:10C5A8000423184602DFEFF31185102383F3128862
:10C5B800BFF36F8F2846BDE8F843FFF7B1BE0027E9
:10C5C800BCE785F31188BFF36F8FBDE8F88300BF20
:10C5D8009C3B00205032002049B9EFF3058030B968
:10C5E800054B9A699B689A4201D0FFF799BE81F37F
:10C5F8001188BFF36F8F70479C3B002070B50F4DBB
:10C6080006462B4653F81C4F9C4200D004B9EC68F0
:10C61800AB681A7CD20604D1DA897F2A01D9A269CB
:10C628002AB1A34202D020463DF0C2FD2346AB61A9
:10C638003146BDE870400248FFF7CEBF9C3B002062
:10C648008349002070B5EFF31186102383F3128815
:10C65800BFF36F8F1A4CA168206A0B68814214BF20
:10C668001A46002249680B605960A368216A2AB9F2
:10C67800144AC3E900210B6023620AE092F90E50C4
:10C6880093F90E00854216DD5168C3E900210B605D
:10C698005360E5690B4B9D4200D005B9E568A36876
:10C6A8009D4202D028463DF083FDA5613046BDE895
:10C6B8007040FFF735BE8A42DAD01268D7E700BF6C
:10C6C8009C3B0020B83B0020F8B5DDE906670C4626
:10C6D8001146EFF305833BB1002383F31188BFF3C1
:10C6E8006F8F0423184602DF0D4B0E4A98681060BE
:10C6F800EFF31182102282F31288BFF36F8F9D68C7
:10C7080028463DF04DFC32463B4605F118000649E7
:10C7180000F0EAF92046BDE8F840FFF701BE00BF87
:10C728009C3B0020CC3B00203FA00508F8B5044600
:10C73800EFF31187102383F31288BFF36F8F037C05
:10C7480049B203F01F02002A0CBF0126002635D18A
:10C7580003F07F032A4D03743DF001FC2A46037C55
:10C76800817363F07F03037452F81C3F286A934275
:10C7780007D1C4E9002004602C620DE09842F8D08B
:10C788001B68002BF5D093F90EC08C45F6DD59686F
:10C79800C4E900310C605C60EC69944200D004B9D3
:10C7A800EC68AB689C4202D020463DF001FDAC61CC
:10C7B80087F31188BFF36F8F3046F8BD9B071CD5F0
:10C7C80085683DF0CCFB81732B689D4209D16B686D
:10C7D800C4E900531C606C60EAE76A689A42F6D0C4
:10C7E8001B68002BF3D093F90E208A42F5DD5A68B6
:10C7F800C4E9003214605C60DAE78173D8E700BFEF
:10C808009C3B0020034648B9EFF3058232B9064A3B
:10C8180091699268914201D0FFF782BD83F3118834
:10C82800BFF36F8F704700BF9C3B0020F8B550EAFC
:10C83800010305460C4603D13DF08FFB0020F8BDEF
:10C84800EFF31187102383F31288BFF36F8F144E11
:10C85800144BB0681860FFF7F3FDB0682A4623460A
:10C868001149183000F040F9B36804461A7CC3F83F
:10C87800947042F004021A746FF00A02C3F8982008
:10C888000A4A536843F080535360002383F31188A6
:10C89800BFF36F8F3DF093FC201A20EAE070CEE7DB
:10C8A8009C3B0020CC3B00203FA0050800ED00E0A9
:10C8B800024B03F11C02C3E9072270479C3B00208E
:10C8C800EFF31181102383F31288BFF36F8F054BA9
:10C8D8009A68D37B013BD37381F31188BFF36F8FC1
:10C8E800704700BF9C3B0020EFF31180102383F3B7
:10C8F8001288BFF36F8F034B9A68D37B0133D373CE
:10C90800FFF77CBE9C3B0020014B9868704700BF36
:10C918009C3B0020D3B5DDE90667089CCDE900679C
:10C92800FFF7D2FE1CB1034B9B685B69236002B022
:10C93800D0BD00BF9C3B0020027C034612F01F02C2
:10C9480010D10A4988420DD00949086868B1D989C7
:10C958007F2909D893F90E20064B1B689A42B8BF65
:10C968000020704700207047104670479030002024
:10C97800CC060020D03B00200122044BC01A044BF7
:10C98800C0105843034B1A54704700BF303300207F
:10C99800ABAAAAAA83490020F8B50B4B04461E7C13
:10C9A80018230A4D0A4F03FB0655284600F02CF9B8
:10C9B80034B1BB5D2846E21A0649D31700F094F853
:10C9C8000023BB55F8BD00BF9C3B0020303300203E
:10C9D8008349002081C90108F8B5EFF311871023B6
:10C9E80083F31288BFF36F8F124E134BB568186824
:10C9F800A84206D13DF0DCFB87F31188BFF36F8FA7
:10CA0800F8BD00221A60337C0C4AD35C002BF3D0AB
:10CA18002846FFF791FF04460028EDD02B7CDB0663
:10CA2800EAD1FFF797FCB369AB42E5D12046FFF79F
:10CA3800B3FFE1E79C3B0020CC3B0020834900206A
:10CA4800EFF31181102383F31288BFF36F8F0A4A23
:10CA5800536A834207D1DB6F536281F31188BFF3B6
:10CA68006F8F70471346002BF7D0DA6F8242F9D1E7
:10CA7800C26FDA67F1E700BF9C3B0020024B1868E1
:10CA8800984208BF00207047D006002008B502462B
:10CA9800FFF7F4FF6FF00041C8B18A4215D2D0E920
:10CAA8000230B0F1FF3F08BFB3F1FF3F03D16FF091
:10CAB8000040801A08BD8B4270F1000001DB054878
:10CAC800F7E79A4201D2981AF4E70020F2E78A427F
:10CAD800EDD3EFE7FEFFFF7F024B186808B1FDF7C3
:10CAE800B9BD7047D8060020B3F1FF3F08BFB2F1C7
:10CAF800FF3F2DE9F84F04469A461546984679D0E7
:10CB08000161EFF31187102383F31288BFF36F8F4E
:10CB1800BAF1000FDFF8E89023DBFFF7DDFF374BB2
:10CB280006461A68003A18BF012245194AF100035F
:10CB3800521943F10003D9E90051551943EB010893
:10CB48000121DFF8C090C4E90223FFF797FFD9F865
:10CB580004A0D0B9C4E9009ACAF80040C9F8044052
:10CB680025E06FF00102D9E90013521A4FF0FF31A6
:10CB780061EB0303521B63EB0A03012A73F1000103
:10CB8800BCBF012200230021DBE7D0E9022ED4E953
:10CB9800023C93427CEB0E0B23DAD21A6EEB0C03A9
:10CBA800C0E902234368C4E900031C604460FFF73E
:10CBB80065FF84420DD1114B1B68013309D111B9AE
:10CBC800FFF78AFF06463046FFF760FF0021FDF7B2
:10CBD800DBFC87F31188BFF36F8F28464146BDE819
:10CBE800F88F9B1A6CEB0E025045C4E90232B1D0A3
:10CBF8000068AEE70025A846EFE700BFD80600208A
:10CC080048330020D0060020F8B50446EFF311861B
:10CC1800102383F31288BFF36F8F026872B3FFF794
:10CC28002DFF184B5B689C4208D0D2E90231D4E949
:10CC38000275DB1941EB0501C2E90231D4E9003282
:10CC48000025844213605A60C4E900550ED00020C4
:10CC58000D4A136823F001018C4204BF43F001031D
:10CC6800136086F31188BFF36F8FF8BDFFF734FFA9
:10CC7800FFF70CFF2946FDF787FCE8E76FF0150082
:10CC8800E6E700BFD0060020D43B0020EFF3118276
:10CC9800102383F31288BFF36F8F064B40F0010017
:10CCA8001B681B1A5842584182F31188BFF36F8FD3
:10CCB800704700BFD43B002000232DE9F0470C4605
:10CCC800334E344DDFF8D490334F30602B60D6F8B4
:10CCD8000080B8F1000F10D14FF0FF3340462B60B1
:10CCE800FFF7D4FE4146FDF74FFC84F31188BFF3EC
:10CCF8006F8FBDE8F047FFF76FBEFFF7BFFE6FF01D
:10CD0800004330B1D0E90212994272F10002B8BF73
:10CD18000B464345194684BF434641464FEAE37CE8
:10CD280038B18268B2EB030AC26862EB0C0EC0E944
:10CD380002AEA8EB01014FF0000A4FF01008D9F835
:10CD480000203160D218D9F8043043EB0C03C9E94C
:10CD58000023FFF793FE0028B9D0D0E902120A4356
:10CD6800B5D1D0E900210A6051600269C0E900AA82
:10CD7800386084F31188BFF36F8F9047EFF3118405
:10CD880088F31288BFF36F8FC7F800A0E1E700BFF0
:10CD9800D83B0020D8060020D43B00204833002090
:10CDA80010B5EFF31184102383F31288BFF36F8F4C
:10CDB800FFF792FE054AD2E90031C01841F100019F
:10CDC80084F31188BFF36F8F10BD00BF4833002074
:10CDD8002DE9F0410446EFF31186102383F31288FE
:10CDE800BFF36F8F03682BB186F31188BFF36F8F82
:10CDF800BDE8F081FFF74AFF07460028F4D1D4E9DF
:10CE08000A586A1C48F10003022A73F1000324D36C
:10CE18003DF0D9F9281848EB0101012871F100010A
:10CE280042DB3DF0D0F96FF00203281848EB01010E
:10CE380083426FF000438B413BDB3DF0C4F96FF058
:10CE480001022D1848EB01034FF0FF31521B61EB33
:10CE5800030320461949FFF747FE236B0133236379
:10CE6800236A63B186F31188BFF36F8F2046984712
:10CE7800EFF31186102383F31288BFF36F8F54F8F2
:10CE8800185FA542B0D0002DAED028463DF0AEF8D0
:10CE98000023C5F8983086F31188BFF36F8F2846B2
:10CEA800BDE8F0413DF06DB86FF001024FF0FF337F
:10CEB800CFE73A464FF00043CBE700BFD9CD010892
:10CEC800B3F1FF3F08BFB2F1FF3FF8B5044616467D
:10CED8001D4618D0EFF31187102383F31288BFF390
:10CEE8006F8FFFF791FEDDE90623C4E90A230023CB
:10CEF8003246236320462B460349FFF7F5FD87F3A7
:10CF08001188BFF36F8FF8BDD9CD010870B50546FC
:10CF1800EFF31184102686F31288BFF36F8FFFF7A3
:10CF280073FE20B184F31188BFF36F8F70BD6B6AF5
:10CF380063B184F31188BFF36F8F28466B6A9847F3
:10CF4800EFF3118486F31288BFF36F8F05F1180091
:10CF58003DF086F80028E5D03DF013F82146BDE8FD
:10CF680070400148FFF738BB84490020034610B5DC
:10CF7800EFF31184102282F31288BFF36F8FC16020
:10CF8800012181600068834205D184F31188BFF3D1
:10CF98006F8F002010BDD0E9003213605A60002363
:10CFA800C0E900333DF068F921460248FFF714FB59
:10CFB800EFE700BF84490020F8B507460C4616463F
:10CFC8003CF0A1FF08B10020F8BD0E4B9B68D3F8D8
:10CFD8008C50002DF7D0221DF5D2EFF311841023C9
:10CFE80083F31288BFF36F8F284647F00401B047D8
:10CFF80084F31188BFF36F8F0028E4D040F8045BF6
:10D00800E2E700BF9C3B00200146024A0020FFF7F0
:10D01800D3BF00BFF550050807B5064B4FF4406273
:10D02800009305494FF0FF330448FFF75DF803B05C
:10D038005DF804FB5449070820C90020503300203C
:10D04800F0B504468BB03DF079FB042C2BD0354D60
:10D05800286818B115F0A8FA00232B601CB3324BCE
:10D068009C4220D0002601AB0293304B214602A8F7
:10D078000393019641F06FFE01983146013015F097
:10D0880073FA0246286070B106AF384601993EF03F
:10D0980020FF274B214604A80593049741F05BFE27
:10D0A8002A68019BD65402F04BFD3DF033FA43F059
:10D0B80032FA3DF042FB01F02DFD00221D4D1E4BC2
:10D0C800D5F8F0401A7084B120460DF015F830B349
:10D0D800A06805F0CDF8D5F8F040002CF4D1D5F8CB
:10D0E800F0301C46DB68002BFBD1C5F8EC4000256E
:10D0F800124C01F0C9FE14F0E7FB0DF0EDF82068C2
:10D1080015F052FA25600E4C206815F04DFA25608E
:10D118003DF05FF90BB0BDE8F0403DF0FCB9E468C4
:10D12800DBE700BF383D0020844000208BA30508C2
:10D1380053BE05080C40002084490020183C0020FC
:10D14800143C0020002270B50446154B00EB810505
:10D15800C3E900229A60264630683EF03AFE02286B
:10D1680004F1040418D130680E4C206098B10E48C0
:10D178003DF0A9FB20683DF070F90C4802F042F937
:10D1880001F00EFD064920683DF062F90023236096
:10D1980001F006FD012070BDAC42DCD10020E3E7C0
:10D1A800E03B0020103C00206A6B0808E695080860
:10D1B80073B506463DF0AFF905F0EEFA15F0D6F86E
:10D1C800054615F0DFF80446641B002505F0ECFA67
:10D1D800A4F5806005F0EEFA01F09CFC00F028FC54
:10D1E8006B464FF4006230461F4900953DF0CDF87C
:10D1F80001461E4B1E4C1860009B194412F01AFD84
:10D208004FF4005201AB30461A4901953DF0BDF884
:10D218000146194B1860019B19440CF03FFF06F0BA
:10D22800F1F82946D4F8E80005F0E4FE1621D4F810
:10D23800E8003FF07DFA6621D4F8E8003FF078FA7C
:10D2480040F6B651D4F8E8003FF072FA294604F1E6
:10D25800D80005F0CFFE094804F0D2F80122084BA7
:10D268001A7002B070BD00BF97280808143C00204F
:10D278000C400020AE280808183C0020DC0C0808E8
:10D28800844900202DE9F04109280546A4B000F0A2
:10D29800878001F059FC044640B1002D40F083809E
:10D2A800424BD3F8F040003C18BF01242846FFF752
:10D2B8007FFF3DF05DFA002C6CD002AC3C4F01F0D2
:10D2C800D5FC4FF4007120463EF0E8FD3C6001F0CB
:10D2D80043FC0121054600F180083DF0FCF9354B7F
:10D2E800354A364936483FF044FF06A800F00CFBA3
:10D2F800344933483FF062FF002606AC14F8012B8E
:10D3080031492F4801363FF059FF202EF6D12F49D9
:10D318002B483FF02EFF43F0FFF802212C48FFF77F
:10D3280011FF00233B6001F0A7FC01234046294A76
:10D338000EA944F076F8A0B9029842F0C9FA039A07
:10D348000446014601AB01320EA844F08AF940B9FF
:10D35800039A019B9A4204D12146049856F039F861
:10D36800A0B14FF47A703DF032FA0A23194A0EA997
:10D37800404644F056F8DDE9032101AB0EA844F01D
:10D3880024FA0EA844F08EFB01F0C4FB00212846C5
:10D398003DF0A1F9104C6068FFF752FE002363606E
:10D3A80024B0BDE8F081002480E700BF0C400020D5
:10D3B800DC3B0020C8280808DB28080829290808B9
:10D3C800EC650708348D0808D2950808C5320808A6
:10D3D8009049070839290808E03B00202DE9F04F5B
:10D3E8008046AB4E89B0002841D00024202725462E
:10D3F8003368012B00F0B480B8F1000F40F0B4801E
:10D4080001264FF4405301933DF0DDF90390002CC1
:10D4180040F05E814FF4C87BA1460BFB06F3012662
:10D4280003F59C5A04930AF1080A01F0FBFC01F089
:10D43800AFFC05460290002800F0998047F01007DD
:10D4480001F05AFC934E306828B103781F4002D18E
:10D4580015F0AAF83760B9F1000F04D0002001F0E8
:10D468001DFF01F015FF284609B0BDE8F08F01F057
:10D4780051FB01F0ABFC05460028B6D1854FFFF7FC
:10D4880097FE3DF07CF93B68002B55D01A7822F0C6
:10D4980020021A703B689A681C78127892B1586812
:10D4A80008B103F0ADFF3B6801219B6807A807930B
:10D4B800FFF748FE98B93B6898683DF004FA76484B
:10D4C80001F0A0FF04217548FFF73CFE38B9082198
:10D4D8007348FFF737FE10B1724801F093FF3368C5
:10D4E80018052BD500F0BCFF012827D16E484FF056
:10D4F800000901F087FF6D4B706883F80090FFF713
:10D508009FFD3A68C6F804902AB11378990644BF7B
:10D5180043F02003137033681A0511D500F0A0FFFB
:10D52800441E18BF01243027336803F48073002B8E
:10D538000CBF254601245BE72C46C3E75C48D6E7C9
:10D548001BB9242704F00104EEE714F0020418BF05
:10D5580083F480634FF0280718BFC3F38024E3E700
:10D5680002264FF440134EE70326524B4BE73DF09B
:10D5780083F9059080B13DF09EF968B101F026FC71
:10D58800054648B93DF085F904287FF45BAF0320D0
:10D5980000F06CFF059D55E71CBB3DF06DF908B325
:10D5A80001F014FCF0B944483CF057FF01F0CCFB03
:10D5B80000283FD0414801F025FFB8F1000F02D004
:10D5C8003F4801F01FFF404601F066FD3D483DF031
:10D5D8007AF93D4801F016FFB8F1000F01D042F08A
:10D5E8009AFF01243DF048F92040C4B22EB101F061
:10D5F800EDFB10B903F002F806463DF0E4F8039B92
:10D60800049AC31A9A42054623D9B3FBFBF20BFBD3
:10D618001235632D10D9B9F1000F04D0002001F0A4
:10D628003DFE01F035FEC5F5C87066B3B04228BFAF
:10D63800304628E02548BEE7B9F1000F04D101F0D3
:10D6480047FE019801F02AFE0123C5F16400029308
:10D65800EBE79A4506D23DF0B6F8CDE90290DDF841
:10D668000890E2E6B9F1000F04D0002001F016FEA0
:10D6780001F00EFE039B5344581B16B1B04228BF5D
:10D6880030460028EBD014F0A1FE14F0E9FEE6E7DE
:10D69800E03B0020343D0020EC950808804907084D
:10D6A80060490708598C0808C88B08088449002075
:10D6B800E28B0808003030006A6B0808BC93080841
:10D6C800598E08085A2A0808D18E0808E8930808CD
:10D6D8004FF00009B6E600BF07B5114B186820B136
:10D6E80003B05DF804EB3DF0EEB80E4B1A68012A62
:10D6F8000FD19A68002A0CDD596851B109680C33BA
:10D70800C9880948009109493FF033FD03B05DF825
:10D7180004FB074803B05DF804EB01F073BE00BFDB
:10D72800103C0020E03B0020EC650708472908086A
:10D7380064920808F7B514F0FDFD01F0EBFB3CF02E
:10D7480048FE14F0AFFE3DF0DFF801F05BFD5048F5
:10D758003CF083FE3DF015F801F098FA01F0D4FB97
:10D76800B0FA80F00021400901F008F910B908204A
:10D7780001F0D0FB01F0C8FB18B901F0D1FB01F0B2
:10D78800C9FB42F0C8FE3CF0D8FF3CF0D5FF02F0E0
:10D7980011FB3F483CF061FE002000F067FE01F0FD
:10D7A800B3FB08B901F0AEFA0125012001F0C6F972
:10D7B800012001F0BDF901F0A7FBFFF763FD3CF084
:10D7C800ABFE012001F0E0F94FF480742846314E99
:10D7D80014F4106754D015B92F4801F013FE3578AA
:10D7E800002D3ED101F090FBFFF7F8FD0028EFD1A6
:10D7F80001F08AFB044601F08DF92046FFF7D8FCBA
:10D808003CF0BDFF012001F08FFA01F07DFB28B943
:10D81800224B012101A80193FFF794FC01F058FD68
:10D828001F4801F03BFD01F033FD3378012B1AD17D
:10D8380001F01CFA00F0A4FC044601F01DFA0420D3
:10D84800FFF7FEFB01F044FD002001F027FD01F089
:10D858001FFD012001F070FA032000F007FE0020F0
:10D86800B6E70025C4E70F4B0F4F3B6001F098F96E
:10D8780000F00CFD002304463B6001F091F9DEE75F
:10D88800002CB3D03FF0B3F8384603B0F0BD00BF6A
:10D898006A6B080885490020DF7F080850290808B6
:10D8A8003030300058290808103C002008B50CF02A
:10D8B80033FC00F027FB042107483FF0D3FE3CF07F
:10D8C80052FF01F015FB02F0B7F904F099FABDE830
:10D8D80008400CF035BC00BFFC400020014B187814
:10D8E800704700BF844900209FED010A704700BFC0
:10D8F8000000000000487047006889099FED010A90
:10D90800704700BF3333534038B505462021FBF735
:10D918008BFB041E11DA2146094837F0EEFE00247D
:10D9280021462022074837F0E8FEC4F120022819D2
:10D938000021BDE8384055F044BD1F2CF0DD38BD4E
:10D94800E8290808022A08080428034607B506D863
:10D9580001460E4803B05DF804EB01F0E5BC062172
:10D9680068460B4A33F0ECFA052801DD38F0F8FC7C
:10D97800442200F108036B44411C684603F8082C54
:10D9880001F0D2FC03B05DF804FB00BF292A0808A7
:10D998002E2A0808F8B5244DAB7DDB0731D52E6853
:10D9A800706801282DD9B168431ECA5C0A2A28D19B
:10D9B8004A1E002B01DC1A4608E0D45C0A2CFAD077
:10D9C800013BF6E78C5C202C02D101329042F9D859
:10D9D800002B0CDD541CA04209D15C1E0C448C4267
:10D9E80005D014F8017D0A2F0BD0202FF7D0014461
:10D9F800D21A11F8023C94083A2B00D10134013CA8
:10DA080000D2F8BD0422304608493EF01EFA04212F
:10DA1800064801F089FC2B6904332B61AB7D43F088
:10DA28000203AB75EBE700BF1C3C002086690808C1
:10DA380020220021014855F0C4BC00BFC44000208A
:10DA4800002238B50B4C0546A26062754FF0FF32D4
:10DA58006B680846C4E9032363602560A1613CF054
:10DA6800FCFC6B680BB90123A375BDE83840FFF7D0
:10DA780091BF00BF1C3C0020F8B503780446DBB119
:10DA88000E4FD7F8B80018B12146F3F73FFA98B10E
:10DA98002046F3F74DFA461C304641F01CFF054678
:10DAA80050B13246214655F066FC05491C22081D36
:10DAB80055F06EFCC7F8B850F8BD00BF0C40002008
:10DAC800C44000202DE9F347A44C06462368D3E957
:10DAD80001103EF054FDA5688146042D00F20E8227
:10DAE800DFE815F005002A013301CE010702731E95
:10DAF800042B15D8D4E900325B689A4200F0818083
:10DB0800012E0FD123686568986826698119284411
:10DB18003CF086FC761B00250746A846A5606BE10D
:10DB28000D2E11DC022E13DDF31E0A2B10D8DFE8B0
:10DB380013F068000F00C1010F000F006F000F0005
:10DB48000F000F0024005D001B2E5ED07F2E5FD0DB
:10DB5800A37D9A0740F19780092E00F08B80202E34
:10DB680040F0BF804FF000080321206884F8168039
:10DB78002F463EF05AFA03266DE079483CF06DFCDA
:10DB8800A0693CF06AFC2268636821699068C91A38
:10DB9800184401F0C9FB00252368D3E901103EF0C1
:10DBA800EEFC484503D203216E4801F0BDFB236813
:10DBB8002769D3F80880D3F80490781908EB09018D
:10DBC80040443CF02DFC0646A9EB070108EB070092
:10DBD80001F0AAFB236822695B689B1A5B1B981BF0
:10DBE800FFF7B2FE23692B44236145E05E483CF011
:10DBF80034FC20683EF0A2F963682E461844FFF70B
:10DC08003BFF304602B0BDE8F0870123A36033E054
:10DC18002669626896422FD92B462068B11AD0F837
:10DC280008C08B4203EB02071CD1042BB4BF0127A9
:10DC38000427F71B3B461CF80320194602F0C002D4
:10DC4800802A03F1FF33F6D0761A32467F1A4FF056
:10DC580001083EF0F1F9F01BFFF776FE23699B1BE4
:10DC68002361CCE01CF80770202F01D10133D8E7DD
:10DC78000127DEE70023A375A37D4FF0FF3623F0CD
:10DC88000203A375BDE7092E2BD123685A68C2B1D8
:10DC98009B682269134413F8010C04F091FD80B1CC
:10DCA8000426324B01930025019B21695A1C0192DD
:10DCB80029441A78206801353EF0ABF9B542F3D112
:10DCC8006AE7236860689D682169294A091A01ABD7
:10DCD800284408F0BBFF06460028CDD0431CE2D1FB
:10DCE8004EE71F2EC8DD06F0C0032068802B08BF52
:10DCF8008368276912BFF3B2DB5D217D03F140021F
:10DD080008BF0131D2B214BF0021C9B2372A97BF68
:10DD1800E5250025DB0803F0060398BF1D412175A2
:10DD28003246394498BF05F003053EF078F9237D63
:10DD3800AB42A1D101352FE74F2E04D05B2E40F026
:10DD4800DD80022362E7042360E7A6F13003092B94
:10DD580010D803236675A3608EE700BF1C3C002023
:10DD6800332A08083C2A08085A2A08088669080835
:10DD7800EC6507080023413EA360072E3FF67CAF01
:10DD880001A353F826F000BFB1DD010811DE010838
:10DD980051DE010875DE010881DC0108BDDE0108DD
:10DDA80081DC01080DDB0108E368062B3FF764AF4F
:10DDB800534D03F1010A2D3305EB8305AB68002BA6
:10DDC8003FF45AAF2668D4F80480B068216901444A
:10DDD80040443CF025FB07463046C6F80480A96855
:10DDE800C4F80CA03EF008F94FF0010822686368F7
:10DDF80026695568F61AED1A002E3FF72CAFB8F1D0
:10DE0800000F7FF4C9AE26E0E568002DFFF634AFB9
:10DE18002668D4F80480B0682169013D0144404473
:10DE28003CF0FEFA71680746A1EB08013046E56050
:10DE38003EF0FBF8E268002AD6DB314B206803EBA2
:10DE48008203D3F8B810CDE7236825695B689D4243
:10DE58002CBF00250125002D7FF70EAF236829462A
:10DE680098682369184401F05FFABBE62269636881
:10DE78009A427FF601AF00250126A8462F46EAE61A
:10DE88007E2E3BD1637D313B072B37D801A252F858
:10DE980023F000BF0DDB010805DF0108CBDE010818
:10DEA800BDDE010805DF010805DF01080DDB0108FB
:10DEB800BDDE010823685D682369ED1A0023A360AD
:10DEC800C9E7206821694368994217D20122856809
:10DED8005B1A0D4415F8016F06F0C006802E01D1BB
:10DEE8009A4204D13EF0A8F80023A36053E6013219
:10DEF800F0E7462EDED0482E3FF404AE002385E638
:10DF08000C4000202DE9F04F8BB068460A4BCDE954
:10DF180000451968CDE90267091A8908CDE904891D
:10DF2800CDE906ABCDF820C0CDF824D03FF09AFB60
:10DF38000BB0BDE8F08F00BF0C40002070B506782C
:10DF480004461EB14FF0FF35284670BD3CF0DFFC9B
:10DF5800C31E012B05460CD801210C48217001F085
:10DF6800E3F9032DEED10A48836E60309E600EF00F
:10DF780033F9A388013B9BB2A380002BE4D1012194
:10DF8800044801F0D1F96388A380DDE7402A080836
:10DF98000C4000205E2A08082DE9F0431D460023A6
:10DFA80097B0044603A81746049388460EF0FAF87B
:10DFB80007F001060346002877D1F90665D5D4E9AC
:10DFC8000121DC2040F073FD0446B8F1010FD4F8BC
:10DFD800009007D14FEA09114FF4397041F006015A
:10DFE80005F078FA2146424601A811F0DBF84946C7
:10DFF800C7F3800201A80DF01FFFB8F1010F044616
:10E0080001D1FFF753FC380602D4032000F0E6F9EB
:10E0180014B120463EF024FD4FF0FF3000F0DEF949
:10E02800012005F051F911F0DDFA1EB10121454832
:10E0380001F07AF90024FDB12C60ECB14FF0FF3308
:10E04800049FAB6038466F603EF07AFFA0B1694626
:10E05800384601AA3EF0A3FF019B6BB15A68AA603B
:10E06800002285F82C20186842F0F6F92022014693
:10E0780005F10C0055F0DCF91EB10121314801F021
:10E0880053F9204617B0BDE8F0837A0605D594E821
:10E098000E00DC2040F0C3FC96E7BB0695D5204671
:10E0A80042F0BAF940F011FD8EE74FF0FF3000F072
:10E0B80095F9022005F008F9790602D5A3682068C9
:10E0C80098471EB101211F4801F02EF9049C2046F3
:10E0D8000FF010F81C4913F01DFBF0B104983EF046
:10E0E80044FF0E2817D0C20705D4830708D1026859
:10E0F800164B9A4204D141F07EFB40F480749AE7B3
:10E108000146002212480FF011F8124910483EF05B
:10E11800B0FF0120F1E70020EFE70F4B9C420DD044
:10E1280004990B4840F017FE049B0C49186813F03B
:10E13800F1FA002814BF822401247CE74FF400641C
:10E1480079E700BF402A08082465070840600708E7
:10E15800EC650708C53208088440002000650708F8
:10E1680008B503784BB901210170044801F0DCF8C7
:10E178003CF0CDFB03380128FAD808BD402A08082E
:10E18800F0B58BB0202106A83DF088FE0025364862
:10E198003CF063F9079535483CF05FF93CF0B7FB74
:10E1A800431E032B43D8DFE803F002353F470799A6
:10E1B8000229ECD1089B1A78052AE8D15F78412F0B
:10E1C80005D02B4801F0B0F800230793E3E780243B
:10E1D8000126284801F0A8F803216846ADF8004058
:10E1E8008DF8026001F0A0F8002301AA0392224AE8
:10E1F80031460492214A03A805923A468DF8043024
:10E20800ADF80640ADF80840FFF7C6FEC305DBD5FC
:10E218000BB0F0BD1A483CF020F906A83DF060FEAE
:10E228000020184B1870F3E700230793B6E7C1B234
:10E2380006A83DF092FEB1E713483CF00EF9079BA3
:10E2480043B90F483CF009F906A83DF049FE4FF4E0
:10E258008070DDE700231122012106A8FFF79CFE4C
:10E2680010F4106F96D0D3E7422A08080C33080838
:10E27800F03F07085D2A080845DF010869E1010841
:10E288005A2A080885490020602A080870B598B0FD
:10E29800202101A83DF002FE474E48483CF0DDF839
:10E2A80047483CF0DAF845483CF0D7F8B28A0023F2
:10E2B80002B1B38205A8029306930DF073FF0446DA
:10E2C80088B9404901A83CF0B9F8012805462BD186
:10E2D8003A483CF0C2F801A83DF002FE20463A4B0D
:10E2E8001D7018B070BD022004F0EEFF33483CF0FA
:10E2F800B4F80699354840F02EFD029B002BD5D086
:10E3080001A83DF01BFE08F0E3FB58B10A2101A863
:10E318003DF023FE2E4901A83CF090F80328C2D016
:10E328000428EDD100212CE0851E032DE5D801A39A
:10E3380053F825F04DE30108AFE2010855E3010861
:10E3480067E301081D483CF088F8A6E71B483CF045
:10E3580084F801A83DF0C4FD4FF48070C1E71D4862
:10E368003CF07BF8002302933CF0D1FAC1B20329B8
:10E378008DF8031097D004290CD110483CF06DF8A3
:10E3880001210023162201A8FFF706FE10F4106FE2
:10E398008CD0A6E701A83DF0E0FD9DF803300D2BD9
:10E3A80003D10D483CF059F8DEE701210DF10300D7
:10E3B80000F0BAFFD8E700BF0C4000205A2A08082E
:10E3C800DB280808632A080885490020EC65070847
:10E3D8009F2A0808682A0808982A0808014B186024
:10E3E800704700BFDC060020024B986A003818BF4F
:10E3F800012070470C4000202DE9F04106460D46EB
:10E4080000270DB9BDE8F08133780A2B15D1A7B9DB
:10E4180001210D4800F088FF01243319A5429846D0
:10E4280004D013F8012B57B90A2A08D130462146DF
:10E4380000F07AFF46462D1BE3E70024EDE70D3A8E
:10E44800574257410134E9E7A42A0808024B034818
:10E4580019783EF0F2BB00BF86490020E451070856
:10E46800014B1878704700BF86490020014B18708F
:10E47800704700BF864900206FF013030B41DB078C
:10E4880010B502460C4615D50B490C483EF096FED1
:10E49800022C03D0052C0BD0094900E00949074894
:10E4A8003EF08CFEBDE81040074904483EF061BECE
:10E4B8000649F4E710BD00BFF4930808EC650708A7
:10E4C8001E910808D2900808C5320808DD9008088F
:10E4D8002DE9F04F99B000AF81460C46904600F008
:10E4E8003BFB28B9012528466437BD46BDE8F08FB7
:10E4F80001239F4A07F10801803042F092FF00286B
:10E50800F0D1D7E91002D7E906139A4208BF88422A
:10E5180000F02C8197F83930002B40F0278107F163
:10E5280008003CF00FF85B28064606D1D7E9062319
:10E5380007F1080043F0AFFBE3E7002EF6D009F13E
:10E54800FF3A1AF8015F2DBB304604F039F920B1C3
:10E5580007F108003BF0F6FF06463D2E1CD107F1F7
:10E5680008003BF0EFFF22280CBF0123002388F8A6
:10E57800003040F0CB8007F108003BF0D4FF2228A0
:10E5880029D016D828B30A2823D0C1B220463BF098
:10E59800F1FFF0E7B54206D00A2EB2D007F1080025
:10E5A8003BF0DFFFADE707F108003BF0BCFF064694
:10E5B800C7E75C28E9D107F108003BF0B4FF7628EB
:10E5C800E3D861281CD80A2803D0552854D000283D
:10E5D800DBD1052509E007F108003BF0B3FF0A2865
:10E5E80003D0232807D00028F3D1EDB207F10800A3
:10E5F80043F058FA77E707F108003BF0B2FFF4E779
:10E60800A0F16203142BC0D801A252F823F000BF76
:10E6180011E7010893E5010893E5010893E501086E
:10E628007DE6010893E5010893E5010893E50108F3
:10E6380093E5010893E5010893E5010893E50108CE
:10E6480071E6010893E5010893E5010893E50108DF
:10E658006DE6010893E5010875E60108F5E601088D
:10E6680079E601080D2090E70A208EE709208CE75B
:10E678000B208AE70C2088E74FF0080909F1080306
:10E6880023F007036E46ADEB030DEA46E8460DEBB3
:10E69800090B07F108003BF046FF08F8010BD845C5
:10E6A800F7D10023391D0AF809301022504632F0FC
:10E6B800E5FC7B680146434524D1B0F5881F1ED28E
:10E6C8007F2816D9B0F5006F15D3B0F5803F2CBF61
:10E6D80004230323227B22B16268134422689A42EE
:10E6E8000BD920463DF040FCB54644E74FF00409FD
:10E6F800C4E70123EEE70223ECE76360F4E70225B1
:10E70800B54672E7B54664E708203EE70A283FF4B5
:10E7180060AF00283FF45DAF00250D281CD00ADC4F
:10E72800092819D00A2812D088B1C1B220463BF076
:10E7380021FF002515E020280ED02328F5D1636895
:10E7480007F108005B1B63603BF00BFF02E06368A6
:10E758005B1B6360002548E7C1B220463BF00AFF17
:10E76800013507F108003BF0DEFED6E704253DE75A
:10E77800A62A080830B587B00D4610220DF1070308
:10E7880002A93BF002FF044648B99DF8073083B957
:10E79800094902A8F2F7BAFB20B901232B702046D9
:10E7A80007B030BD054902A8F2F7B0FB08B92C70D4
:10E7B800F5E70524F3E700BFB52A0808BA2A0808D0
:10E7C8002DE9F0418EB002AC0F46302221460DF102
:10E7D80003033BF0DAFE054628B99DF80380B8F13B
:10E7E800000F04D0052528460EB0BDE8F08120466C
:10E7F800F2F79EFB2618A6420CD99DF808302B2B61
:10E8080001D02D2B06D12D3BD3F1000848EB03088E
:10E818000DF10904311B022923DD2378692B15D159
:10E8280063786E2B1DD1A378662B1AD14FF0FF4366
:10E83800E01C0193B042D5D1DDED017AB8F1000FAB
:10E8480001D0F1EE677AC7ED007ACCE76E2B08D1DC
:10E858006378612B05D1A3786E2B02D1054BE01CA0
:10E86800E7E7204601AA04F077F90028BAD08442E5
:10E87800E0D1B7E70000C07F70B5054688B004A8AE
:10E888000C4620213DF00AFB28460DF1060204A99A
:10E89800FFF71EFE064630B99DF8063033B104A8CE
:10E8A80009F098FC2060304608B070BD28460DF18C
:10E8B8000701FFF75FFF38B99DF80730002B0CBF41
:10E8C8001E233E232360EEE7284602A93BF082FE82
:10E8D80018B9029840F052FFE4E7284603A9FFF769
:10E8E8006FFF88B9DDED037AF4EE677AF1EE10FA7E
:10E8F8007DBF17EE903A23F0030343F00203034B66
:10E9080078BFA3F1FF43DDE70526CCE7020040000E
:10E9180000B597B002460A236946044842F081FDD3
:10E92800684643F0BFF817B05DF804FB40140020B8
:10E9380010B5064C23783BB14FF47A72044B1A6039
:10E9480017F002FD0023237010BD00BF8749002087
:10E95800E0060020074B1A685AB11A68012A09BF55
:10E9680005491A680A704FF47A7218BF02F1FF322B
:10E978001A607047E0060020874900202DE9F04121
:10E988004FF00008514EADF5287D0746504C3046F3
:10E998000D46A6F8048017F0E5FC06F18000C4F8DF
:10E9A800048042F03AFD0D2802D127B91DB98BE049
:10E9B800002D00F087804FF4007300220093072198
:10E9C800444828AB14F0FAFE00287DD117F0BCFCAF
:10E9D8004149404814F00AFE002875D13F493D4896
:10E9E80043F02EFC00286FD13D48FFF791FF3D48CA
:10E9F800FFF78EFF3C48FFF78BFF3C48FFF788FF87
:10EA08003B49344843F01CFC3A4B03AA03F138074E
:10EA1800154618685968083303C5BB422A46F7D11A
:10EA28001B88354A2B80392302AD12A92B6029484F
:10EA38000A2342F0F6FC2B462A6803A912A842F0E2
:10EA4800C4FE12A843F02EF82C48FFF761FF2C4BA8
:10EA580003AA03F1100C174618685968083303C74E
:10EA680063453A46F7D1186899889B793860BB7135
:10EA78001623B980234A2B6012A90A23154842F0AD
:10EA8800D0FC03A92B462A6812A842F09EFE12A8C1
:10EA980043F008F81C490F4843F0D2FBA0B917F01F
:10EAA80053FC1A4B012523600023E360184BC4E98B
:10EAB8000156C3E93B443CF0D3FD28460DF5287DBB
:10EAC800BDE8F0810028ECD00020F7E7C013002053
:10EAD800383C0020401400206D370808C02A080878
:10EAE800CC2A0808DF2A0808F62A0808002B080894
:10EAF8000D2B0808332B0808112B0808A62A08082C
:10EB08006D2B0808252B08082E2B0808DC0C080894
:10EB18000C4000204FF47A7208B5044B1A6017F0C5
:10EB280013FCBDE8084013F0A5BA00BFE0060020BA
:10EB3800014601483BF0A7BDC0130020014601482B
:10EB48003BF0BFBDC0130020024B5868003818BF07
:10EB580001207047383C0020034B04485B68002BB9
:10EB680008BF0020704700BF383C0020C0130020B9
:10EB7800034B1B7813B903483BF0A5BE704700BF91
:10EB880088490020842B080810B10122024B1A7012
:10EB9800024800F023B900BF89490020483C002002
:10EBA800F8B5234B1E7826B1BDE8F8400120FFF7E1
:10EBB800EBBF204B20481E703CF096FE1E483CF0F0
:10EBC80079FE78B33BF058FE80F00105EDB21A48A3
:10EBD8003CF082FE80F00104E4B21DB1012000F097
:10EBE80047FB064604B3012000F04AFB07461348DA
:10EBF8003BF069FE12483BF066FEFEF76DFD1148DA
:10EC08003BF061FE10483BF05EFE10483BF05BFEB7
:10EC180015B1304600F02CFB44B13846BDE8F84049
:10EC280000F02EBB0125D2E72746E0E7F8BD00BF7C
:10EC38008849002089490020A00700208B2B08085C
:10EC4800902B0808952B0808992B0808882B08088A
:10EC5800044B1B7823B9044B1B780BB1FFF7A0BFFB
:10EC6800704700BF88490020894900200122014BD4
:10EC78001A707047884900200022024B02481A7017
:10EC880000F0ACB888490020483C0020034B044AF7
:10EC980004481A6000225A603CF020BE483C00201C
:10ECA80059EC0108A00700201FB50B4901A800F086
:10ECB8006DFE012101A83BF0C2FE01203CF033FFAC
:10ECC80001A83BF078FE044601A83BF069FE84F0F9
:10ECD8000100C0B204B010BD3CAD070808B5FFF78D
:10ECE800C5FB044B03F178029A62BDE8084013F0B3
:10ECF80037BB00BF0C4000200022014B1A60704750
:10ED0800583C00200122034B1A700022024B1A6063
:10ED1800704700BF8A490020583C00200022014B60
:10ED28001A7070478A490020024A13680343136027
:10ED3800704700BF5C3C0020024A136823EA0003C6
:10ED4800136070475C3C0020014B1878704700BF87
:10ED58008A49002038B50B4B1B7893B10A4B1B68C6
:10ED68007BB90A4C25683BF02EFD2060236813B957
:10ED780023680133236025B9BDE838400120FFF737
:10ED8800ADBF38BD8A4900205C3C0020583C0020BB
:10ED980010B50C4C206890B10B4B1B6883B93BF045
:10EDA80012FD236883422368A0EB030040F2EE23A0
:10EDB80088BF00F1FF30984294BF0020012010BDA9
:10EDC8000020FCE7583C00205C3C0020024B1868FF
:10EDD800003818BF01207047583C002010B5044681
:10EDE80002F062F9E3681BB90C4A1168A14203D129
:10EDF800BDE8104002F072B9A360094B1968E160E0
:10EE0800196809B119688C60116801B914601C602F
:10EE180002F064F913F0A4FA10BD00BF683C0020AA
:10EE2800643C00202DE9F041144E44F075FD336830
:10EE38000BB3134D02F038F92C681CB1BDE8F04152
:10EE480002F04CB901230F4A2B6033683460146018
:10EE58001BB92B68013B2B60F0E79F68C3E90244AC
:10EE6800D3E9006802F03AF90EB14046B04702F023
:10EE78001BF93B46ECE7BDE8F08100BF683C002089
:10EE8800603C0020643C00202DE9F7430025A8469B
:10EE9800144E019502F008F9346801AF54B9019B8A
:10EEA8003360114B1D60114B1C6003B0BDE8F0438B
:10EEB80002F014B9D4F808902046C4F808800BF082
:10EEC8001BF918B10023E3604C46E7E760680BF0D4
:10EED80013F90028F6D12B463C60254604F10807B3
:10EEE800F1E700BF683C0020643C0020603C002043
:10EEF80010B5044B1C6804B910BD60683EF0E6FB11
:10EF0800A468F8E7683C0020014B1878704700BFF8
:10EF18008B490020014B1870704700BF8B490020B7
:10EF28002DE9F34113F000FA3E4B074620F47F0029
:10EF380020F47F4098423C4D0BD117F47F4FC7F324
:10EF4800072406D013F0EAF92C70204602B0BDE879
:10EF5800F08100232B703BF043FA072803D8A22343
:10EF6800C340DB0735D4314813F0D8F900F0B0F9C5
:10EF78004FF07E532E4801A901933BF071FBDDED64
:10EF8800017AF5EEC07AF1EE10FA24DB9FED297ACA
:10EF9800F4EEC77AF1EE10FA1DD89FED277A67EEE6
:10EFA800877AFCEEE77A17EE905A3BF0FDFB0024D7
:10EFB8000646884620462146A84271F100030DD333
:10EFC800002000F06BF900F063F94CBB384613F0F1
:10EFD800A5F90024B9E74FF47A75E6E7ACB9FA2247
:10EFE8000023F1F739FF7D2A73F100030DD3204682
:10EFF80000F054F9FFF758FE044658B13BF0D4FB33
:10F008004FF47A750646884604E00C4800F046F945
:10F01800002CEFD03BF0C8FB801B61EB0801CBE76D
:10F02800112492E7AF0000AD8B490020AF1100AD6D
:10F03800A02B08080000804F00007A440030300000
:10F04800024B43EA002013F069B900BFAF0000ADDE
:10F058000D4D08B52B780446012B0FD901280DD981
:10F068000A4836F04AFB2146094836F046FB29781B
:10F07800084836F042FB37F044F9FCE72046FFF732
:10F08800DFFF41F044FA00BF8B490020BA2B080883
:10F09800D02B0808DC2B080810B50446002838D007
:10F0A8001C4800F0AFF9631E112B12D8DFE803F0FB
:10F0B8002D1111111111112B11291111272125239E
:10F0C800091F154800F09EF9BDE81040134800F0EC
:10F0D80099B9023C1248E4B200F094F90A2C16D807
:10F0E800104B53F8240000F08DF90F48EAE70F4859
:10F0F800E8E70F48E6E70F48E4E70F48E2E70F487C
:10F10800E0E70F48DEE70F48DCE70F48DAE70F488B
:10F11800E9E710BD738B0808FD8B0808888B080881
:10F12800D3920808004B0708988B08080D91080827
:10F138008C930808078D08081C8D08081C8E080881
:10F14800EB8D080833930808F28E0808BB8C080872
:10F1580008B544F0DEFB3BF016FB00F06BFCFFF754
:10F16800E7FB44F0D8FB3BF00EFB002041F0D5F95B
:10F17800034BC3E90001BDE8084044F0CBBB00BF26
:10F188005034002008B5FFF7E5FBBDE80840002231
:10F19800014902483BF0E8BA59F10108703C0020E7
:10F1A80010B5074C01F080FF23680BB913F0FAF88B
:10F1B800236801332360BDE8104001F08FBF00BF12
:10F1C8006C3C002008B501F06FFF074B1A6812B1BC
:10F1D8001A68013A1A601B680BB913F0F1F8BDE818
:10F1E800084001F07BBF00BF6C3C0020034B18684F
:10F1F800034B002808BF1846704700BF803C00201A
:10F208007185214910B5054C23782BB93BF024FBB7
:10F2180041F0A6F90123237010BD00BF8C490020DE
:10F2280073B505460C46C1B10E4B1B78C3B90A46E7
:10F2380001AB01460C4802F07BFA06460B4B1B78E3
:10F2480053B902F03DFC40B1214628463BF00CFB87
:10F258002146284613F05AFA3446204602B070BDBB
:10F268000E46EBE78D4900206C0800208E490020EF
:10F27800024B1A7818701046704700BF8E4900205C
:10F28800024B1A7818701046704700BF8D4900204D
:10F2980001483BF085BB00BF883C002038B5094DCC
:10F2A80004462B6883420CD0074B19783BF015FBBA
:10F2B8002C60011E18BF0121BDE83840034800F04A
:10F2C80081BB38BD843C0020580C0020883C0020BD
:10F2D80070B50B4C257895B901260A490A4826705D
:10F2E80000F054FB2A46314607483BF081FB4FF0BB
:10F2F8008072064B18681A60FFF7D0FF257070BD42
:10F308008F49002004AF0708883C0020843C002077
:10F31800014B1870704700BF580C0020014B18783B
:10F32800704700BF580C00202DE9F843DFF88080B3
:10F3380000AF05460E463BF0E9FAD8F8003043B373
:10F348001A483BF0FDFAC0F500720446D8F80000F0
:10F3580043689919914223D90734D21A294624F0CF
:10F3680007043CF072FDE946ADEB040D69460F4811
:10F37800D8F8004000F050F8014620463CF03CFE2A
:10F388000A21D8F800003CF0E8FD0023C8F8003056
:10F39800CD4631462846FFF743FFBD46BDE8F88312
:10F3A800324629463CF051FDF3E700BFEF8B0808D1
:10F3B800DC3B0020A1F18003612B70B5064619D80B
:10F3C800194602230D480E4C10F8012B914205DA1C
:10F3D80003FB0144E518A54206D870BD891A12FB43
:10F3E80003F201331444EFE7304614F8011BFFF72A
:10F3F800E1FFF0E7BDE870403CF0B6BD736B08086C
:10F408007D6B08080246024902483DF0B2BE00BFC3
:10F41800F32B0808645A07082DE9FF4105468024A4
:10F428000A4615F8011B684601313CF052FD009E62
:10F43800234FDFF89080013E019B9E4205D8684625
:10F448003CF07CFD04B0BDE8F08100239C461946E1
:10F458001A46287852002040003818BF0120640856
:10F4680042EA000204BF8024013501316245C9B275
:10F4780004D3785C00EB4C0C0344EAE7A3EB0C03E1
:10F488004244D15C012916D10B2200202B78400080
:10F498002340003B18BF0123640804BF80240135C2
:10F4A800013A40EA0300F1D140F0D6FF0146684630
:10F4B8003CF0A2FDC0E76846FFF77CFFBCE700BF51
:10F4C800186E0808606D080808B5024836F015F986
:10F4D800002008BDF62B080838B5FFF73DFB0446A9
:10F4E80020B90D4836F009F9022038BD3BF0DEF8A6
:10F4F80020B90A4836F001F90420F6E7084D2B78C0
:10F508002BB920463BF00AF908B90648F2E701236F
:10F5180000202B70E9E700BF092C08081B2C0808FD
:10F52800924900202E2C0808F8B514460E461F46AE
:10F53800FFF712FB05460420FFF7F6FB3B46224681
:10F548003146284643F00CF9D5F8CC30A34207D110
:10F5580034B14FF40072314605F5807053F00BFF5B
:10F56800D5F8BC300020A3429EBF0122014B1A707F
:10F57800F8BD00BF9149002038B50C461546FFF785
:10F58800EBFA022C03D0052C07D0012C15D12A4602
:10F59800214614F0E9FE002038BD2A4600210A4C15
:10F5A80014F0E2FE0420FFF7C7FB2378002BF2D00B
:10F5B800FFF7D0FB00232370EDE70448214636F01F
:10F5C8009CF86FF08500E7E7914900203E2C080879
:10F5D80070B505460C4636F090FFD8B1237853B97C
:10F5E800144A28461370F5F7ABF820B10121124AE6
:10F5F800124836F0D1FC2678012E0BD100220D4B93
:10F6080028461A70F5F7FEF820B10D4A31460B4826
:10F6180036F0C2FC2378052B06D16368054A003B07
:10F6280018BF0123137070BD042B02BF0022014BC9
:10F638001A70F8E7904900205B2C08086C3E070810
:10F648007B2C080813B5964836F057F8954836F0DD
:10F6580054F89549954836F0B1FF034638B1944AB5
:10F668000121944802B0BDE8104036F09EBC924992
:10F678008E4836F0A3FF034608B1904AF0E7904958
:10F688008A4836F09BFF034608B18E4AE8E702F045
:10F6980017FA98B90E2002F093FA02F017FAD8B9BF
:10F6A8000E2002F09BFA8848F3F7FEFE014608B3E5
:10F6B800864802B0BDE8104036F01FB8012180200E
:10F6C80012F052FF03460028E4D080228049814886
:10F6D80002F0E0F97F48DEE70121802012F044FFC4
:10F6E80003460028DCD080227B497C4802F0D2F90E
:10F6F8007A48D6E76D4836F0C0FE0128044650D156
:10F70800774835F0FAFF2146764A6848F6F7A0F9B7
:10F7180038B1754A0121674802B0BDE8104036F09B
:10F728003BBC724835F0E9FF02F0CAF948B17049AC
:10F73800234622465D48F6F7ABFA014608B16D4804
:10F74800B7E702F0C3F940B101236B491A4657489D
:10F75800F6F79EFA01460028F1D1012367491A46B7
:10F768005248F6F795FA014608B16548A1E7654899
:10F7780035F0C3FF02F070FA60B1634835F0BDFFA1
:10F78800012362491A464948F6F782FA014608B148
:10F798005F488EE701210223EF224448009136F0AA
:10F7A80073FE5C4835F0A9FF00215B4A3F48F6F735
:10F7B8004FF9044608B1594AACE702F081F978B12B
:10F7C800574835F09AFF0123224649493748F6F74A
:10F7D8005FFA28B1534802B0BDE8104035F08DBF3C
:10F7E80002F074F950B14E4835F087FF012300222A
:10F7F80041492E48F6F74CFA0028EBD101230022A4
:10F808003E492A48F6F744FA044608B10146ACE7EF
:10F8180002F022FA60B1444835F06FFF3B490123FA
:10F8280022462248F6F734FA014608B13F4840E735
:10F8380001240223EF2200211C48009436F024FE04
:10F848003B4835F05AFF0021184836F041FE394848
:10F8580035F053FF3849154837F07CF908B1374A75
:10F8680058E7374835F049FF02F022FB354835F0B4
:10F8780044FF0E48F4F724FF034608B1324AEFE686
:10F88800324835F03AFF094836F037FE30B90748B4
:10F89800F4F756FF034608B12D4AE1E602B010BD61
:10F8A8009C2C0808AE2C080884070020841200202D
:10F8B800CA2C08086C3E07086C070020F82C0808BA
:10F8C800540700202A2D0808E4060020572D0808B0
:10F8D800AC3B0708A8340020903B070858340020A8
:10F8E8007A2D0808FC0600209B2D0808C22D080860
:10F8F800251B0808E82D0808051B0808941B08089C
:10F908000B2E0808302E0808552E0808061D080872
:10F91800772E08089D2E080810070020BE2E08081C
:10F92800E52E08080B2F08082B2F08084D2F08086C
:10F93800732F0808892F0808D9F501089F2F080890
:10F94800C32F0808D52F0808E02F08080930080831
:10F958001A30080808B5064B1B7803F0FF002BB1D6
:10F96800044836F0C5FD80F00100C0B208BD00BFF4
:10F97800904900208412002008B502F0A1F8002860
:10F98800014808BF002008BDA834002038B50C463F
:10F99800054608463AF021FD6C6060683AF002F8C6
:10F9A80020B9074835F0A9FE012038BD4FF4803250
:10F9B800217A60683AF0E3FF0028F5D12872F4E76D
:10F9C8006530080838B5436804460D4658681A7A01
:10F9D800012303FA02F1036982681B680B40003BAC
:10F9E80018BF0123AB4214BFD36813699847014677
:10F9F80010B1024835F081FE657238BD7C300808C8
:10FA080038B543680129094A04460D4618BF4FF422
:10FA18000032197A58683AF0B2FF014620B104481A
:10FA280035F06BFE012038BDA572FCE70600020028
:10FA38009430080808B5FEF7D7FC10B9FFF7A8F905
:10FA480070B108BD0D4A934203D1BDE808403BF0B0
:10FA5800FEBB0B4A9342F4D1BDE8084000F066BDF6
:10FA680008480368002BECD0074A9342E9D0074ABC
:10FA78009342E7D1BDE8084044F0DEBA7C4E07085F
:10FA8800544C0708F8340020B8560708C8BC0708C3
:10FA98004FF0FF3370B5204E204C336023682BB9EC
:10FAA8003368E3B9BDE8704016F0E2BD1C4DAB42C7
:10FAB800F6D01C4A934204D1204644F0D6FA256079
:10FAC800EEE7194A934203D1204600F05FFDF6E7BE
:10FAD800164A9342F3D1204601F0C4F8EFE7144CDC
:10FAE8002368002BDED00E4DAB42DBD0114A934287
:10FAF80004D120463BF087F82560D3E70E4A9342AD
:10FB080003D1204601F02CFAF6E70C4A9342F3D1D0
:10FB1800204601F035FDEFE79C070020F83400206F
:10FB2800B8560708C8BC0708544C07087C4E070895
:10FB3800943C0020F44D0708F84F07089C5107082B
:10FB4800F8B5334C334E23680BB1B3420DD1266060
:10FB580031480368002B59D0B34257D02F4A9342FB
:10FB680046D1BDE8F84018F069B92D4A934216D13C
:10FB78006568A54203D304F198039D42E8D9284655
:10FB88000AF0BAFA0028E3D0264B6C222946184618
:10FB980053F0F1FB6060284644F0C8FBD8E7224ADE
:10FBA80093421ED16568A54203D304F198039D4290
:10FBB800CED928460AF0A0FA0028C9D0194A2B46FF
:10FBC800944605F1200E174618685968083303C78C
:10FBD80073453A46F7D12846C4F804C044F00BFBF5
:10FBE800B6E7124A9342B3D120463BF0BBFDAFE7DC
:10FBF8000F4A934203D1BDE8F84000F0F3BC0D4A28
:10FC0800934203D1BDE8F84001F03EB8F8BD00BF0B
:10FC1800943C0020B8560708F8340020C8BC0708F0
:10FC2800F44D07089C3C0020F84F07089C51070832
:10FC3800544C07087C4E070808B5144803681BB9DC
:10FC4800134803684BB908BD124A9342F8D0124AC8
:10FC58009342F5D13BF017FEF2E70E4A9342F2D0F9
:10FC68000E4A934203D1BDE8084044F00DBA0C4A4D
:10FC7800934203D1BDE808403BF002BB094A9342D6
:10FC8800E1D1BDE808403AF054BF00BF943C0020E1
:10FC9800F8340020B85607089C510708C8BC070864
:10FCA8007C4E0708544C070810B5084B084C1B68D5
:10FCB800A34200D043B9B4220021064853F081FB87
:10FCC800044840F8044D10BD0020FCE7F83400203B
:10FCD800B8560708FC34002008B5FFF7E5FF10B94F
:10FCE800014803F019FD08BD528D080810B5084BEE
:10FCF800084C1B680BB1A34208D194220021064886
:10FD080053F05FFB044840F8044D10BD0020FCE7A9
:10FD1800943C0020B8560708983C002008B5FFF727
:10FD2800E5FF10B9014803F0F7FC08BD588D080835
:10FD3800094B1B685A1C0DD0002B0BDCB82253430F
:10FD4800064A9818D358064A934203D0002B08BF96
:10FD58000E2070470E2070479C070020F8340020C2
:10FD6800B85607080E2807B506D14FF0FF330D4ADD
:10FD7800136003B05DF804FB0B4B98421A6803D17B
:10FD88000A4B9A4200D05AB90DF0B4F9C388E92257
:10FD980000934FF48D7140F26113054803F0F8FCAD
:10FDA8000023E4E79C070020F8340020B856070831
:10FDB8005C950808074A1368013304D1064B0749C4
:10FDC8001B688B4200D17047002BFCD000231360C6
:10FDD800704700BF9C070020F8340020B856070879
:10FDE8002DE9F04F04464FF0000887B0CDE9031223
:10FDF800059300F15009059B984502D307B0BDE86B
:10FE0800F08F049B03EB080694F8B530757896F9E3
:10FE180001B0002B35D0B57806F1030A484619F031
:10FE280029F998B3012300930021334694F8B620AA
:10FE3800206D276EB84700955346012194F8B620E7
:10FE4800206D276EB847484645F07FF8BBF1000F94
:10FE580023DB00203BF067FE039B3BB1D4F88430E2
:10FE6800164A934202D020463AF0F2FDFEF7BCFA59
:10FE78000028C3D194F8B5304544DBB905F1020830
:10FE8800B9E706F1020A05F07F05C7E7FEF7ACFA05
:10FE98000028C7D1FEF7C6FFC0E76B1C94F8B52051
:10FEA800DDB256FA83F313445878FF2808BF4FF49D
:10FEB800FA70CFE705F103089DE700BFB8560708B9
:10FEC800F0B54B6B05460C468BB0002B00F0D0808C
:10FED800012380F84030486B44F081FD85F83C00F0
:10FEE800636B002B00F0C780A36B002B00F0C3806E
:10FEF8004FF48073A5F84030A06B44F070FD85F88E
:10FF08003D00B4F85630002B14BF0123002385F8B8
:10FF1800B43094F8573018BF002685F8423094F86A
:10FF2800563018BF042185F8433008BF0123626B9F
:10FF38000ABF1946334694F855600AB9A26B32B124
:10FF4800228EB2F5807F02BF0026022133460122AD
:10FF58000027CDE90422CDE90222CDE9001305F1FD
:10FF68000800638C228BE18A44F008FC94F859302D
:10FF78000897099394F8543005F15000CDE90673B9
:10FF8800638D0593238D0493E38C0393A38C0293D1
:10FF9800B4F920300193B4F91E300093A38B628B1F
:10FFA800216818F0DFFFA38D9FED357AA5F8AA30F8
:10FFB80094F82E3085F8B030238EA5F8AC3094F83C
:10FFC800323085F8B130D4ED117A67EE877AFCEEDD
:10FFD800E77A17EE903AA5F8A83094F84C3085F8EF
:10FFE800B27085F8AF30D4ED147A67EE877AFCEEFC
:08FFF800E77AC5ED247A94F8C4
:020000040802F0
:10000000543085F8B36085F8B6306368C5F894302D
:100010002389A5F8A030D4ED037A67EE877AFCEE49
:10002000E77A17EE903AA5F8A6302369C5F898301C
:10003000A38AA5F8A230E36BC5F89C30B4F8403031
:10004000A5F8A430114BC5F8843094F8583085F8E1
:10005000B530A36C4BB128460D4B40F8843FA16CE2
:10006000FFF798FCA06C3AF0BAF9284609490BB0A2
:10007000BDE8F0403AF035BD80F8403034E7002369
:1000800085F8413041E700BF00007A44B8560708C0
:100090009CC10708780A0020DFED077A20EE270AC6
:1000A000BCEEC00A0B68C0F894304B6880ED240A9F
:1000B000A0F8A030704700BF00007A4410B5038F4D
:1000C00004465A2B28D0A3F5877CDCF1000343EBD0
:1000D0000C035A291ED0A1F5877042424241934237
:1000E0001FBFA38EE28EE386A28604F1080044F0CF
:1000F00008FB0C4B9C4205D116F0BEFAE18EA08E97
:1001000016F05CF9A06858B104F11801BDE8104080
:1001100045F0D8BA0122E2E75A29E6D00123DAE70E
:1001200010BD00BFF83400202DE9F04F97B090F8D3
:10013000B230044602AFE3B1D0F88420B24B9A4209
:1001400017D184303AF03BFC94F8AF30834204D1AD
:1001500000205437BD46BDE8F08FFFF737F8002187
:100160002046B4F8A230D4F8982084F8B210FFF7F3
:100170003BFEA368002B00F0C28120463AF0BAFC97
:100180000028E5D104F1500A504644F0DBFE002877
:10019000DED094F84810002900F09C8000232363EF
:1001A00004F12803FB6294F8B430002B40F0A380E4
:1001B000FEF71EF938610028CAD120463AF05EFCED
:1001C00004F1080B5846F96A07F13802C7F808D05D
:1001D00044F076FB002800F0878107F1380045F0F5
:1001E000F3F9202594F83A30064607F13800B5FBBC
:1001F000F3F545F0EEF9814607F1380045F0E9F9ED
:10020000B0EBC51F4FEAC51800F2CC800123FB619B
:1002100080231FFA89F09B00BB614009073323F05C
:1002200007030130ADEB030D78637B6B0DF108081C
:100230009B00073323F00703ADEB030D02ABBB625A
:10024000B4F8AC30B3F5807F14BF022301237B6088
:10025000BB694344FB6000237B6207F1380045F033
:10026000B3F9B4F87A303862B3F5807F05D05946D7
:10027000504607F1380244F06FFEB4F8AA3087F810
:1002800033307B6A1BB1B4F8AC3087F8333050465A
:1002900018F0F4FE002800F02781012394F8B6201E
:1002A0000093002107F13303206D256EA8475046C7
:1002B00044F04FFE002399467B61BB8AFA69934262
:1002C000C0F0A48001227B6A7A627A6801339A4284
:1002D000C3D809E1A068002800F0118145F0E7FAD1
:1002E000F862002800F00B81B4F87A30B3F5807F13
:1002F0007FF459AF52E7204604F108063AF0BEFBFE
:100300003046C7F828D044F0A0FA0546304644F0FD
:100310009EFAC5F34F05EB1D23F00703ADEB030D6C
:100320000DF108092A4677218046484653F04DF8DA
:10033000B4F8AA30504687F8443018F09FFE834640
:1003400088B12046D7F828D03AF0B7FB94F8B230FD
:10035000002B3FF42DAFFEF74BF800287FF428AFB9
:10036000FEF764FDF2E70123014694F8B6200093FE
:10037000266E07F14403206DB047504644F0E9FD76
:100380001FFA8BF39845DCD9504618F077FE0BF135
:10039000010B0028D5D094F8B62000954B460121DA
:1003A000266EE8E707F1380045F009F9B8FBF0F8E8
:1003B000464607F13800012EB8BF012645F004F982
:1003C000B0FBF6F083B207F13800FB6145F0FCF8B2
:1003D000B0FBF6F303FB160080B218B1FB690133E2
:1003E0009BB2FB6107F1380045F0E9F816FB00F01D
:1003F00080B2B0FBF5F293B205FB1202002A3FF483
:100400000AAF01339BB206E79CC107083B69386A13
:100410007A8FFB643B8F8642A7F8443002EB0903D6
:1004200088BF3A6A9BB298BF9219A7F8463095BF29
:100430004A449B1893B29BB2A7F84A303B6AB7F97B
:100440003C109B1B9BB207F14400A7F848103B628D
:1004500045F0BFF8082294F83A300021B2FBF3F3DC
:10046000B0FBF3F37A6BB86A92001D4652F0ADFF11
:1004700000214046BA6952F0A8FF94F8B43013B98D
:1004800040F20713E3877B6AD3B194F8B33063B1CA
:10049000062384F83E3043465846BA6A07F14401C1
:1004A00044F001FA94F8B13013E094F8402012B10E
:1004B00084F83F30EFE7B4F84230002BF2D0EAE79F
:1004C00043465846BA6A07F1440144F0ECF994F8FF
:1004D000B030B3B9504618F0D1FD7B69B144013357
:1004E0007B611FFA89F9A8B9FB6AD7F808D09B6825
:1004F000FB62002B7FF464AE20463AF0DEFA012066
:1005000027E64346FA689A42E4D01A68D24343F891
:10051000042BF7E7ABB294F8B620009301214346D1
:10052000206D256EA847504644F013FDFEF77EFC73
:10053000C3E600BF10B590F8B23004463BB3D0F824
:100540008420134B9A4214D184303AF038FA94F84C
:10055000AF3083421BD0FEF739FE002184F8B21081
:100560002046B4F8A230D4F89820BDE81040FFF738
:100570003BBC3AF01DF9D4E90432C01AB4F8A830F3
:1005800061EB020183424FF000038B41E3D310BDC6
:100590009CC1070810B590F8B230044693B1D0F86A
:1005A0008420104B9A4201D03AF056FAFEF70EFE24
:1005B00000212046B4F8A230D4F8982084F8B21074
:1005C000FFF712FC04F1080044F061F9D4F884202C
:1005D000054B9A4205D104F18400BDE810403AF081
:1005E000E3B910BDB85607089CC1070810B5044907
:1005F0000446083044F0FBF8012384F8483010BD6D
:10060000780A002010B50B4C0B4B22689A420ED191
:10061000A2680A4B9A420AD120463AF06BFA28B9EE
:100620002046FFF781FD80F00100C0B210BD002020
:10063000FCE700BFF8340020544C0708780A00207B
:1006400008B5014803F064F82494080810B504497B
:100650003FF0C4FE044611F043F8204610BD00BF31
:10066000544C0708F0B50C4689B0064654F8040B04
:100670001746FFF7EBFF054603AB01930B4B3A46DA
:1006800021460093701E022306F0FAFE052205A9FA
:1006900003980DF0D5F804980CF0E0FE284605A963
:1006A000FFF7FAFC0E2009B0F0BD00BF444C07086C
:1006B00008B5FFF7CBFFFFF737FD10B9024803F08D
:1006C0002FF80E2008BD00BF8F8E080808B5FFF771
:1006D000BDFF3AF00FFAD0B16430EFF7D7FE0D4B03
:1006E0000022F0F777F8F0F70DFA07EE900AF4EE33
:1006F000677AF1EE10FA7DBF17EE903A23F003000F
:1007000040F00200044878BFA0F1FF4008BD034854
:10071000FCE700BF00408F400200400002008080E4
:100720002DE9F04F2DED048BC9B0084611461A464D
:1007300028AB01936E4B08AF009320233CF05EFC86
:10074000289B05223946299802930DF079F8052255
:100750000BA92A980DF074F840F246313E983AF011
:10076000CFFE5A22319E824696FBF2F302FB1363C0
:1007700013B1604802F0B6FFFFF7B2FA04463D98A5
:100780000CF06CFE4098F0EE408A0CF067FE469844
:10079000B0EE408A0CF062FE3A9B389803933B9B84
:1007A0000E28B0EE409A049300F091803EF0DAFA01
:1007B0000546DDF8F0B00DF11C09494658469DF894
:1007C00014810CF0C9FD002800F0848003203FF064
:1007D0008BF8079A03460270002208F10209427062
:1007E0008270454A002122600DF14E00522205938D
:1007F00052F0EBFD3A68029B12927A681193ADF8C1
:100800004C200B9A8DED149A15920C9AADF86660F7
:10081000ADF858202B9A2046ADF85A202C9A11A9F1
:10082000ADF85C202D9AADF85E202E9AADF86020D0
:100830002F9AADF86220309AADF86420329AADF864
:100840006820339AADF86A20349AADF86C20359A56
:10085000ADF86E20369A039BADF870201E93049B72
:100860009DF8DC201F93059B8DF8722020939DF846
:10087000FC309DF8E4208DF890309DF80431CDEDEA
:10088000228A8DF898309DF808318DED258A8DF8F3
:1008900099309DF80C31ADF874508DF89A309DF870
:1008A00010318DF876208DF89B309DF81C31ADF815
:1008B0008490CDF88CA08DF89C808DF89D30FFF74A
:1008C00003FB204649B0BDEC048BBDE8F08F4FF42C
:1008D00080756EE7012258460EA90CF0B1FF10B1E9
:1008E000DDE90E397DE740F20251044802F040FF95
:1008F000444B070868920808544C0708F190080810
:1009000070B58AB004AB01931B4B0C4600930431C5
:100910000323013806F0B4FDFF22002140F26733C3
:10092000049806F049FE05228DF80F0007A90598E6
:1009300024680CF085FF20463AF024FAC0B1012566
:100940009DF81860204632460DF10F0300210095F6
:100950003AF038FA089B3246294620460093079B16
:100960003AF030FA20463AF0ACFA0E200AB070BDE8
:10097000FEF75CFADFE700BFDC4D070870B58CB00E
:10098000084611461A4605AB0193184B00930723FE
:100990003CF034FB40F277521549059806F08AFE88
:1009A0000646FFF7BFF9134B04460360012240F2ED
:1009B000DC4300210A9806F0FFFD40F2D1430546D2
:1009C000012200210B9806F0F7FD099BC0B20193AC
:1009D000089BEDB2039000932046DDE906233146E3
:1009E00002953AF05DF920460CB070BDA44D0708A1
:1009F000A0C00708F44D070808B53AF035F920B94A
:100A000040F21451024802F093FE0E2008BD00BFD0
:100A1000FE8F080810B5038F04465A2B28D0A3F583
:100A2000877CDCF1000343EB0C035A291ED0A1F5AF
:100A300087704242424193421FBFA38EE28EE386FB
:100A4000A28604F1080043F05CFE0C4B9C4205D1E9
:100A500015F012FEE18EA08E15F0B0FCA06858B122
:100A600004F11801BDE8104044F02CBE0122E2E779
:100A70005A29E6D00123DAE710BD00BFF834002080
:100A8000F8B590F8783004460D46174643B1002378
:100A9000204684F879303AF024FA01263046F8BD31
:100AA00090F87960002EF2D14B1CF0D039F080FE26
:100AB0002369C31ABB4202D90D4802F031FEA26E6F
:100AC000C4E91A01821A9542E8D3B3FBF5F205FB9B
:100AD0001233ED1A39F06CFED4E91A32C01A61EB08
:100AE0000201A84271F10001D1D2FEF79FF9F1E7AE
:100AF000AE9308082DE9F04F1F4600238BB0044643
:100B000080F87830016540F2E74090460BF034FB06
:100B10006065C369002B00F09080206D984786B215
:100B2000636D206D1B69984783B20793636D206DD9
:100B30005B69984783B20893636D04F1080B5B6AA5
:100B4000002B7CD0206D98478146636DDD6A15B11E
:100B5000206DA8470546636D9B69002B76D0206DFC
:100B600098475FFA80FA636D1B6B13B1206D98474D
:100B70000346626D526B22B1206D09939047024685
:100B8000099BCDE90432DDE9071200235846CDE97F
:100B9000025ACDE9006943F0F5FD636D1B6A13B19C
:100BA000206D984783B2A4F87430636D9B6B002B63
:100BB0004FD1A38E94F83A205343DB10A4F876303B
:100BC000636D206D5B6804F158019847E28EB4F8BC
:100BD0007610B4F87430013A01FB023394F83A20ED
:100BE000A18EE06D51434FF47E7203EBD10106F00C
:100BF0002DFD87F0010384F87930636D9B6A83B320
:100C0000206D984780B24FF47A73B3FBF0F3A4F8E9
:100C10007000A4F87230B8F1000F03D041462046AE
:100C2000FFF7F8FE5846104943F0E1FD39462046EB
:100C30000BB0BDE8F04F3AF0FABA102670E7072E75
:100C40008CBF4FF000094FF001097EE74FF0020A18
:100C500089E7206D984780B2A4F876000028AFD1CC
:100C6000A7E73C20CFE700BF780A002010B5044674
:100C700000213AF0DCFA04F1080043F008FE636D4D
:100C8000206DDB689847014B236010BDB8560708FC
:100C900010B50446006D0CF031FA78B10A4B984259
:100CA0000CD0012120463AF0C2FA084904F10800AC
:100CB00043F09DFD012384F8483010BD2046BDE877
:100CC0001040FFF7D3BF00BFB8560708780A0020CE
:100CD00008B5083043F08BFD10B9024802F002FD60
:100CE0000E2008BD8891080808B5014802F010FDE3
:100CF0002494080810B504493FF070FB044610F036
:100D0000EFFC204610BD00BF7C4E070830B50C46F6
:100D100085B002AB0193154B0431009301380223D7
:100D200006F0AEFB2068FFF7E5FF039B0546002BAE
:100D3000C8BF4FF47A740298CCBF94FBF3F44FF021
:100D4000FF340E280FD03EF00DF84FF47A7191FB6E
:100D5000F0F122462846FFF793FE00280CBF1E2024
:100D60003E2005B030BD4FF0FF31F2E76C4E070872
:100D700008B5FFF7BFFF3AF041FAB5EEC00AF1EE51
:100D800010FA02D5094802F0CBFCB4EE400AF1EEAD
:100D900010FA7DBF10EE103A23F0030040F002007D
:100DA000034878BFA0F1FF4008BD00BF7F9308084B
:100DB0000200400038B50C46FFF79CFF0E2C05469C
:100DC0000AD0204619F0E0FD01462846FFF780FFD3
:100DD00020B9034802F086FC0021F6E70E2038BD5A
:100DE0008891080870B586B0084611461A4603ABCC
:100DF00001930F4B009303233CF000F9DDE90365F9
:100E00005A2295FBF2F302FB135313B1094802F087
:100E100069FCFEF765FF0446074B314603609DF809
:100E20001430AAB2FFF766FE204606B070BD00BFC0
:100E3000444E0708689208087C4E070838B50D46EE
:100E4000FFF758FF044628460CF008FBB5EEC00A31
:100E5000F1EE10FA06D4B7EE007AB4EEC70AF1EE5E
:100E600010FA06DD0123002240F23E31054802F06F
:100E70007FFC20463AF0CAF910B9034802F050FC52
:100E80000E2038BD8B9508087F9308082DE9F043A4
:100E90000C468DB002AF07F1080301932E4B0431CD
:100EA00000930138022306F0EBFA2068FFF722FFD7
:100EB000D7E9028605460622304607F110010CF0FC
:100EC000BFFCBB69012B02D0244802F00BFC95F853
:100ED0003A30102B01D02248F7E70024B5F83490BF
:100EE000FC6107F11C00A7F81E8008F101087C6274
:100EF000A7F82090A7F8228044F06BFB00F00102D5
:100F000081B2786902EB5902B0EB820F3B6920D3C2
:100F10004A09A446214601327A607A689200073273
:100F200022F00702ADEB020D02AA7C6888B284426F
:100F300001F101010AD807F11C0105F1080043F095
:100F4000B2FC30462C37BD46BDE8F08342F820C0E5
:100F5000EBE70448B9E700BF5C4E07087493080844
:100F60007B9208085E93080810B50446406804F1B7
:100F70000803984201D143F041F90023A26A63605B
:100F8000044B9A4205D104F12800BDE8104039F025
:100F90000BBD10BD9CC1070810B50A4B826A9A426E
:100FA0000ED000F1280400212046FEF70FFD04209A
:100FB0003AF059FA20460121FEF708FD012010BD44
:100FC0000020FCE7B85607082DE9F04104460E461C
:100FD00015461F467BB9154B83623046E9B243F094
:100FE0000FF9E0B9114B20462360FFF7BDFF2946FA
:100FF0000F4802F0BDFB80460E4B394648F8283FAB
:101000004046FEF7C7FC00220121404639F0F4FCBF
:10101000384639F0E4F92046FFF7BEFFDDE73046F9
:10102000666043F083F9A586BDE8F081B8560708ED
:10103000E08C08089CC1070870B586B008461146C8
:101040001A4603AB0193104B009303233BF0D6FFEA
:1010500040F2145105983AF053FA40F22E420646F7
:101060000A49039806F026FB0546FEF75BFE044698
:10107000074B29460360BDF810203346FFF7A4FF55
:10108000204606B070BD00BFE04F0708F0BE07085D
:10109000F84F070808B5FFF77FFF20B940F2145159
:1010A000024802F045FB0E2008BD00BFFE8F080875
:1010B00010B50A4C23686BB938F029FF08B9FBF763
:1010C00003FCEFF31182102383F31288BFF36F8FB9
:1010D000034B1A6023680133236010BD2C3D0020B0
:1010E000303D002008B50C4B1A6812B90520FDF7F9
:1010F000B3FF1A68013A1A601B6863B9074B1B6893
:1011000083F31188BFF36F8F38F001FF18B9BDE882
:101110000840FBF7EDBB08BD2C3D0020303D002012
:1011200008B539F061F9BDE80840014601483BF0D7
:1011300088BD00BFE4D10708F7B5184CA568E6687C
:1011400001950025019FECB2A74215D8144CA56863
:10115000E66801950025019FECB2BC421CD206EB6B
:10116000C40CDCF804700135B842F4D140F28A4076
:10117000086040F2D3410AE006EBC40CDCF80470CE
:1011800001358742DED1002008604FF44E711160B6
:1011900056F8342012091A6003B0F0BDB49807085D
:1011A000249A070840F2922310B586B00393059362
:1011B00004AA05AB0446084603A9FFF7BDFFDDE915
:1011C0000312059B41B10093204613460A46064987
:1011D0003BF0D3FF06B010BD2046044906B0BDE881
:1011E00010403BF0CABF00BFB1300808B430080857
:1011F0000A46014906F05EBA105107081FB50446B9
:1012000088B10E280FD039F0EDF860B940F2922382
:101210002046039301A903AB02AAFFF78DFF0399B0
:10122000024802F0A5FA04B010BD00BFCD95080831
:101230000E2373B50B600D4601A901F069F8012872
:1012400004460FD9019E3046EFF776FE0246012A8A
:1012500003D9531EF15C2F2907D03146044807F00B
:1012600005F82860204602B070BD1A46EFE700BFBF
:10127000D05607080E2373B50B600D4601A901F087
:1012800047F80128044609D9019E3046EFF754FE7D
:1012900031460246034806F0E9FF2860204602B0C6
:1012A00070BD00BFD0560708F8B5037806462F2B4F
:1012B00000AF6BD0514CD4F8B45045B902203EF089
:1012C00013FB05464E49EFF72FFEC4F8B4502846ED
:1012D000EFF732FE04463046EFF72EFE2044023090
:1012E0003EF002FB04462846EFF726FE294602465A
:1012F000204652F044F82846EFF71EFE054638B166
:10130000231813F8013C2F2B1EBF2F230135235424
:101310003046EFF711FE3146421C601952F02FF8AB
:101320002046EFF709FE002221461346154690425B
:101330002ED145B39B00073323F00703ADEB030D1C
:101340002046EFF7F9FD00236E4619461A46651E42
:10135000204415F801EF01F1010CBEF12F0F04F844
:1013600001E002D0BEF1000F45D1012B2FD115F8BD
:10137000013C2E2B3AD1531E56F823100023A842CD
:10138000E7D1002363542046BD46F8BD1D4D9EE7BE
:1013900011F8016B02F1020E2F2E08BF01337045C8
:1013A00002F1010C0FD92F2E0DD10E782E2E0AD15D
:1013B0004E782E2E07D10332904206D08A782F2AFB
:1013C00008BF45F001056246B1E70125FBE7022BA6
:1013D0000CD115F8013C2E2B08D115F8023C2E2B10
:1013E00004D1012A88BF02F1FF32C4E746F822C0C7
:1013F00061460132C2E761460133C0E70C4000207C
:10140000DC0C08085F2A080837B5FFF74DFF124CBF
:101410006946C4F8B400FFF70BFFC4F8EC00B0B99C
:10142000D4F8F0400CB903B030BD6568012D0CD183
:1014300029460A4806F0F4FE2A46019040F252314D
:10144000204601AB3AF06FF8EDE7E468EAE76B4657
:10145000012240F25231F5E70C400020DC0C080874
:1014600010B5084BD3F8B4404CB12046EFF764FDFB
:101470002146BDE810400246034806F0F7BE66204C
:1014800010BD00BF0C400020D056070837B5FFF74D
:101490000BFF01A9FFF7CCFE28B9144BD3F8F000DD
:1014A000A0B966230193012240F2324101AB3AF028
:1014B0003AF80021054608463BF052FA0446284611
:1014C00002F02AFD38B9204603B030BD4368012B35
:1014D000E7D0C068E4E7042201210CF075F9014669
:1014E00020463BF029F9FDF7A1FCE8E70C4000207D
:1014F00013B5FFF7D9FE01A9FFF79AFE044610B90C
:10150000112003F08DF8012807D0019807F0C6FBE1
:101510000649EFF7FFFC0028F2D0012240F291418A
:10152000204601AB39F0FFFF02B010BDDC0C08080B
:1015300007B5FFF7B9FE01A9FFF79CFED8B9114B1B
:10154000D3F8F00080B901460A200EF00FFC01210B
:10155000031D00F1280243F8041F9342FBD1C1236D
:10156000C36203B05DF804FB4368012B01D0C0687F
:10157000E8E766230193012240F2825101AB39F082
:10158000D2FFEEE70C40002010B50D4B0268044678
:101590009A4214D1406804F10803984201D142F004
:1015A000C8FEA06F38F01CFFD4F8800011F000F8DE
:1015B0002046BDE810409822002151F006BF10BD22
:1015C0009C51070870B58AB0084611461A4604AB0C
:1015D0000193124B009306233BF010FD40F2533170
:1015E000059839F085FF40F277510646049817F0C8
:1015F0007DF90546FEF796FB0446094B324603602B
:101600009DF8243029460293079B0193069B009383
:10161000089B3AF012F920460AB070BD6C510708D9
:101620009C51070838B5437904468B420D4609D0D2
:10163000837913B104483AF04AFA6571BDE838403D
:10164000FDF7B2BA38BD00BF6C08002038B50C46B3
:101650000F4D11461A460F4B9D4201D134F084FEC6
:101660000D4B9D42FAD00D4B9D42F7D00C4B9D4245
:10167000F4D0A3070AD12368AB4207D143F037FE69
:1016800001462046BDE8384045F0BFB838BD00BF30
:101690009CCF07089065070840600708D0560708E8
:1016A000B8560708F7B514460AB1002313701C4B4F
:1016B000DFF87CE0734501D134F056FE194FBB4290
:1016C000FAD0194EB342F7D0DFF868C06345F3D0C3
:1016D00010F003020FD105689D420CD18DF8072050
:1016E0000DF1070244F07BFE14B19DF80730237022
:1016F00080B203B0F0BD0D4B7345DDD0BB42DBD0F3
:10170000B342D9D06345D7D012B14FF6FF70F0E79E
:1017100002689A42F9D144F0BDFCFF28E9D1F4E710
:101720009CCF070840600708D056070870CB070811
:1017300090650708B85607082DE9F04FC36885B0D3
:1017400004468846019223B1458901EB020AD0453F
:1017500003D3019805B0BDE8F08F40463AF0E2FEB1
:10176000064608F101075745B84606D03A4612F832
:10177000013B03F0C003802B10D094F8201039B344
:101780001B2E0DD157450BD23B785C2B08D1002383
:1017900007F1010884F820306361D8E71746E2E7D3
:1017A000E38B002BD3D12369002BD0D0E28A5B8B53
:1017B0009A42CCD2636923B90122204611463AF0FD
:1017C00064F901233246194620463AF0D7F8BEE7BD
:1017D0001F2E00F237810D2E09D8072E09D9083E99
:1017E000052E06D8DFE806F05E4E5A05054B1B2E87
:1017F0005DD0E0682389028B29469A4208D8628925
:1018000001326281028BB3FBF2F502FB15332381B7
:101810006589428B954221BFB5FBF2F302FB13535E
:101820009DB26581A94292D0438BA78BEA18511EC5
:1018300091FBF3F603FB1616418C3944B1FBF3FC24
:1018400003FB1C118E4282D1618B51B95D1EAF42E8
:1018500007D10132B2FBF3F503FB152292B243F03C
:1018600004FE002665892681E26833B2128B0136B8
:101870009342C0F2ED8000236581238167E7002356
:101880002381B6E704260123202200212046013EC1
:101890003AF074F816F0FF06F5D1AAE76389013330
:1018A0006381A6E72389002BA3D0013BE8E701224F
:1018B000ADF80A10781C82455FFA82F927D910F832
:1018C000013BA3F1300CBCF1090F1ED801EB8101E3
:1018D00003EB41030132303B062A19B2EBD19146AA
:1018E000574586D23B785B2B40F09E804FF0020E2E
:1018F00002A83B2E0DD03F2E33D13B1D9A453FF61B
:1019000078AF09F10108B84473E71E46E8E70026FE
:10191000E6E7002309F10102D2B25FFA82F9B9F1D8
:101920000B0F438013D802EB070CE24517D917F8C9
:1019300002C00132ACF1300BBBF1090F06D803EB4A
:1019400083030CEB4303303B1BB2E6E76646BEF174
:10195000010F00F10200CED04FF0010EC9E70026C2
:10196000F5E7443EE068072ECBD801A353F826F0F4
:10197000B71902080319020803190208031902081B
:10198000E119020803190208C51902089119020891
:101990002689D4F80880B0F918B05E4502DBC4F897
:1019A0000880AEE70123202200212046013639F0CD
:1019B000E5FFB6B2F1E723899942CCBF00235B1A59
:1019C00023819EE702299CD100220025114643F085
:1019D0004CFD012229462046A5603AF056F890E7D2
:1019E000BDF90A300029C8BF01F1FF31428BC8BFE1
:1019F00009B2002BC8BF03F1FF33058BC8BF1BB270
:101A00009142A4BF02F1FF3109B2AB42A4BF05F17C
:101A1000FF352BB2458C23810D4495FBF2F102FB7F
:101A20001155ADB265816CE75D2B7FF4E2AE3B2EC4
:101A30007FF4DFAE0123994484F82030E18357FA24
:101A400089F8D6E601233246204639F097FFD0E6E2
:101A5000012320220021204639F090FF04E700BF37
:101A6000002373B50DF107008DF807303EF059FDE6
:101A7000094B9DF80760A0FB035403FB0144430896
:101A800043EAC173E81847F2367344EB5101C6FBD1
:101A9000830102B070BD00BFB2E60E0010B504466F
:101AA00016F0AEFB014B2046236010BDC85207085C
:101AB0000122034B1A700022024B1A70704700BFBC
:101AC0009449002093490020014B1878704700BFCB
:101AD00094490020014B1878704700BF93490020BB
:101AE0000023034A01201370024A1370704700BF9D
:101AF0009449002093490020024B1870024B0120AA
:101B000019707047944900209349002008B53AF0B5
:101B100029F8B5EEC00AF1EE10FA0FD4B4EE400A7F
:101B2000F1EE10FA7DBF10EE103A23F0030040F002
:101B30000200034878BFA0F1FF4008BD0E20FCE77B
:101B40000200400008B53AF009F8B5EEC00AF1EE1F
:101B500010FA0FD4B4EE400AF1EE10FA7DBF10EE89
:101B6000103A23F0030040F00200034878BFA0F1D0
:101B7000FF4008BD0E20FCE70200400008B5FFF75B
:101B8000AFFF10B9024801F0CBFD0E2008BD00BF29
:101B9000099308081FB502AB0193094B0093022378
:101BA00005F06EFC9DF80C109DF80800FFF7A4FFEF
:101BB00010B9044801F0B4FD0E2005B05DF804FB37
:101BC0000C5407080993080810B50022044643F294
:101BD000F66103480CF050F900B1446010BD00BF3D
:101BE000AC07002010B50022044643F61601034856
:101BF0000CF042F900B1446010BD00BFAC070020FA
